:020000040000FA
:20000000C0070000D1060000D1000000B106000000000000000000000000000000000000BA
:20002000000000000000000000000000510700000000000000000000DB000000E5000000A8
:20004000EF000000F9000000030100000D01000017010000210100002B010000350100000A
:200060003F01000049010000530100005D01000067010000710100007B0100008501000068
:200080008F01000099010000A3010000AD010000B7010000C1010000CB010000D5010000C8
:2000A000DF010000E9010000F3010000FD01000007020000110200001B0200002502000024
:2000C0001FB5C046C04600F0EFFA04B00FB41FBD08205A49096809580847382057490968BF
:2000E000095808473C2055490968095808474020524909680958084744205049096809584A
:20010000084748204D490968095808474C204B49096809580847502048490968095808472E
:2001200054204649096809580847582043490968095808475C2041490968095808476020CF
:200140003E4909680958084764203C49096809580847682039490968095808476C20374996
:20016000096809580847702034490968095808477420324909680958084778202F4909687F
:20018000095808477C202D4909680958084780202A49096809580847842028490968095861
:2001A0000847882025490968095808478C2023490968095808479020204909680958084746
:2001C00094201E4909680958084798201B490968095808479C201949096809580847A020A7
:2001E0001649096809580847A4201449096809580847A8201149096809580847AC200F49D6
:20020000096809580847B0200C49096809580847B4200A49096809580847B8200749096896
:2002200009580847BC200549096809580847000003480449024A034B7047000000000020BA
:20024000C0070000C00700000122D84B5A6000BFD74A1268002AFBD0016000BFD44A126809
:20026000002AFBD00022D14B5A6000BFD04A1268002AFBD07047F0B505460E4617460024CD
:2002800006E0A200B158A2005019FFF7DDFF641CBC42F6D30020F0BD0120C043C549086042
:2002A0004010486070470146012292040868904201D9102070470020FCE7F0B505460C4647
:2002C0001646002706E028462168FFF7BDFF2D1D241D7F1CB742F6D3F0BD70B505460C46B5
:2002E0002E460BE0304600F075F9FF2C01D8002401E0FF3C013C012080023618002CF1D16B
:2003000070BD0146012212044868904201D909207047A9484069401C01D10F20F8E70020FE
:20032000F6E7FEB504462068030000F037FA05042B4249598B00201DFFF7E3FF0546002D07
:2003400001D02846FEBDFFF7A7FF0120C00200F041F9042221469948FFF78DFF002801D011
:200360000320EFE708222146944800F06DF9002806D1002192480068FFF766FF00F00CF90F
:200380000320DFE7A768E6686068019031463846FFF7A3FF324638460199FFF78EFFB2006C
:2003A0003846019900F050F9002800D1CAE70320C8E700F0E3F9834800688349086041E01C
:2003C00060680190E668A0680090B2000099019800F03AF90746002F00D1B3E70E20B1E72A
:2003E000201DFFF760FF0546002D01D02846A9E76068002807D1FFF74FFF0320800200F083
:20040000E9F800F0C9F8FFF747FF0120C00200F0E1F8042221466948FFF72DFF002801D009
:2004200003208FE708222146644800F00DF9002806D1002162480068FFF706FF00F0ACF82F
:2004400003207FE700BF00207CE770B505460C46182D04D12068FFF764FF206002E0012091
:20046000206000BF00BF70BDF0B589B05248406903905248806881000398081802900398B2
:20048000000B01900121090302984018401E000B00900124002520462946019A00F0C4F841
:2004A0000022401E9141079106900126002730463946009A00F0B8F80022401E9141059157
:2004C0000490049BDB43059AD243069818430799114307910690374906980860079848602F
:2004E00009B0F0BD70B534484469344885684668AA003146204600F0A7F8002801D0002002
:2005000070BD0120FCE72D484068002801D0012000E000200546FFF7E5FF002807D0FFF759
:20052000BBFE0320800200F055F800F035F8FFF79BFF002D0ED0204846692048846847684E
:2005400021463046FFF7C9FE224639463046FFF7B4FE00BF00F020F810B5184844681A4802
:200560000460204600F0DCF810BD154800680068401C01D100BFFEE710480068002802D067
:20058000042806D101E0FFF7BEFFFFF7E5FF00BFFEE700BF00BFFEE7BFF34F8F0B480C49AB
:2005A000C860BFF34F8F00BFFEE7000000E5014000E4014000060040001000100008000026
:2005C000B8070000BC070000000000200400FA0500ED00E010B50146104B1A68084602234D
:2005E0000F4C636000BF0F4B1B68002BFBD0531C04D0904202D20A4B186101E0084B986068
:2006000000BF084B1B68002BFBD00023044C636000BF044B1B68002BFBD010BD00100010A5
:2006200000E5014000E4014010B5202A04DB0146203A9140002010BD914020239C1A03460F
:20064000E3401943904010BD034610B50B439B070FD1042A0DD308C810C9121FA342F8D00B
:2006600018BA21BA884201D9012010BD0020C04310BD002A03D0D30703D0521C07E000202C
:2006800010BD03780C78401C491C1B1B07D103780C78401C491C1B1B01D1921EF1D1184627
:2006A00010BD70477047704710B500F007F810BD014B1B68DB6818470000002019481A4972
:2006C0007047FFF7FBFFFFF7FBFC00BD20BFFDE71649174C24688C420BD1164B1B6899424F
:2006E0000CD1154B154A1360186810498842EDD00AE0134880F30888124B18470F4A1360BB
:2007000018680A498842E1D080F308880E49884204DD0E48026802210A4302605B681847D2
:200720000346DFE7C0070000C0070000FFFFFFFF000C0000141000100010000000000020B0
:20074000000400206B05000000200020240500400D48704502D1EFF3098101E0EFF30881C7
:20076000886902380078182802D1C046074A1047074A12682C3212681047000000B5054B16
:20078000054A9B58984700BDFDFFFFFF4B04000000000020001000000400000030B4744660
:2007A000641E2578641CAB4204D3635D5B00E31830BC18471D46F8E7000C00000010000017
:20100000F0210020FDB101005D22000063B10100000000000000000000000000000000005C
:201020000000000000000000000000006DB2010000000000000000005D2200005D22000092
:20104000D9B20100DFB201005D2200005D2200005D2200005D2200005D2200005D22000078
:20106000E5B201005D2200005D220000EBB201005D220000F1B20100F7B20100FDB20100BF
:201080005D2200005D2200005D2200005D2200005D2200005D2200005D2200005D22000058
:2010A00003B3010009B301005D2200005D2200005D2200005D2200005D2200005D220000C2
:2010C00000F002F81AF07BF80CA030C8083824182D18A246671EAB4654465D46AC4201D1E9
:2010E0001AF06DF87E460F3E0FCCB6460126334200D0FB1AA246AB46334318477CA301004A
:20110000ACA30100103A02D378C878C1FAD8520701D330C830C101D504680C60704700009A
:201120000023002400250026103A01D378C1FBD8520700D330C100D50B6070471FB5C04605
:20114000C04619F0DEFF04B00FB41FBDF0B44046494652465B460FB402A0013001B50648C4
:20116000004700BF01BC86460FBC8046894692469B46F0BC70470000C1100000826902495D
:201180008161024810447047911100000100000001B41EB400B501F000FF01B4019886462F
:2011A00001BC01B01EBD0000401E00BF00BF00BF00BF00BF00BF00BF00BF00BF00BF00BF53
:2011C00000BFF1D17047000070B505460C46164602E00FCC0FC5103E102EFAD2082E02D3C5
:2011E00003CC03C5083E042E07D301CC01C5361F03E021782970641C6D1C761EF9D270BD74
:201200008307FF22DB0E9A408907090E994000280BDA0007000F0838830828489B001818B7
:20122000C36993430B43C3617047830824489B001B181868904308431860704710B50446E2
:2012400000210120FFF7DCFF00211820FFF7D8FF00210B20FFF7D4FF02211920FFF7D0FF1F
:2012600002210D20FFF7CCFF02210E20FFF7C8FF02210F20FFF7C4FF0221C81FFFF7C0FF85
:2012800003211620FFF7BCFF03211520FFF7B8FF204600F019F8002010BD67210180704729
:2012A00010B500F020F810BD0648704710B500F022F810BD704770477047000000ED00E001
:2012C00000E400E003F9004370B505462D4C08202070A01CFFF7E1FF5920A080294620466A
:2012E00000F0B3FB70BD10B500F0B8FB25490020891E087010BDF8B5224E0446B61E30785E
:2013000001270D46002807D0204660380B2808D8204600F059FF2BE0602CF9D01A4808606A
:20132000F8BD20466C38032803D8204600F08DFF1EE0204670381F2803D8204600F047F942
:2013400016E0204690380F2803D8204600F0EAF80EE02046A0380F2803D8204600F076F81D
:2013600006E02046B0380F2804D8204600F0E2F9286000E02F60602CD2D128680028CFD177
:201380003770F8BD1A0000200130000001202549C003086024490020087007202349C0056F
:2013A0008860704770B5204D04462878A04207D0002C05D0002803D01DA14D2019F0CBFE60
:2013C0002878A0420ED000211E4A18482C70002C1BD01D4B012C06D0022C0DD014A168205E
:2013E00019F0B9FE70BD1160022111605361032109068160416070BD1160032111605361AB
:201400000121C9058160416070BD116011600721C905816070BD10B505A1712019F09BFEA9
:2014200010BD000080E100E02000002000F501407372635C68616C5F63636D5F6161722EFC
:201440006300000000F500408401002010B5A038030019F0A1FF0B070E172028313A414B90
:20146000525C65004B6808788A68194603F0D9F910BD88888A6883B20888194680B203F0F8
:20148000DFF910BD08884C68CB688A6880B2214603F0DAF910BD08884B688A6880B219464C
:2014A00003F0EEF910BD88888A6883B20888194680B203F0FAF910BD88888A6883B20888B3
:2014C000194680B203F034FA10BD08884A6880B2114603F073FA10BD088982B2888883B28B
:2014E0000888194680B203F074FA10BD08884A6880B2114603F091FA10BD08894C6882B20E
:201500000888CB6880B2214603F00AFB10BD08884C68CB688A6880B2214603F01BFC10BDD1
:20152000012010BD10B59038030019F035FF09060F161D242C363F464E0088888A6883B20F
:201540000888194680B204F01DF910BD08884A6880B2114604F051F910BD08884A6880B249
:20156000114604F056F910BD08884A6880B2114604F05CF910BD08884B688A6880B219465D
:2015800004F067F910BD088982B2888883B20888194680B204F066F910BD08894B6882B267
:2015A0000888194680B204F07CF910BD08884A6880B2114604F087F910BD888882B20888F4
:2015C000114680B204F0DBF910BD012010BD10B57038030019F0E0FE1B0F15192125282FB3
:2015E000363B4044484C53585F68707881889095999CA2A5AC004A680878114607F019FC1D
:2016000010BD086807F066FC10BD0C790B7B8A680868214607F06FFC10BD086807F000FD00
:2016200010BD07F08CF910BD08884A6880B2114607F034FE10BD0A790888114680B207F040
:20164000C4FE10BD087840B207F0CDFE10BD088880B207F0E1FE10BD086807F0EFFE10BD74
:20166000086801F0ECFB10BD086801F016FC10BD088982B209C9194607F0F8FE10BD05C997
:20168000114607F042FF10BD08884A6880B2114609F0FAF910BD0C790888CB688A6880B2FE
:2016A000214609F0CDFA10BD0B7908888A6880B2194609F07DFC10BD08884B688A6880B2F9
:2016C000194609F0EEFC10BD08884C68CB688A6880B2214609F053FD10BD08884A6880B26F
:2016E000114609F08CFD10BD0B7908880A7A80B2194607F02DFF10BD088880B207F02DFF46
:2017000010BD086807F030FF10BD07F0FCF810BD8A6809C9194607F08CFF10BD07F0DCF8A4
:2017200010BD08884A6880B2114608F05BF810BD012010BD10B5B02805D0B12808D0B2280E
:201740000BD0012010BD088880B20AF056F910BD088880B20AF070F910BD08884B688A68C1
:2017600080B219460AF079F910BD000010B5030019F012FE0A0609060C0C0F0F0606061245
:2017800007F005F910BD09F027FF10BD01F042FA10BD06F075FA10BDFAA1FE4819F0DBFCAE
:2017A00010BD7FB5FC49054603C9019002911320800169468881F94A0F2310460A212838E6
:2017C0000AF043FE0024F6480AF05DFE641CE4B20A2CF8D304200090F04801231A4603A9E4
:2017E000F0300AF05DFA002804D0FF20E5A1533019F0B1FC686800F024FC00211E2208460F
:2018000004F040F907F0C6FA02222421E54801F07FFBE44801222C214C3001F079FBE1493C
:201820000B20B03901F000FA002804D0FF20D5A1673019F090FC09F09FFE02F075F901AB4A
:2018400000220821D8A007F085F9002804D0FF20CCA16D3019F07FFC284602F0C2FC002861
:2018600004D0FF20C7A16F3019F075FCDB218900D04819F045FBCF4801214171022181710E
:201880000621C1717FBD10B5CA4CA078092804D3FF20BCA1A73019F05EFC2078602148435E
:2018A000001900210173417BF722C908C900C91C1140EF22114041730121E1700C3010BD43
:2018C00070B50E4600211C4619801546030019F063FD0723050B1711231D23002246294610
:2018E000304609F096FE70BD22462946304606F098FE70BD22462946304601F0C2FF70BD86
:2019000022462946304603F0C0FD70BD22462946304600F010FC70BD9E489AA1D53819F0F0
:201920001AFC032070BD70B5A24CE078002818D02078602148430019407B00254007400F93
:2019400001190879401E08712078401CC0B22070092800D12570A078401CA0700AF01DFFEE
:20196000E57070BD9348C079002800D08BE7704770B5904DA86800280CD0FFF7F3FF00288A
:2019800062D06022A968FFF71FFCFFF7CCFF0020A860EFE76879002856D0FFF774FF0446D0
:2019A00080484C3001F0C4FA6060002804D1C92074A1800019F0CFFB60680AF0EAF800285A
:2019C0000DD0204606F011FD6078010703D5C008C000401C2BE0734861684C302DE0714853
:2019E00061684C3001F0ADFA00F05AFB00282BD1FFF749FF04466B4801F09AFA60600028F9
:201A000004D164485FA16D3019F0A5FB60680AF0C4F8002814D0606800886080204609F0E6
:201A20002BFE6078010706D5C008C000801C6070FFF779FF9EE75B48616801F082FA99E782
:201A40005848616801F07DFA70BD10B55A4CE160A0605A4800F034FC607010BD56490020BE
:201A60000870704770B5564E0546706A94B00C46401C04D1B06AC0430004000C0BD0306AE0
:201A8000C007C00F2870706A19F03CFAB06A2071000A607114E02B206946087009A96846B3
:201AA0000AF04BF8002804D0972036A1800019F052FB0120287006220AA9204619F0C1F9CC
:201AC0002878002803D06079C0210843607114B070BDF0B53A4C0646206895B00D46374690
:201AE0000837401C08D16068401C05D1A068401C02D1E068401C11D02068314619F002FAB8
:201B00006068311D19F0FEF9A068394619F0FAF9E06831460C3119F0F5F925E02B2069463A
:201B2000087009A968460AF008F8002804D0194814A1553819F00FFB08220AA9304619F0C5
:201B400080F92B206946087009A9684609F0F5FF002804D0A3200BA1800019F0FCFA082239
:201B60000AA9384619F06DF920692E460836401C29D16069401C26D1A069401C23D1E06976
:201B8000401C1FE07372635C686F73745F636F72652E6300DA020000B4B30100D8010020B2
:201BA0006D170000A40B00206E52463531383232000000008807002024000020711900004D
:201BC0008000001012D02069294619F09BF96069291D19F097F9A069314619F093F9E069F8
:201BE00029460C3119F08EF915B0F0BD2B246846047009A909F0A1FF002803D0F649F74802
:201C000019F0A9FA082209AF28460AA919F019F96846047009A909F090FF002804D0EF486B
:201C2000ED49C01D19F097FA0822391D304619F008F9D9E770B5EA4C0546A068002804D08D
:201C40000320E549000219F086FAA56070BD10B50146E44801F075F9E1498879401CC0B2E6
:201C60008871012803D1E048407800F04DFB10BD70B50446DD4816460D46814204D1D7488F
:201C8000D549CB3019F067FA012E05D0E120D249800019F060FA70BD6620207000202072C9
:201CA000A5810120A07370BD70B515460C460646FFF758FE00280CD066210170468001214F
:201CC000017221680161A18881820573FFF72BFE70BD1321304607F078FB70BDC2494968B9
:201CE000884201D210207047032101700020704770B5BD4C05462078002694B0002801D080
:201D00000820E4E6BA4A6260954201D21020DEE66868002809D00921D82804D3C31C9B0819
:201D20009B00834205D00846D1E60320400268600EE0012109074B6B896B4B43AD49511A83
:201D40000122591AD202891A814201D20421EAE700F052FF6178A0680CF04EFBE068401EDD
:201D600007280BD8302269460A70887068460DF088FF002802D009A80CF0FBFC2846FFF7AA
:201D800010FD012020703046A1E6F8B5044696480F464068814208D3002C01D0844204D37E
:201DA000E01C80088000A04201D01020F8BD8C488178002911D0398800914178602251438F
:201DC0000D18287B0C350007000F3B4600222946FFF776FD060004D015E00020388005209D
:201DE000F8BD002C13D039880098814201D90C260DE028783B460007000F22462946FFF706
:201E00005FFD060005D00C2E01D0002038803046F8BD734C6078401CC0B26070092801D145
:201E200000206070A078401EA07068784107490F01290ED0022906D003291AD066496E4828
:201E400019F089F9E3E7C006E1D46868FFF7FFFEDDE7644869684C3001F073F86079401CA1
:201E6000C0B260710128D2D15F48407800F04CFACDE7E079401CE071C9E7604A10B5904213
:201E800009D3594A0124A4045268A04201D3904201D3914201D2102010BD00F0FEFE10BD84
:201EA000564B10B5994209D34F4B0124A4045B68A14201D3994201D39A4201D2102010BDC9
:201EC000022803D0102801D0092010BD00F00BFF0028FAD0052010BD484B10B598420DD316
:201EE000414B0124A4045B68A04201D3984205D3994203D3002A03D09A4201D2102010BD04
:201F000000F017FF0028FAD0072010BD10B50446354894B04068844202D2102014B010BD02
:201F20000F2008A9087369460BA809F006FE0028F4D16846007A207068464089608068463D
:201F40008089A0800020E9E710B500290BD0264A5268914202D30B68934201D2102010BDB5
:201F60008A88002A02D001F037FE10BD092010BD10B5224A94B091420ED31B4A01239B0419
:201F80005268994201D3914206D3441E1E2C41D8994203D3914201D21020BFE7012837D109
:201FA00008780024C007C00F002803D003206946887001E06846847038206946087009A96E
:201FC000684609F0BAFD002804D004480CA18B3819F0C1F82046A1E7841B0000AA020000F0
:201FE00088070020A40B002024000020FFFF000000220020000000202104000000C00100D9
:202000007372635C686F73745F636F72652E6300072083E70246203A1F2AF9D806F001FE83
:202020007CE710B5604A5268914201D2102010BD0246203A1F2A02D806F068FE10BD07205C
:2020400010BD70B50546594C002020702046461955484660E01C80088000A04204D0FF200D
:202060005349293019F077F801200007C06AC0430006000E03D14F480068401C03D04E48F2
:202080004E49301AC862A8B20422214604F00DF9002804D0FF204649393019F05CF870BDB7
:2020A000F0B595B03B2008A9087369460BA809F044FD002804D0FF203D49813019F04BF875
:2020C0003F4E00246D4630E02F19B87DC10706D0400704D460004019C08809F0E9FB3948F3
:2020E000807900281FD0B87D80071CD560004019C0880022062109F0F7FB002813D03C2186
:2021000008A8017360004019C1886846C18569460BA809F012FD06000BD0FF202449963008
:2021200019F019F805E0641CE4B268460079A042CAD8304658E5F7B505460078002700098D
:202140000C463E46062804D0FF201949BF3019F002F8287A00280ED0012814D0FF20144903
:20216000E03018F0F8FF0298002C068001D0278066800020FEBD02270926002C10D0A88936
:20218000A080A87B0AE003271426002C08D06888A0802869E060A88A2082287B2072E2E7F7
:2021A00002980680E5E7000024000020002200200020000000100010000000200005004008
:2021C000043000008807002010B56038030019F0E3F80A060A0F13181F252930353A086808
:2021E000FFF786FD10BD05C91146FFF7CEFD10BD0868FFF773FD10BD05C91146FFF73DFEED
:2022000010BD4B6808788A681946FFF749FE10BD8A6809C91946FFF75FFE10BD0868FFF7BA
:2022200075FE10BD08884A6880B21146FFF78CFE10BD05C91146FFF79BFE10BD05C91146A0
:20224000FFF7EFFE10BD012010BD0120704700000E4A12680C498A420AD118470B4A12680C
:20226000094B9A4204D101B500F08EFE03BC8E46074909680958084706480749054A064BE5
:202280007047000000000000BEBAFECA6400002004000020F0210020F021002001203F4994
:2022A000400608603E4908603E490A68FF231B029A4383121A430A603849803908607047B7
:2022C00010B502460420384904E0C3005B181B79002B0AD00346401EC0B2002BF5D133A1BB
:2022E000432018F038FFFF2010BDC300CA50002259184A718A7101220A7110BD2A4A00212A
:20230000C00080180171704710B50446042803D326A1522018F01FFF2348E1000C182079C3
:20232000012803D021A1532018F015FF6079A179401CC0B2814200D0607101201749400664
:202340008031086010BD70B5164804250068164E0004800F1B4C02281AD014A1692018F0CB
:20236000FAFE15E02078C10088190279012A07D1427983799A4203D0427982717058804755
:202380002078401CC0B22070042801D30020207028466D1EEDB20028E4D170BD80E100E0B4
:2023A00080E200E018E400E0200C00207372635C736F635F7369676E616C6C696E672E63B2
:2023C000000000003400002010B5EFF31080C407E40F72B6D2484178491C417040780128C2
:2023E00001D10AF0FFF9002C00D162B610BD70B5CB4CE07800280AD10125E570FFF7E4FF4C
:202400000AF0F8F9002804D000200AF0CBF9002070BDC44865714560F9E770B5EFF31080AC
:20242000C507ED0F72B6BE4C6078002803D1BEA18F2018F090FE6078401E60706078002824
:2024400001D10AF0D3F9002D00D162B670BD10B5B348C178002904D000214171C170FFF7B1
:20246000DCFF002010BD10B504460AF0C3F9AC49C978084000D001202060002010BDF8B546
:202480000246A74C0026A6710820042101251027130018F081FF0D080A0C0E101214161EDC
:2024A000262123252800257122E0022001E021711EE020711CE027711AE02020F9E70126D4
:2024C00016E0FFF781FF0AF095F90028FBD002260EE02171A5710BE02771FBE7202000E0D2
:2024E00040202071F6E7FF208FA1763018F033FE0AF08CF9002809D00AF08EF9B04205D117
:2025000030460AF08CF90028FAD02CE001208007C560894900224A60884A9661814B0222A4
:202520005A60856086480269D243D206D517026910231A4302610F466D1C00E020BF78680F
:202540000028FBD030460AF06AF90028FAD0002D04D17B48026910218A4302617149022056
:20256000886000207860A07900280CD00AF042F905460AF09FF8734A002D02D0A260E0604F
:2025800001E0E260A060002E01D100F0A5F8F8BD10B504460AF034F9002805D060490120D9
:2025A000C8704A78521C4A702046FFF768FF10BDF8B5614DA8680026012802D1AE600AF0D4
:2025C000F1F86868012800D16E6028680127544C012812D12E606079002803D000200AF09A
:2025E000E1F866712078002807D00AF003F9002803D0012080070761A770286901282AD1C7
:202600002E6100F05FF8012080074761A079002815D00AF0EFF800900AF04CF800990029FD
:2026200001D0E16800E0A168411A022901DA8A1C11DC0099002901D0E06000E0A060FFF7FA
:20264000C3FE0AF0D7F8002804D0012080070761A77000E02770E868012812D100F032F8E0
:2026600000F030F800F02EF8A078002804D1FF202DA1033018F06FFDEE60A6702670FFF793
:20268000CCFEF8BD10B5264CE078002801D10AF0ADF801208107886100F014F8A0780028C5
:2026A0000BD0254CE068002803D10AF0B8F80028F8D10020E06000F005F800201949C0431D
:2026C000886010BD08B55020694608806A461088411E1180FAD208BDF8B5124819278760EA
:2026E000154900200860C8600AF084F8BE0701240B4D002802D03461AC7000E02C70FFF7F7
:2027000063FE084847600D4928798863FFF7DAFFB461FFF7D7FF0849002008617461F8BD6B
:2027200038000020000300407372635C736F635F636C6F636B2E6300000100400005004093
:2027400000ED00E0FFFFFF7F8107C90E002808DA0007000F083880082E4A80008018C06930
:2027600004E080082C4A800080180068C8400006800F704710B50D20FFF7E6FFC4B204203C
:20278000C043FFF7E1FFC0B2844203D023A11A2018F0E1FC26490120486010BD0121254ADC
:2027A00048031060244B00221A60244A5160244A1060244A11601F49803908607047012115
:2027C0001C4A480310601F4A51601B4A002111601B490860704710B517490868012804D0B2
:2027E0000EA1572018F0B7FC10BD114880680022C0B20A6009F0BEFC10BD10B50E480168E8
:202800000029FCD0FFF7E7FF01200D494003086010BD000000ED00E000E400E07372635CC3
:20282000736F635F68616C5F726E672E6300000000D5004080E100E000D1004000D300400E
:2028400080E200E000D0004030B40121BC48C9020160CD1005604A030260BA4803681B0275
:202860001B0A036004680023240A24020460B6480468240A24020460B448012444608460BE
:20288000B34C23606360A360B24B19601D601A60B14B19601A600121016030BC704710B4AA
:2028A0000121A748CA0202600B0203600C060460A64841608160A94841680029FCD1A44906
:2028C0000020086048608860A24802600360046010BC704701219F48C9020160C9100160DB
:2028E0007047002805D0012805D0022805D19C4870479C4870479C48704710B59BA18B20A9
:2029000018F029FC002010BD70B500219E4C9F4D9F4A8F4B002808D001281DD0022822D08C
:2029200092A1B32018F017FC70BD01200004A060A86011601960974BC2039A60964A9060C1
:202940007F4A001210609548016086480160944801609448017070BD01204004A060A8609B
:202960005160596070BD01208004A060A8609160996070BDF8B59446834A8B4F834D0024DA
:202980000126002808D0012832D0022840D077A1E82018F0E0FBF8BD891E0902090A01200D
:2029A000000490603C6468606C4A1164012B1DD000217C4A7D4B51706146DC63DE637C4B19
:2029C0005C6002249C6004241C61744B3D31196073490E605F4B891519606F4B58605E48CB
:2029E00001606C49C00548601670F8BD0121E0E70120704E4004704F012B04D13464506005
:202A000068603964F8BD9060346468603964F8BD01206A4E80046A4F012BF4D1EEE74F4887
:202A20004068704770B54A4D28680026564C012806D1A068C00303D501200004A0602E60CD
:202A40006868012809D1A068800306D501204004A0606E6001200AF0B9FEA868012809D125
:202A6000A068400306D501208004A060AE6002200AF0ACFE70BD10B54A490878002818D0A2
:202A80000120444AC0079060434AC00B90602C4A00121060414A00201060324A1060404AFF
:202AA000106008704A78002A02D048700AF08EFE10BD0320FAE70120424900060860704790
:202AC0000120244900060860704701203D4940050860704701201F494005086070473349CF
:202AE0000020C86388151B4908607047410A364AC005C00D5043801C5143400A081870472A
:202B000010B4324C430B63431B0C5C020C602E4C6343C31A2E485C0258432B4B400D4343D9
:202B2000E31A0124DB0324041B191B1613700A681018086010BC704710B50AF01BFF10BD5A
:202B400080E100E008E400E018E400E000B0004040B1004080E200E000E100E000B5004073
:202B600048B100404081004044B100407372635C72656D5F68616C5F6576656E745F7469AD
:202B80006D65722E6300000000B3004040B3004040B5004000F50140008300404085004007
:202BA000008200404800002000B10040C08F00400085004004B1004004B5004008B10040BF
:202BC00008B5004000E200E0093D0000378600006F0C010010B50AF0B9FE10BD0020044907
:202BE000C863012001218140024A116000BF7047C01F004080E200E010B50DF05DF909F001
:202C0000F7F9FEF7C3FB0FF0F5FA0DF08FFF0DF01BFF10BD70B50C46054603F0A7FA2146F7
:202C200028460EF0C2FF70BD70B50D46040012D0002D10D02101284618F060F9102254490F
:202C4000284618F0FEF8524801210838018044804560002070BD012070BD70B54C4E0024A4
:202C60000546083E11E0716820014018817BAA7B914209D1C17BEA7B914205D10C222946CB
:202C800018F0B2F8002806D0641C30888442EADB0020C04370BD204670BD70B50D46060060
:202CA0000AD0002D08D03A4C083C20886188401C884203D9042070BD102070BD3046FFF7BE
:202CC000CCFF002801DB401C0AE020886168000140181022314618F0B4F82088401C208014
:202CE0002870002070BD70B514460D001FD0002C1DD00021A170022802D0102817D108E025
:202D0000687829780002084311D00121A17010800BE02846FFF7A1FF002808DB401CA070DB
:202D2000687B297B000208432080002070BD012070BD70B5054614460E000AD00020307012
:202D4000A878012807D004D9114908390A8890420BD9012070BD002C04D028782070288865
:202D6000000A50700220087010E0002C0CD049680001411810222046103918F062F8287809
:202D800020732888000A607310203070002070BD540000205A4910B5884207D301218904C7
:202DA000884205D357490968884201D2102010BD0146012005F0CBF810BD30B5044693B067
:202DC00000200D46079014210BA818F099F81C21684618F095F86A46112010770020507799
:202DE000107802210843107007A80C90012008AA907245486A4610850AA80B9020881084E2
:202E000060885084A0889084E088D084907FF9210840801C4008400090770820908610878D
:202E200008A80F9010AA0BA9684600F05CFF002803D110A800882880002013B030BD3EB535
:202E400004460820694608802D48844207D301208004844205D32B480068844201D21020CD
:202E60003EBD2146012005F072F80028F8D12088694688806088C880A0880881E08848810E
:202E800005F065FE01AB6A46002101F0BBFB694609880829E4D003203EBD1FB50446002035
:202EA000029008206946088115480391844207D301208004844206D312480068844202D2EF
:202EC000102004B010BD05F042FE014602AA0F4801F02EFD0028F4D169460989082901D076
:202EE0000320EEE769460988218069464988618069468988A1806946C988E180E1E700008E
:202F000000C0010028000020042A0000FFFF000010B5031D03600020521E04E05C181C60D0
:202F2000401C2346C0B29042F8DB0020186010BD01460A680020002A02D0104612680A6041
:202F4000704702680A6001607047000010B501462022094817F075FF07490020C8770846B7
:202F600010BD0649012048610548064A0168914201D1002101607047B00E00200005004064
:202F800064000020BEBAFECA0C4908784A78401CC0B2904200D008707047094A074820BFB6
:202FA00040BF20BF4178037843701368002B02D103788B42F3D00020704700006B00002066
:202FC00000E200E00A4A022151600A490B68002BFCD0906008680028FCD0002050600868B6
:202FE0000028FCD070470120000740697047000000E5014000E40140704770477047704777
:2030000010FFFFFFDBE5B15100C001006700FFFF03B40148019001BD09000020002803D048
:203020008178012939D101E0102070470188FE4A881A914233D01BDCFC4A881A91422ED0A2
:203040000BDC00292BD00320C002081A27D0012825D001210903401A07E001281FD0022898
:203060001DD0FF281BD0FF380138002815D116E0FF220132811A904211D008DC01280ED050
:2030800002280CD0FE280AD0FF2806D107E0012905D0022903D0032901D0002070470F2045
:2030A000704700B50B2826D009DC030018F074F90B1D2125251B25292325271F1B00112840
:2030C0001BD008DC0C2816D00D281CD00F2814D0102808D10FE0822809D084280FD0852810
:2030E0000FD0872811D0032000BD002000BD052000BDCF4800BD072000BD0F2000BD0420FA
:2031000000BD062000BD0C2000BD0D20800200BD70B500290BD0CB1FFA3B81241E46CDB2EA
:20312000112B1BD2012805D0022806D009E0002010701DE0FF20043001E0FF200330814299
:2031400018D0330018F028F911161313161316161316161613131313161316000846FF3824
:2031600081381F2803D9FF39FE39022902D81570002070BD1470072070BD00B5030018F095
:203180000BF9060406040C080A0C002000BD112000BD072000BD082000BD032000BD007801
:2031A0000207120F04D0012A05D0022A0AD10EE0000907D108E00009012805D0022803D04F
:2031C000032801D00720704708700020704706207047002807D0012807D0022807D00328BE
:2031E00007D007207047002004E0112002E0212000E0312008700020704738B50C460500FE
:203200004FD06946FFF7CBFF002822D12088032189028843694609788907090D0843208022
:203220006946681CFFF7BBFF002812D12188032000038143684600788007800C01432180EF
:20324000A8784007820F2020012A03D0022A03D0072038BD814300E00143218088B2010554
:20326000890F08D0012189038843A9780907C90F89030843208080B28104890F0AD0A9789B
:203280004004C906C90F400CC903084320808004800F02D12088400403D520884021084342
:2032A0002080002038BD70B504460020088015466068FFF7A2FF002815D12189A0898142E4
:2032C00010D861688978C90708D001214902884208D8491C17F01EFE298009E0FF21FF3113
:2032E000884201D90C2070BDFF30FF3003302880002070BD10B5137804785B08E4075B00D6
:20330000E40F23431370FD2423400478A407E40F640023431370FB24234004786407E40F8A
:20332000A40023431370F724234004782407E40FE40023431370EF2423400478E406E40F4C
:20334000240123431370DF2423400478A406E40F6401234313700078BF244006C00F2340BF
:20336000800103431370002906D00878C10701D1800701D5012000E00020C0015906490EF5
:203380000843107010BD30B50A8803239B0204889A4323059D0F02D1A3049C0F01D09B0F7E
:2033A00000E001239B021A4303230A801B039A4303889804840F02D11805830F01D0800FC8
:2033C00000E00120000302430A8030BDF3B593B00D000FD0139800280FD01221284617F0FC
:2033E0008DFD03AAFF21012003F0D5F80024264637467AE0102015B0F0BD0720FBE76846D5
:20340000807D01280BD16846818A0520C002081A10D0012810D0022812D0032812D0042CB6
:2034200014D0052C15D113E0022900000128000003300000012400E002246846468A08E086
:20344000032406E068460424478A02E0052400E006246846418A1398814246D12C74002ED7
:2034600041D00DAA0EA9052002920191009010230022FF21304603F02FF9002823D1684622
:20348000808E2A46C0B20EA9FFF72DFC00281AD1AE81002F27D00DA9052008AE029100904A
:2034A000132300220196FF21384603F015F9002809D16846808EF11CC01EC0B22A1DFFF726
:2034C00012FC002801D0032095E708A88178427808021043E881062C05D16846807DA87250
:2034E0006846808A2881002085E703A803F05CF8002884D0FFF7D5FD7DE7002805D0FE4A00
:20350000012903D0022903D003207047518800E09188814201D1002070470720704770B595
:203520000C4605461C21204617F0E8FC00202080002D08D0012D04D0F0A1F54817F00BFEBB
:2035400070BD062000E00520A07070BD70B592B01546064601206A461071107453740846DD
:2035600008300395029048889082FEF7FBF9040019D06580172069468883203600940AABBC
:203580007178023307AA01A80EF017F906466078000701D5FEF7C7F9002E0AD03046FFF77B
:2035A000ECFD12B070BD1321284605F00EFF0320F7E708A800906846838B042201212846DC
:2035C00007F0B3FEEDE770B506468AB000200D4607900590069003A904900524024602914B
:2035E0000190102300942946304603F075F800280DD108A804A90091029001946846838959
:2036000000222946304602F083FE002801D0FFF748FD0AB070BD10B50EF0D5FA10BDF0B511
:2036200089B000260546059600780C460827030017F0B2FE0CFD070C390B75759BBEFCD320
:20364000E3FD68680A38FEF702FB07E1A888002280B20421009008F067FB0290002C04D079
:20366000AB48A6A16E3017F076FD0298002804D1A748A2A16F3017F06EFD029800990830B3
:203680000DF0D0FCFEF76EF9040007D060783843607000986080FEF746F9E1E013210098CE
:2036A00005F093FEEAE0002C04D1BD2093A1800017F051FD60880022042108F035FB0090EC
:2036C000002804D192488DA1883017F044FD0099002008802A7994461EE0C3005B199B68EF
:2036E00007936B469B8B1A0708D5DA0606D56046C20050194038C08F088006E05B0409D55D
:203700000871C2005019C08848806078384360700226A3E0401CC0B28445DED89EE0E888EC
:20372000694608800090002C04D1794873A1983017F011FD2878062813D10098C00B10D01A
:2037400060880022042108F0EFFA060004D170486AA1A23017F0FFFC00203071A888708006
:2037600039E060783843607078E0002C04D1684862A1B43017F0EFFC60880022042108F004
:20378000D3FA0090002804D161485CA1B73017F0E2FC009808300EF068FA0121484002D1B0
:2037A000E888C00B5AD0009861880226C180D8E7002C04D1564851A1D03017F0CCFC6088B3
:2037C0000022042108F0B0FA002804D150484BA1D33017F0C0FC0226C3E7002C04D14C4852
:2037E00046A1DC3017F0B7FC0226618801222046FEF73EFA01200590B3E7A889002280B280
:203800000421009008F090FA0746002C04D040483AA1EE3017F09FFC002F04D13C4837A1A1
:20382000EF3017F098FC6868029001E009E010E0288969468881012202A90098FEF734FAC0
:203840000CE0002C8DD16D202CA1C00017F083FC87E72F4829A1FE3017F07DFC002C0DD0EC
:20386000607800070AD50598002807D1842020702046582229460830FDF7A6FC304609B06D
:20388000F0BDF7B50C460546007A224688B00A320492921C01920027811E16323E460292DF
:2038A0000B0017F079FD08F405F348488ED0F2F368880022042108F037FA0190002803D1CC
:2038C0000EA1144817F047FC01980088002802D05227072600E151271E26002C70D06888D9
:2038E000A0800120A071019804990079C0004019C089FFF76BFD0FE0400C00207372635C08
:2039000067617474735F636F72652E63000000006F0200008603000000287DD10198007969
:20392000C0004019C089208101980079C0004019408AA083F0E0698A0091062820D1E88988
:20394000C00B1DD008462230512786B2002CC5D0A8890199FFF73AFD002872D16888A0802B
:203960000220A071A88920810120A072288AE083009820846969009A029817F062FACBE0AA
:2039800008462030502786B2002CA7D0A8890499FFF71CFD002854D16888A080A889E0806C
:2039A000287A06280AD002202072288AA0830098E083204669692030009ADEE70120F3E7F7
:2039C0008FE068880022042108F0AEF90690688A00900698002803D1FD49FE4817F0BBFBA7
:2039E000069808300EF041F90121484002D1E889C00B25D000985127223086B2002C7AD0FB
:203A00006888A080A8890199FFF7E0FC002818D10220A071A88900E013E020810420A072DA
:203A2000288AE083009820846969009A029817F008FA0699002008710698A98941806BE012
:203A400003200BB0F0BD688804F0DDF9009068880022042108F068F901900098002804D1DB
:203A6000DC48DB492C3017F076FB0198002804D1D848D7492D3017F06EFB0198D649C08887
:203A8000884205D05127222604E01EE03FE035E050272026002C2ED06888A080502F07D064
:203AA0000220A0712146287B0831FFF738FD33E0287BA11DFFF733FD6A8800230199009884
:203AC000FFF744FD0028BCD126E0C449A889C988814207D154270626002C0CD06888A0800B
:203AE0001AE008E053270826002C04D06888A080A889E08010E00A98068013E055270726E7
:203B0000002CF8D0A889A0800020A07104E08D20AF49C00017F01FFB0A98002C068001D0A0
:203B20002780668000208CE7AC4900200870704730B585B00C4601F0DBF90546FF2804D1A9
:203B4000A448A349953017F006FB0020208020716080401EE0802046294608300DF056FA77
:203B60006A462946012002F016FD102412E06846808800070ED56846C0882946FFF723FDBF
:203B800068468188FF2321438180C0882946019A02F02CFE684602F007FD0028E7D005B041
:203BA00030BD0A46014610B5104608300DF042FA10BD70B505460022042108F0B5F80400C8
:203BC00004D184488249B73017F0C5FA2046294608300DF027FA70BDF0B591B00C460746EF
:203BE00004F011F9050005D02878222804D2082011B0F0BD7A48FBE700220421384608F036
:203C000093F80646002C02D0A08800280CD00120694608710220087400204874002C05D0DF
:203C2000A0880883206802E00920E1E7088305903046083003970290FDF794FE040018D00A
:203C40006780172069468883203500940AAB6978023307AA01A80DF0B0FD054660780007AA
:203C600001D5FDF760FE002D09D02846FFF785FABEE71321384605F0A8FB0320B8E708A8D2
:203C800000906846838B04220121384607F04DFB0021C943F180ABE7FFB585B00E9E77880F
:203CA000384604F0B0F8054600220421384608F03BF80446002D03D145494A4817F04BFAF8
:203CC000002C04D147484249401C17F044FA0834089869460394C1C105A80DC820356978CC
:203CE0000DF0DAF9CBE5F0B50446002099B00D4601460D9010A88181164601818180374A9B
:203D000068469180018510A8018068460187818581841078012808D0022806D0032804D05C
:203D2000042802D0082019B0F0BD2F4A944273D32E4F0121890438688C4201D3844278D3D3
:203D4000294A954275D3012189048D4201D385426FD36168002913D0234A914269D3012202
:203D60009204914201D3814263D360892189884203D801225202914201D90C20D3E70D902E
:203D800016AA0EA92846FFF78EFA0028CBD1686880784007800F02280AD16846008F800498
:203DA000800F05D02869002802D03968884240D30AA92069FFF721FA0028B4D120690028EB
:203DC0001CD0607880076846008D14D580040FE0FC380000EE030000FFFF0000400C002072
:203DE000023000000C05000000C0010028000020800F68D002E08004800F64D16846008D4B
:203E0000810618D58004800F606806D0002812D0396888420DD302E00BE000280BD0FE4911
:203E2000884206D301218904884204D33968884201D2102077E709A96069FFF7DEF9002853
:203E40009CD16069002808D06846808C0105890F012938D18004800F35D00BA9A069FFF7D6
:203E6000CCF900288AD16846808C80062BD46846808D810627D4A169002906D00105890FD7
:203E8000012920D18004800F1DD0E068002804D00078002817D01C2815D204AA611C204680
:203EA000FFF728FA0121890210A80180012768468773DA49818104AA033217A92868FEF7E7
:203EC00038FF002801D007202DE710A8007F15A9C01CC2B200200C920190FF3200900346D9
:203EE0000291FF3203A80332109902F0ACFA002826D110A9888A0F902A892969C84801916D
:203F00000092029010A90A8B6B8928680E9902F09AFA01007ED1C2480025001F8188684629
:203F20004174090A8174052104A86A4623C210A82A46FF21808A0C9B02F0EAF9002802D095
:203F4000FFF7AFF8EFE66846007C0322C1090020920290430122920280181490002928D03B
:203F6000014610A8018068462921877309028181058608A8007C0023410860784900C007B7
:203F8000C00F014308A80174FD2001406078A54A8007C00F4000014308A801740CA90220EE
:203FA00001910090029503A8109902F04CFA010030D16068002828D0206900280DD10AA990
:203FC0000EA8FFF7E0F96078800706D46946088D0321090388436946088590496846877327
:203FE000FE3181818F492089891E16F093FF62680D9811AB0192009002930A46002303A8CF
:204000000A9902F020FA010004D12078C10603D4800600E085E02AD56846058660690028F1
:204020000DD109A90EA8FFF7AEF96846818C03208002814301208002091868468184694653
:20404000888CC82108436946888474488F73FF30888112AA0CA902200292019100900023FB
:20406000704A03A8099902F0EEF9010059D12078C00729D068460586A06900280DD10BA9E1
:204080000EA8FFF780F96846818D032080028143012080020918684681856846818D402042
:2040A00001436846818587735F49818113AA0CA9022002920191009000235A4A03A80B9904
:2040C00002F0C1F901002CD1E06800282DD010A814990180544968468773491C8181E168EE
:2040E00008A80A78027449784174E0684122418868464186E0680023017908A80175E06866
:20410000D200C18808A84175090A81750CA8072101900091029503A8109902F094F90100AC
:2041200003D00F9800F0E8FEFDE53D480321001F0170002E0AD08088308010A880887080A4
:2041400010A80089B08010A88089F0800020EAE530B501248BB015460B46012802D00228B8
:204160001CD104E0684605218473C90203E02B4968468473891E8181002B12D003210020E2
:20418000890288430121890240186946888405AA04A91846FEF7CDFD002804D007200BB0B2
:2041A00030BD1020FBE76A46127C1D480092801E05A9FF3201910290FF32002303A80332F6
:2041C000099902F040F9002802D0FEF76AFFE6E71348001F002D01D041882980047000206F
:2041E000DDE770B592B00446012608A886700F496846018410AA08A93046FFF7A9FF00284B
:204200004ED12078064DC00700242D1F002849D01C2168460CE0000000C001000328000059
:20422000440C002003020000032900000118000016F066FE68460178202001436846017090
:2042400008A88670F9496846018411940794817FF92001406846891C817700200146684649
:204260000177002001466846417704218185C485018607A80A9011A80D9008A809900EAA5E
:2042800009A96846FFF72FFD002809D16846008FE8806846808F2881401C68812C7000208E
:2042A00012B070BDEC802C8110A80088F4E7F7B5DF4900260A789EB0012A04D0022A02D014
:2042C000082021B0F0BD4A88824201D00620F8E71F98824201D10720F3E7012210A98A75A3
:2042E000D4488882002003239B02014699439302CB1810A90B8669468A81CF4ACA8118A9F1
:20430000887110A9888419A904916946CA820690FF20087503A802F06AF90024254627465F
:2043200008AA052103A802F065F9002810D082286FD1002C6FD0002D6DD010A88480C580E2
:204340000021017418A8807B11AC012865D06DE008A88079002F21D0012857D16846818CCF
:20436000B44881421CD113AA0DA905206B4607C36846408C10230022FF2102F0ADF90028CF
:2043800068D110A88089042801D006284CD16846818E1F98814239D10F2092E7012835D1C3
:2043A0006846808C0521C902884202D0491C88422CD19F4841886846408C814201D10127A3
:2043C00000E00027002C01D0002D10D01F9988421CD113AB0DAA05216E460EC604461023BD
:2043E0000022FF2102F078F9002833D101E035460CE010A88089022801D0102814D1C0B259
:204400001BAA0DA9FEF76FFC00280DD16846468C86E71FE0FFE7052053E714A91BA8221DCB
:20442000FEF787FC002801D003204AE710A8007C0023001DC2B210A80274209802900194C2
:20444000009215A81C9901F0FEFF002802D1784902220A70FEF725FE33E710B50B46401E6A
:2044600086B084B203AA00211846FEF743FF04AA052103A802920191009001230022FF21D2
:20448000204601F045FF04466846008A012804D06D206A49000116F05EFE2046FEF701FE05
:2044A00006B010BDF0B5624F0446387887B00E46032804D0042802D0082007B0F0BD04AA67
:2044C00003A92046FEF7EFFE0500F6D1606880784007800F02280DD1684680898004800FB4
:2044E00008D02069002805D055490968884201D21020E2E7208905AA6B46216907C36946AD
:204500000A8A63892068039901F09DFF002802D0FEF7C7FDD1E7002E02D06846808A308097
:20452000042038702846C8E738B50C00054609D000236A46FF2102F031F9002804D0FEF775
:20454000B0FD38BD102038BD69462046FEF755FE0028F8D1A078FF21C307DB0F2846009A52
:2045600002F044F9EBE73EB50C0009D002AB6A46FF2102F013F9002804D0FEF792FD3EBD6C
:2045800010203EBD0321204616F0B8FC6846008801A90005800FFEF71CFE00280BD1684677
:2045A000007920706846008801A98004800FFEF710FE002801D003203EBD684600796070EE
:2045C000A278EF20024068460088C10B09010A43F7210A404104C90FC9000A43A270F92156
:2045E0000A40800601D5022000E00120400069460243097A50084000C907C90F0843A070A0
:2046000000203EBD7FB514460522019203AD029500930A462388FF2101F07AFE6946898918
:204620002180FEF73EFD04B070BD0000052A0000400C002002280000FFFF0000FC380000D1
:2046400028000020F3B5002799B068460C4607873D4600291DD0E068002806D0A06800285D
:2046600017D001886A4611870780199803F0CBFB002811D0007822287ED3199800F038FCA0
:20468000009000220421199807F04EFB060009D104E010201BB0F0BDFC48FBE7FC49FD4836
:2046A00016F059FDA078012803D0022801D00720F0E72088002808D0401E80B203AA009913
:2046C00001F069FF002859D11DE0F048401CE1E76946498A228891420BD26846807D00252A
:2046E000012810D16846808AEB4988420BD1012509E0914203D1002D2AD06D1C01E0022DA8
:204700000BD0032D04D203A801F04EFF0028DFD082281BD0002831D11DE06946897D01295D
:20472000F1D16946DC4B8A8A5B1ED11A9A420FD005DCDA48101A0BD00128E4D108E00129B6
:2047400006D0FF390129DED10325E1E7022D15D10D2080029EE7E068002816D00EA9052205
:2047600002910192009069460B8FA2882088FF2101F0CEFD002800E01DE002D0FEF791FC33
:2047800088E76846A168008F08806846008AC00601D5C3487EE70798002803D06846008BC5
:2047A000022801D0032075E70798A1780078012903D0800710D408206CE7C007FBD00022B8
:2047C0000721199807F090F8002802D00725022004E0AE48801C5DE70225032008A908700C
:2047E000218868468185199808360A90099617216846818712AB02330FAA052108A800972E
:204800000CF0DBFF002802D0FEF7B7FC42E710A800906846838F04222946199806F085FD31
:2048200038E770B5064615460C460846FEF7F6FB002804D12A4621463046FFF789FCF3E669
:2048400010B5FFF734FD10BD70B51E4614460D0014D0002C12D0616800290FD00121FEF7D5
:204860004CFE002809D12068FEF7D8FB002804D1324621462846FFF736FAD5E61020D3E688
:2048800070B515460C000ED00221FEF736FE002808D12068FEF7C2FB002803D12946204656
:2048A000FFF700FEC0E61020BEE6F8B506467D480D46016814468A4231D36068002808D01E
:2048C000794A90422BD301229204904201D3884225D37648864204D0304603F094FA0028AB
:2048E0000CD0304600F004FB0646284600F0BDFA002804D16068002802D012E06348F8BD05
:2049000000236A463146284601F048FF002802D0FEF7C7FBF8BD68460088800601D4102080
:20492000F8BD6188224628466368FFF76BFEF8BDF7B55C4E0746306886B01446824202D2C1
:20494000102009B0F0BD384600F0D2FA05465748874201D0FF2D08D0002304AA2946079820
:2049600001F01CFF002826D101E04848E9E76846008AC00601D54A48E3E703A9002002913C
:204980000527019000976288484B2946079801F0A3FE00280FD161683268914208D30191FB
:2049A00002900097238862882946079801F094FE694689892180FEF774FBC2E7002907D039
:2049C0003B4B0A881B899A4202D83048401C704738E610B586B004236C46A382344BDC88E0
:2049E000002C07D01B898B4201D2914204D92748401C55E5062053E56B4619825A82002114
:204A0000009101911C800221997005A9029104A903916946FFF716FE42E5F3B50C4685B01A
:204A2000812069460873002C1AD0059803F0EBF9070017D03878222868D3059800F058FA1F
:204A4000049000220121059806F04EFF00280BD000220421059807F067F905000AD105E09B
:204A600010202AE5094828E5112026E50849114816F071FB284608300CF0F6FA06462078CB
:204A8000012819D0022838D0072016E502300000FC380000E108000003280000002800000E
:204AA000013400002800002000C00100FFFF0000400C0020840A0000A18803AAFEF728FBD2
:204AC0000028CED1B00721D56846007B00281FD1A079C0071CD0E068002205216B4607C34A
:204AE000638922896888049901F012FC6946087300280DD0FEF7D5FADFE4A18803AAFEF712
:204B000007FB0028ADD13420064201D10820D4E46846037B29463846059AFEF717FDCCE42E
:204B2000FFB597B0002001901F4615460C460E46179803F068F9002804D00078222803D2CD
:204B40000820A7E5F348A5E5B80801D00720A1E5032F00D10027179800F0CAF90890002C4E
:204B60001BD0022D77D3EC48006884427CD361190091012902D0491E814275D3AD1EAAB280
:204B80002146E6480DF0F0F800991E394A7F0B7F11021943884267D1ADB2E148B90702D5C8
:204BA0000189491C00E0012189B20091F90701D0078900E0D94F03AA0899009801F0EBFC11
:204BC0000DE0F078B1780002084310284CD80199091D401880B20190A84245D82618002E60
:204BE00060D0707831780002084300998842E8D358E06946098A0A0754D5002C3FD0019AFF
:204C0000A618121D92B20992F278B37812021A439446102A28D8099A6244AA4224D8727893
:204C2000337812021A4390421ED1C8061ED509980AAA052120186B4607C370783178000215
:204C4000084363460022089901F062FB002803D0FEF727FA1EE507E0F078B1780002084376
:204C60006946098D884201D00B2013E5F078B178000208430999401880B2019006E0C906E1
:204C800004D50899FEF79FFC0028E3D16946088A1021884369460882488AFF23049A089985
:204CA00001F0A4FD03A801F07FFC002803D16846408AB8429DD900220421179807F034F84E
:204CC000040003D19749984816F045FA20880028C0D0012108A80170017300264673218858
:204CE0006846018620460830099017980A90FCF739FE05001BD01798688017206946888060
:204D000010AB023301AA052108A800950CF055FD07466878000704D583488249223016F044
:204D20001AFA002F09D03846FEF727FAB2E41321179804F04AFB0320ACE40EA8009068466A
:204D4000838804220121179806F0EFFA00288CD126809FE4F0B500248DB01F4615460E46AA
:204D6000002A04D0B90804D007200DB0F0BD1020FBE7032F00D1002700F0BAF80390FF2877
:204D800004D06749B80703D5488902E06148ECE70120FA0702D04989491E00E05F4906AA64
:204DA0008FB2039901F0F7FB38E06946898B090734D504AB05210022029300910192574BED
:204DC000039901F089FC002821D1002E21D06A46128A2988A2183019121D914234D36946D0
:204DE000CA8B0270120A42700A8A8270120AC27004A90522001D0092029101906946C88BA1
:204E00000B8A0022039901F067FC002801D00320ABE76846008A2018001D84B206A801F0DB
:204E2000C3FB002804D0822806D0FEF73AF99CE76846C08BB842B8D9002C07D0002E10D0F8
:204E40002988A01C814203D20C208EE705208CE72246314631480CF087FF31190870000A6E
:204E60004870A41C2C8000207FE700B585B06946FEF7ACFA00280AD16846007C030016F01E
:204E80008BFA08052F2F2F2F08080531032005B000BD68468078012807D1684600880321E8
:204EA000C902401A1CD001281AD068468079012806D16846808815214902401A05280FD981
:204EC0006846807A012811D16846018929200002081A05D0022803D0032801D0042805D1AA
:204EE0000F20D4E711A1164816F035F90020CEE710B506F00FFF10BD10B50C4601F01EFBF8
:204F0000002803D009A10F4816F025F92046FEF7C8F810BD0230000028000020FFFF000011
:204F2000400C0020FC3800003F0B00007372635C67617474735F636F72652E630000000027
:204F400022020000BB060000F8B500780C46164610340E36069F022809D0032836D005280B
:204F60007ED0FF20F6A1E53016F0F5F8F8BDCD890A2068430E30188031203880002AF5D077
:204F8000087B9581801FC7B21AE020886168308048780A7800021043F080C8788A780002FA
:204FA00010433081B21C3846091DFDF79CFE002F01D0002802D000203071708008340A36C6
:204FC00028466D1EADB20028DFD1F8BDCD890A2068430E30188032203880002AF5D0087B6F
:204FE0009581401FC7B243E0616822880878F2803279C30752085200DB0F1A43FD231A4059
:205000008307DB0F5B001A43FB231A404307DB0F9B001A43F7231A400307DB0FDB001A4320
:20502000EF231A40C306DB0F1B011A43DF231A408306DB0F5B011A43BF231A404306DB0FE1
:205040009B011A433271C00970718A784B7810021843308132463846C91CFDF744FE00E036
:205060000CE0002802D00020B070308008340A3628466D1EADB20028B6D1F8BD087BCD8949
:20508000801E86B23046083068431030188034203880002AF1D0174695811037E800D68119
:2050A000C01900900DE0208838800098786032466168009815F0C5FE00980834801908377D
:2050C000009028466D1EADB20028ECD1F8BDFFB581B00A9D1E460C46002A05D0607AFF3004
:2050E0000130D080E089108101980E270078030016F052F90B7E0719293541536C7878782C
:205100007E000092087B082805D0032803D091A1954816F020F8378030200FE0009900201D
:20512000888105B0F0BD0092087B042804D08E4888A1143016F00FF8378031202880009857
:205140000028EBD1EDE70092087B042804D0932080A1800015F0FFFF37803220EEE70092BB
:20516000087B022804D080487AA13A3015F0F3FF37803320E2E7087B1746042804D07A48F5
:2051800074A14C3015F0E7FF1020308034202880002FC6D00020B88116E0207B174605287E
:2051A00006D0062804D070486AA1603015F0D3FF1220308035202880002FB2D0E089B881BB
:2051C0000020388201984088F881AAE70092087B072804D064485FA1713015F0BCFF3780AE
:2051E0003620ABE733460095019800F00AFC98E72F2053A1000115F0AEFF92E770B50C46C5
:20520000054602F000FE002804D00078222803D2082070BD554870BD00220521284606F0F5
:2052200083FD2060002801D0002070BD032070BDFFB58BB00D4607461720694608850E9830
:2052400003261446002805D10EA93846FFF7D6FF002834D1002D0BD000220321384606F0DE
:2052600043FB002834D00E980078002830D108E02078092819D00F2823D031A13C4815F05E
:205280006AFF0E98A760801D03AA606002320AA9204600F00CFC002827D0030016F07CF80D
:2052A000071A182323211C1E2300072600223146384606F019FB0028E3D12C48801C0FB0F8
:2052C000F0BD00220321384606F00EFB0028D8D11120F4E70020F2E70820F0E72348401CC2
:2052E000EDE70720EBE70320E9E701A800906846038D04223146384606F017F80028DED180
:20530000002DDCD00E990D70D9E730B587B01D460C46002A11D0042369460B7013888B81FC
:205320005288CA81A2788A7422880A8200236A462946FFF77DFF07B030BD1020FBE7000090
:205340007372635C67617474635F636F72652E63000000007372635C67617474635F636F15
:2053600072652E630000000025020000023000004F030000F3B581B001980C4600780826B0
:20538000030016F009F8125E46461B134A0A0A0A0A0A0A0A0A0A0A0A0A5E002C02D1F6497B
:2053A000F64808E06078304360703BE0002CF9D1F248F149083015F0CEFEF3E70198002289
:2053C0008088052187B2384606F0AEFC0546002C04D07520E849C00015F0BDFE002D04D1B5
:2053E000E648E549143015F0B6FE3946A81D00F055FBFCF7B7FA040006D060783043607037
:205400006780FCF790FA0FE01321384603F0DDFF15E0DA48D849283002E0D848D6492D30AA
:2054200015F099FE002C0AD06078000707D5932020702046582208300199FBF7C5FE002045
:20544000FEBDCE48CC493130EAE710B500210170801D00F020FB10BD0A4610B50146901D5F
:2054600000F024FB10BD70B505460022052106F05BFC040004D1F920BF49800015F06BFE63
:205480002946A01D00F00AFB70BDF7B5054684B00C4600206946088188806F88024605217C
:2054A000384606F041FC060004D1FD20B249800015F051FE002C03D0A7800020E08020812D
:2054C000297A20461230C91E142700900B0015F063FF0FFDFCFB3809A95E657A2FB2C9E9A0
:2054E0009191FB003078012804D0A3497020143115F031FEA9896A46C8000E3090803020AD
:205500001081002C13D0A18100200DE0C100327909190A747288CA8182005319DA894A824E
:205520001A8A401C8A8280B2A1898142EED8F1E002A8009001AB22462946304600F02AFA62
:20554000E8E03078042804D08B49BD20143115F002FEA8890622014650436A460E309080AF
:2055600033201081002CE2D0A18100200BE0062141434F190919FA89CA81BA7C8A743A8A41
:20558000401C0A8280B2A1898142F0D8C2E0307806280BD078491431D72005E03078062831
:2055A00004D07549EB20143115F0D5FDE88969461230888035200881002CB8D0A989A181E2
:2055C0007188E18126E03078072804D06A49FF20143115F0C0FDA8896A4601460E30908070
:2055E00036201081002CA2D0A1812046AA890E30296954E0E8896946123080B23822888071
:205600000A81002C7ED0A989A181287A102807D00221A173E9892182EA89296900983EE079
:205620000121F6E702A8009001AB224629463046FFF78AFC6EE03078082805D04E49FF200B
:205640001431EE3015F087FD6846372187800181002C5FD0A989A18100206082208201205B
:20566000A07357E03078092805D04349FF201431FF3015F070FD288A69461430888037209D
:205680000881002C46D00421A173A989A181E9892182298A618220462A8A1430696915F0D2
:2056A000D0FB37E030780A2804D033493448143115F051FD6846372187800181002C29D016
:2056C0000521A173002002E01FE004E00DE0A081208260821EE002A8009001AB224629465E
:2056E0003046FFF7F4FC15E00CE00D206946392288800A81002C05D00120E0800020208160
:20570000207307E00699088019E01C481A49A43015F021FD6846069980880880002C0ED04A
:20572000684600892080684680886080287A032805D0102803D0112801D000203070002065
:2057400007B0F0BDF7B5568815460F4682B000220521304606F0E8FA040004D1074806496C
:20576000C43015F0F8FCA41D33462A4639460094029800F022FBD4E44053000095030000F5
:2057800013020000F7B58CB00D46144607A90C98FFF734FD002812D1B64E0127002C0FD0A2
:2057A0000321684601701021818208A802460690204605A9FDF7BDFA00280BD007207EE598
:2057C0000821684601708581C68105218774C90201820BE00798A178017121884180684698
:2057E00005218774C90201828581C68102460121079B0C98FFF71CFD61E508B501236A4657
:2058000093709D4B13800A4602236946FFF77DFD08BD08B501236A469370974B5B1C138031
:205820000A4603236946FFF770FD08BD00B587B000290CD002236A4613700B88938149885A
:20584000D18100230421FFF7F3FC07B000BD1020FBE710B5002903D00523FFF756FD10BD44
:20586000072010BD70B588B00D461446064607A9FFF7C4FC00280DD1002C0DD00621684694
:2058800001708581C481079B02465C8006213046FFF7CEFC08B070BD0521684601708581F9
:2058A000F1E710B588B000290BD007246B461C709A81049100236A462146FFF7B9FC08B05A
:2058C00010BD1020FBE770B50024172288B0002914D00D782B0015F05FFD062305051904C1
:2058E0001B231522D21E93B2CA88002A02D08E68002E03D09A4203D90C20CBE71020C9E743
:20590000042D05D08A88002A0AD101E00620C1E7012D11D0022D05D0042D18D0052D23D06A
:205920000720B7E709236A4613704B889381CB88D381896804911DE00C236A4613704B88FD
:205940009381CB88D38189680824049112E00D236A4613704B8893818B88D381CB8813824F
:2059600089680924059105E00E236A461370497811730A2400232146FFF75AFC8AE700B5BB
:2059800087B00F236A461370918100231946FFF74FFC5AE7FEB50078089D1C4616460F4672
:2059A000012803D03549912015F0D5FBF889C0000E30208030202880387B001FC0B20190FB
:2059C000002E1DD0F889B081002516E0E8008419C0190090224641690E320198FDF783F996
:2059E000002802D000202074E08100986D1C008A60820098ADB2408AA082B089A842E5D848
:205A0000FEBD70B514461425049A1D8037231380002C0ED0CA89A2810022628200780828BD
:205A200008D0092810D00A2819D01449144815F092FB70BD087B0C2804D011480F490C386A
:205A400015F089FB012008E0087B0D2804D00C480A49083815F07FFB0420A07370BD087BDB
:205A60000E2804D006480549001F15F074FB0520F3E70000FFFF000002280000545300001F
:205A8000BB02000010B5FE4B586019721A80C90015F036FA10BD00210180704710B5002253
:205AA000D2430280032006F0A8FD10BD7047F0B50E460446017801208840F24999B008409C
:205AC0000090616815460888EF4A904206D0009A002A06D0EB4A521E104202D0012019B054
:205AE000F0BD009A10430880002D12D0002028702178EA1C0027681C01920B0015F04CFC88
:205B000010F30E16233A59616F3CB4B08AB8F2F1F0F320780B28EBD00420E0E70221297003
:205B2000A1890170090A4170032097E004212970A1890170090A41700198E1890170090AC8
:205B4000417005208AE006212970A1890170090A41700199E2890A70120A4A70218A017174
:205B6000090A4171A28AE81DA16915F06AF9A08AC01D73E0082129702178082901D11021D4
:205B80002970A1890170090A41700198E1890170090A41700520308020466A1D02A9103028
:205BA000FDF7C7F800287DD169463088097A401854E00A212970A1890170090A4170032000
:205BC0000BE00C212970A1890170090A41700198E1890170090A4170052030809CE0A08903
:205BE00084464000401C81B2308888425AD3052958D30E202870002008E0236942009B5A73
:205C0000521953701B0A401C937080B26045F4D33180B9E09A48417A002973D0491E4172C7
:205C2000217B4068C9004518A9882868082240180838216915F005F9022168460171002186
:205C4000417128680390A98868460181002101A8FFF790FB0020A880002E00D0308093E05A
:205C60002978802211432970297840221143297029788909890112312970A1890170090ABD
:205C80004170E289E81C216915F0DBF8E089C01C3080287841063FD5C00975D001216846B4
:205CA000017200E02CE0002141723188091D81810495E189019808180590001D0690704814
:205CC000017A68460177002102A8FFF753FB074630880C303080022F06D0002F54D065E084
:205CE0003DE033E01CE05EE065486946097F4268CB00D218037A994202D29188002902D0B7
:205D0000042753E02FE0417A491C41721560308890800020308049E06168A089888033E000
:205D200029788909890116312970A1890170090A41700198E1890170090A4170228A681DFE
:205D4000616915F07EF8208A401D46E728788009800118302870207B687002207EE760687E
:205D60000188090401D4052720E0C088A189884201D006271AE01E202870012030806068E9
:205D800001884904490C0180009800280ED03C4800220088A1688300032006F087FB61689B
:205DA0002078887007E00020308003276068009902888A430280384691E6FFB59FB0289D7B
:205DC0000E46002805D0172803D82A882E4B9A4202D1072023B0F0BD3278530601D4D20924
:205DE00001D00820F6E700226B461A715A7114463278431E1D939BB2189303AB1A9397069F
:205E0000CB1CBF0E1B93821E711C3B0015F0C4FA209011EE66EE74EEB0EED4EEEDEEECEE7B
:205E2000EBEEEAEEE9EEEEEEE8EEE7EEE6EEE5EE90EE05287CD1042168460171A9780172DB
:205E4000F078B27801021143684641813179417170788006800E0C282ED009DC801E0300D9
:205E600015F09AFA0919661C662166246627660012282AD00ADC0E2821D01028DAD121E0BC
:205E80004C0C0020FF710000FFFF000016281FD01828CFD11FE02878800701E02878400721
:205EA000002845DA45E128780007F9E72878C006F6E728788006F3E728784006F0E728784E
:205EC0000006EDE72888C005EAE72888C004E7E728888004E4E728884004E1E72A7892076A
:205EE00026D50328A6D105206A461071487809780002084310811CE129784907F0D50628AF
:205F000016D3717890B2012902D0022992D101E0022100E01021189106216A4611710021AB
:205F2000118102AF189AB11C0237921C1B921AE0B3E04A780B7812021A433A80801E891CCB
:205F40001790BA1C1A911898FCF7CDFE1A991898189A091817986B46801A1A8980B2521C38
:205F60001A811B9ABF1D8242E3D9002886D1E0E028780007B4D51D98694682B207200871CE
:205F800000200881701C0A3111E0437807781B023B430B80C37887781B023B434B806F46EB
:205FA0003B89121F5B1C001D92B23B81091D042AEBD2002A71D1BCE02978C9066DD5022863
:205FC0006BD30820694608710020488170780872844692B2B01C1A9919E089E090E07EE02B
:205FE00067E05BE030E025E019E013E0BCE0437807781B023B430B80831C4B606346D21A43
:206000006F467B8960445B1C92B27B8108319445EDD9CEE7287880063FD5092203E02878F7
:2060200040063AD50A2268460271AA880281189A428107E0287800062FD50B206A461071A7
:2060400018981081039174E02988C90525D5022823D30C20694608710020488170780872DF
:20606000844692B2B01C1A9914E0437807781B023B430B80C37887781B023B434B80031D7F
:206080004B606346D21A6F467B8960445B1C92B27B8108319445E8D98BE763E02988C904A6
:2060A00060D501285ED10D2168460171A98801813FE02988890455D5052853D30E22694699
:2060C0000A71AA880A811B99401F4A78097812020A4369464A818881701D049029E0298873
:2060E00049043FD501283DD10F206946087120E02A88120436D44A780B7812021A43EA80BF
:2061000003282FD332789206920E1B2A26D011226B461A712A880123DB031A432A804A7849
:20612000097812020A4369460A81C01E48811B98039030788006800E1B2809D01D2807D062
:206140000320229906F059FA2888C00BC003288001A82199FFF70EF920463BE610226B4668
:206160001A71DCE70724F7E70824F5E700B597B0032806D16A461070019100216846FFF73B
:20618000F9F817B000BD000010B58B78002B11D082789A4207D10B88002B0BD003E08B7988
:2061A000091D002B08D08B789A42F8D103880C88A342F4D1002010BD812010BD052826D0C7
:2061C000002A02D0012A0DD102E00988090501E009888904890F07D0012918D0022909D0B5
:2061E00003290ED081207047002A01D0032070470220704703280AD0042808D0002804D08A
:2062000007E0042803D0022803D005207047002070470F20704770B51388054614460B8012
:2062200018061DD5FE481022807AA84203D813430B80002070BDA06893430078E840C007A4
:20624000C00E03430B802078A1788007800D0843F44914F05FFEA06869430818401C70BD94
:20626000906870BD37B569468B88138019061BD5EB4C0125A47A9168844209D8FE280FD188
:20628000D80602D5A5406D1E00E000250D7007E085400C78DB06DB0FAC4383401C430C70CF
:2062A00010881021884310803EBDF8B50746C81C80080E468000B04201D08620F8BD082A35
:2062C00001D90E20F8BDD64D00202E60AF802881AA723446E88016E0E988491CE98081069E
:2062E00010D48007A178800D0843CE4914F012FE206800F0BAFA2989401880B22881381AB4
:206300008019A0600C3420884107E5D40020F8BDFFB589B09F041646139DBF0C019309988A
:2063200000F095FA04000AD02078000609D5BC48817A0A98814204D887200DB0F0BD012012
:20634000FBE7224669460A98FFF765FF0690002069460872052D14D0012221462846FFF765
:206360002DFF0028E9D1207840060AD5022168460172099981810188C181068247821298A4
:2063800005900198000404D500273E460125079709E02078A1788007800D0843A149079009
:2063A00014F0B8FD0D46019840040AD50798A84207D12088E1788005800F00020843B04260
:2063C00001D3AE4201D90720B7E7B81980B20190A84201D90D20B0E76846007A002804D01A
:2063E00002A8FDF718F90028A7D10798A8420BD1208803210902884301998905890F09027C
:20640000084320800198E0701498002800D007801298002815D006983A468019129914F060
:2064200010FD224669460A98FFF7F5FE694608881021884369460880224600990A98FFF7A2
:2064400011FF002079E7FFB5754D0C22E8882968504383B00C180D9F7249059814F05AFDBE
:206460000091049800F001FA29682A898E46611A0C310918944651188AB2A988914202D8B6
:20648000842007B0F0BD6A46168A320603D5B20601D58520F5E7EA88521C92B2EA800E9B4E
:2064A000002B00D01A80B20601D5A76006E0604480B22881091A70460818A0602246FE20CE
:2064C0000499FFF7CFFE0598A0700098E07020880599800889058000890F084303210902D9
:2064E000884300998905890F0902084304210843208003988078A07103980088A0800020A5
:206500002073310601D5AC7A00E00124B10600D5002700260EE005210020019102900097E8
:20652000E88831460C9B069AFFF7F2FE0028A8D1761CF6B2A642EED30020A2E7F1B50098DC
:2065400000F085F9060002D00025009C14E00120F8BD204600F07BF90746007831498007DA
:20656000820DB878104314F0D5FC386800F07DF94019641C85B2A4B22948C188601E8142CD
:20658000E7DC00992648491EC1800189491B018100203070F8BD002804D0401E10809170B9
:2065A000002070470120704710B5044601881C48C288914201D3822010BD00680C225143A6
:2065C00042189079A072908820811088D1788005800F00020843A081A078211DFFF71BFEC5
:2065E00020612088401C2080E080002010BD012101827047F7B50546002084B0C0431080EF
:2066000068681746817868468170686801886846018000218171288A2C88A04205D303E017
:20662000580C00200102000004462C8235E0288A401C2882301D6968FFF7A6FD00282AD134
:2066400039889248814201D1601E38806888A04228D33088F1788005800F000208430290F3
:206660006946301DFFF790FD002814D16989874881421BD0002231460598FFF79FFD00282F
:2066800009D16A890298824205D1E968B06814F0ABFB00280AD0641CA4B2204600F0D7F8E9
:2066A0000600C4D1641E2C828220EAE67C80B079B871B088B8803078B1788007800D0843AF
:2066C00078810298B8813946287A32460831FFF7A2FD38610020D4E6FFB585B01C460F4674
:2066E000059800F0B4F8050009D02878000608D56748807AB84204D8872009B0F0BD012053
:20670000FBE707982A468605B60D69463846FFF782FD07460E98052816D000222946FFF70B
:206720004DFD0028E9D1287840060DD501216846017105990181018841818681C48101A8C3
:20674000FCF769FF0028D8D12888AA788107890D11438005800FEA7800021043079A964285
:2067600007D04C4A914204D3611E814201DD0B20C3E7864201D90720BFE7801B82B2A242EB
:2067800000D922461098002800D002800F98002802D0B91914F055FB0020AEE7F8B51D460A
:2067A00017460E4600F053F8040008D02078000607D53748807AB04203D88720F8BD0120D4
:2067C000F8BD224639463046FFF725FD002D0BD02078A1788007800D08432E49884201D263
:2067E000012000E0002028700020F8BDF8B51E4617460D4600F02BF8040008D020780006BD
:2068000007D52348807AA84203D88720F8BD0120F8BD224639462846FFF724FDFF2E14D0C3
:206820002588A178A807800D08431A4914F072FB002E03D1FF31FF31033189B2A170A808A5
:2068400080008905890F084320800020F8BD1049CA88824207D3002805D00C22096850435A
:206860000C38081870470020704703B50846694609888A0607D4090604D50549897A4143B8
:20688000491C88B20CBD00200CBD0000FFFF0000580C002001020000F8B507780D46044659
:2068A000012F19D0072F02D00C2F19D114E0A068216906780B2E0BD0052005F09EFE052E91
:2068C0000ED0782300220520216905F0EFFD07E0782300220620F8E70520216905F08DFEB5
:2068E000002D0ED0002028702946204603F0E2F9FE482978C05D884201D10320F8BD022098
:20690000F8BD0021204603F0D5F90020F8BD70B50E460C462036317901208AB015460029FB
:2069200009D0012905D12978042902D10520107000200AB070BD6068019005A802900D216B
:20694000C01C14F0DBFA032205A8A16814F079FA01203071062069460870206A0490294694
:206960006846FFF799FFE4E770B50C46154620310A790120062686B0002A2CD0012A28D19D
:206980002978042925D169681022A06801F0B5F96868C07B000606D5D44AA0681023103AFA
:2069A000014601F09FF91022A168E06801F0A5F9A068C07B000606D5CC4AE0681023103AF6
:2069C000014601F08FF92E70A0686860E068A860002006B070BD60680190C44820380290E7
:2069E0000120087168460670206A049029466846FFF752FFEDE7027B032A06D0002224239A
:206A00005A540B78092B02D003E0042070470A76CA61027B9300521C0273C15003207047F8
:206A2000F0B50E4615460C462036024631790120072393B000290CD0012924D002292ED08E
:206A4000032904D12978042901D12B70002013B0F0BD01203071606800280DD0A1690B7056
:206A600060684860206988606069C860206A08621046FFF7C0FFEAE7062028702069686065
:206A80006069A86009E029780629E0D102203071042028709548203868600320D7E72978BD
:206AA0000429D4D1A08910280AD9103880B2A081A1681023091805A86A6801F013F923E049
:206AC00010282FD0C2B21020801AA1680DAF1190C01914F0B6F911980006000E06D0401E5E
:206AE000C1B280207854384614F008FA626910230DA909A801F0F6F8102309A905A86A688B
:206B000001F0F0F8032030716068019005A80290062069460870206A049029466846FFF7C2
:206B2000BBFE94E710232269A168E2E7F0B50E460C4620363179012006278FB01546002935
:206B40000BD0012932D0022905D12978042902D10820107000200FB0F0BD217D08A8CA0739
:206B6000D20F02718807C10F08A801716846027041700722801CE16814F063F902A807222E
:206B80000130216914F05DF9606805900AA8069010236A46A16801F0A5F801203071684651
:206BA0000774206A0890294604A820E029780429D1D1062205A8E16914F043F906A8062278
:206BC0000230A16914F03DF9002008906068019009A80290102305AA696801F083F80220AA
:206BE000307168460770206A049029466846FFF753FEB0E770B50D460C46203529790120D4
:206C00008CB01646002909D0012905D13178042902D10920107000200CB070BD6068019026
:206C200006A802900822E16814F00BF9082208A8A16814F006F901202871062069460870AC
:206C4000206A049031466846FFF726FEE4E770B50D460C462035297901208CB01646002969
:206C600008D00129D8D131780429D5D10A2010700020D1E76068019006A802900822A1689F
:206C800014F0DFF800200890099001202871062069460870206A049031466846FFF7FCFD8F
:206CA000BAE730B50B4620331C7901208BB0002C09D0012C05D11178042902D10B2010707D
:206CC00000200BB030BD4868019005A802908C6868462578057564784475CC682578857553
:206CE0006478C47500200690079001E0E4B30100089001201871062368460370086A049027
:206D000011466846FFF7C8FDDBE770B50C462034034625790120002D0AD0012D14D0022DD6
:206D200005D111780A2902D10C201070002070BD01202071C868052202704A684260F84AE4
:206D40008260921CC2600BE015780B2DEFD102202071C86804240470526842608A68826062
:206D6000096A016201461846FFF745FE70BD30B5011D02463132947803258379ED432C43B5
:206D800023408371DB070DD04B79547923404B710B79127913400B718278C9788A4200D96F
:206DA000817030BD00224A710A71F5E7F7B50C4686B00020694626460870203631790127B2
:206DC0001E2015461F2977D24B007B449B885B009F441E0017023E025602690288029A02BE
:206DE000D102F5022E03590371037F03AE03C303CC03F7031A0464049A04AB04DF04FE044E
:206E000010052A0565059B05C605830587058B056069002802D0007813287DD0A068059055
:206E2000002849D0012168460170206A04900321684601710A214171E069029020790028F5
:206E4000EFD0059909780029E7D00C2964D20B0014F0A2FA0CFD1A4B90B5E8FCFBFAF9F8E1
:206E600007FD022828D16069002802D00078082852D1022168460170206A049005984178A7
:206E8000684601710021B9E20620216A05F0B5FB20790728E6D1606900F051FF02280CD032
:206EA000606900F04CFF042807D060690028B8D000780128D6D103E01BE2616901200870C7
:206EC00005980079C11F0A2901D30A2050E061690722887060690599303013F0B2FF0120D4
:206EE000307161690320087034E00728BAD16069002896D001780929B4D10599C9788907C8
:206F000007D1059949790029DFD1059989790029DBD105994A7900E04EE2014620314B7D1A
:206F20009A43D2D1059A8B7D92799A43CDD1059A1279D31F0A2BC8D20979914236D807222D
:206F4000C01C059913F07DFF0120307161690A200870032069460870206A04906069313078
:206F600001906069001D029060691C300390A1E22076F2E311288DD1606900F0E0FE042818
:206F800004D0606900F0DBFE0B2893D16069059910223730491C13F054FF606901780429CA
:206FA0007CD12421095C8278914201D90620DFE7052101700320307168460170E2E31128CF
:206FC00094D1606900F0BBFE062804D0606900F0B6FE0C288AD1E068002813D020690028D8
:206FE00010D060690178062910D00D2101706069059910225730491C13F023FF60695730C7
:2070000009218CE100206946087072E1072101706069059910224730491C13F012FF606954
:207020004730EDE70228F0D1606900F088FE0028EBD0606900F083FE0128E6D0606900F026
:207040007EFE05E0B1E08DE06CE02AE00AE0D6E00828DAD0052168460171059841786846B7
:20706000417146E11128D0D160690028CDD001780E29CAD1C16A4078022810D00020142241
:2070800050431430085805991022491C13F0D9FE0520216A00F041FE0F205EE0F1E101206B
:2070A000EDE70B28B1D160690028AED001780F29ABD1C16A4078022826D0002014225043BF
:2070C0000C300958059842780A70807848706069C16A4078022819D00020142250431030AA
:2070E000085805990822C91C13F0ABFE0520216A00F013FE60694178022909D00022083244
:20710000825C5208520073E00120D7E70120E4E70122F4E7012100E0002108314254BCE338
:20712000BEB3010011289CD16069002899D00178102996D1C16A4078022811D00020142280
:2071400050431830085805991022491C13F079FE0520216A00F0E1FD112061690870B4E3BD
:207160000120ECE7082884D1606900289DD00178112997D10599C06A4978017060690599BC
:20718000C06A0622401C891C13F05BFE0520216A00F0C3FD60694178022904D00022083203
:2071A000825CFD2323E00122F9E71128BBD160690028BBD001781229B5D1C16A4078022843
:2071C00019D00020142250431C30085805991022491C13F036FE0520216A00F09EFD6069C1
:2071E0004178022909D000220832825CFB231A40022991D18EE70120E4E70122F4E707200D
:20720000B6E6287801288ED16069696814221C30F9F7DAFF6069017F002901D02176ACE35C
:207220000178032901D0032037E00227C77081794907490F8171017A4907490F0172417A59
:207240004907490F41726069FFF791FD377196E228780F28E3D1072069460870216A04916D
:20726000916802916946087161690722C91C029813F0E7FD61690420087000203071BBE03F
:2072800028780328CBD1606901780529696807D00822473013F0D5FD0420307105206FE2BE
:2072A00008225730F6E728780328B8D1606901780529696811D008224F3013F0C2FD05203A
:2072C00030716069006A00280AD002202870002028716069006AA860F9E008225F30ECE7C5
:2072E00004204DE22878022899D12879002801D0207642E36069A96801626069002901D1B1
:20730000F949016206200BE228780F2887D1A868E0616069017805292BD047300721317189
:20732000E16802220A706269126A4A60886060693030C8606069C01C08616269087D926AE2
:20734000400812784000D207D20F104308756269926A521C8A61FD2210406269D26A127871
:20736000D207920F104308756069C06A401CC86153E25730D2E728780828BAD16069017839
:2073800005291AD00B210170072069460870206A0490E06902901120087102980321017018
:2073A00051681022401C13F04CFD00216846FFF773FA00203071E06187E20621E3E728780C
:2073C0000F2896D1072069460870206A0490A86802901120087102980421017061690A78DB
:2073E000072A0ED0002232710C220A7061691022401C473113F025FD00216846FFF74CFA11
:2074000063E21022401C573113F01BFD00216846FFF742FA0A203071E1680320087060697D
:20742000006A486060695730886060694730F3E128780828A1D1606969681022373013F076
:20744000D3FC002801D0042092E560690078072817D00A203071E168032008706069006A90
:20746000486060695730886060694730C860206A08620698FFF7BFFA07466069FFF777FC04
:207480006BE208207AE1287809289AD10B20307161696868897810224018511A13F02EFD56
:2074A000082069460870206A04906868019060698078087268E129780D29BBD1616989794B
:2074C000C90703D00C20307109203EE03071032770E228780E28ADD160691422291D1C30F3
:2074E000F9F772FE6069018DC06A4172090A817260698178C06AC1716169CA6A081D117A26
:20750000C909C90111724379626919438378D26A9B079B0F012B00D0002300799B01C000F2
:2075200003431943117260694078012876D0B4E160694178022901D0012100E000210831C7
:20754000405CC00707D00E20EAE069460870206A1146049019E11320B8E728780F2894D155
:20756000A868E0610F2030710520EEE7287803288BD16069C16A4078022801D0012000E021
:20758000002014225043103008580822696813F058FC10203071E168062022690870606904
:2075A000406A48606069C36A4078022801D0012000E000201427784310301858CA608860F7
:2075C0002BE128780C2886D16069C26A4078022801D0012000E00020142148430C30105847
:2075E00002230932696800F07DFB11203071E168052008706069006A48606069C06A093033
:2076000088603948001F07E128780B28A7D161694878CA6A022802D0012001E059E1002099
:2076200014235843143010588A78696813F009FC60694178C26A022901D0012100E0002124
:207640001423594314315258817850181022511A13F054FC072069460870206A0490E06962
:207660000290112008710298062101706169CA6A4978022901D0012100E0002114235943EB
:20768000143151581022401C13F0DBFB00216846FFF702F90020E06112206FE028780F281C
:2076A00091D1072168460170206A0490906802900B2268460271029801706169CA6A497861
:2076C000022901D0012100E00021142359430C3151580A784270497881706169CA6A49782D
:2076E000022903D0012102E0C4B30100002114235943103151580822C01C13F0A2FB00216B
:207700006846FFF7C9F826E760694178022901D0012100E000210831405C800703D51420EE
:2077200030710A2011E71620D0E628780F287AD1A868E061072069460870206A0490E06972
:207740000290112008710298082101706169CA6A4978022902D0012101E011E100211423B0
:207760005943183151581022401C13F06AFB00216846FFF791F80020E061152030710A20D6
:2077800069460870206A049029466846FFF784F82BE028780F2846D1072069460870206A44
:2077A0000490906802900820087102980921017061690622C969097841706169801CC969E7
:2077C000491C13F03EFB00216846FFF765F8AAE760694178022901D0012200E00022083278
:2077E000805C400703D51720C8E70746B5E0012953D070E028780F2815D1A868E0611820E3
:207800003071E168052008706069006A48606069C06A09308860F848C860206A08620698F8
:20782000FFF7E9F8E1E76FE028780B286CD16069C16A4078022801D0012000E0002014224C
:2078400050431C3008581022696813F0FAFA072069460870206A0490E069029011200871FE
:2078600002980A2101706169CA6A4978022901D0012100E00021142359431C3151581022F9
:20788000401C13F0DEFA00216846FFF705F80020E0616069407801281DD1192016E66069F8
:2078A0004278022A09D0002108314118097800290DD0CA0703D00E2106E00121F4E7890789
:2078C00001D5102100E012210170002772E0012A01D00D20FAE51C20F8E51D2030710B207A
:2078E00033E62978102948D1F0E560690178012943D0082941D00021317100F01AFA0C20F3
:2079000069460870206A049037E028780F2805D01020107003271B2030714BE007216846A8
:207920000170206A0490A8680290022168460171029805210170217E417000216846FEF78E
:20794000ABFF0B2168460170206A049029466846FEF7A2FF07461B203071012F0DD029E022
:20796000012168460170206A0490042168460171217E41710020207612E0207E00280FD0C5
:207980006169132008701A2030710A2069460870206A049029466846FEF77EFF074609E063
:2079A0006069002801D01421017068460078002800D021E5384609B0F0BDF7B50F462037FF
:2079C0003879012686B00C46002804D0012828D002281CD197E02079012804D0022811D0FB
:2079E000032814D10AE0A068407801280ED10620216A04F0DCFD00287FD10CE0A1681320A7
:207A0000087008E0A0684178022901D0052674E00078082871D1012038710A2069460870C5
:207A200033E0089800780F2867D1072168460170206A049008988568029522790220012A3B
:207A400004D0022A29D0032A57D10FE00646684606710B202870207B00214007400F68708B
:207A60006846FEF719FFA068067045E006466846067105202870207B687000216846FEF743
:207A80000BFF3E710B2168460170206A049068460899FEF701FF06462FE0684601710120E4
:207AA0002870207C6870607CC007C00FA870A07C4007400FE870E17C2971C0071FD0207DDC
:207AC0004007400F6871607D4007400FA87100216846FEF7E1FEA06807222946303013F005
:207AE000B0F9E068017AA06820300171A16828798870A16809200870002630465BE7002006
:207B0000A8716871E3E7A16814200870012168460170206A0490042168460171217B417102
:207B20000021FEF7B9FEE7E7F0B585B00F4605460124287B800040198038C66F3078411E9B
:207B40000A290AD22C498000323140188038C36F3A463146284698470446002C01D0012CC4
:207B600011D1287B401E0006000E287301D00324DFE70D2069460870306A0490002101967B
:207B80006846FEF789FE032CD3D0204605B0F0BD70B515460A46044629461046FFF7C4FF89
:207BA0000646002C0FD0207814280CD1207E002806D000202870204629460C30FFF7B4FFAF
:207BC000204600F0B6F8304670BD704710B5012903D0022901D0052010BD417000F0A9F855
:207BE000002010BD002809D0027E002A06D00A4601460C31CCE70000C2B301000120704742
:207C000030B5044687B00D46062004F0F6FC2946052004F0F2FC2078142805D000206946B1
:207C200008702046FFF7DEFF07B030BD7FB50E4600216A4611730178092903D00A2903D08E
:207C4000002407E0446900E08468002C02D0217E002912D0154601462846FEF7CCFE0328FE
:207C600009D1324629462046FFF792FF6946097B002900D0042004B070BD25460C35EAE7A8
:207C800000B50023012285B005280CD0062808D16846027004910221017143710021FEF790
:207CA000FBFD05B000BD6846027004910271F4E710B590B00C4605216B46197001902348A4
:207CC00002900892001D03900AA96846FFF7AEFF002805D1102220460B9913F0B2F80020BD
:207CE00010B010BD30B505E05B1EDBB2CC5CD55C6C40C454002BF7D130BD10B5002409E058
:207D00000B78521E5B00234303700B78401CDC09D2B2491C002AF3D110BD70B50C46054612
:207D200004F06BFC782300222146284604F0BEFB70BD4178012900D0082101707047002850
:207D400001D000787047082070470000BCB3010070B5F84D040008D0012C10D0022C07D07C
:207D6000032C05D0F4A1752007E0F3A16C2004E02878012803D0F0A1722013F0ECF92C70A7
:207D800070BD70B5EB4D044610280AD0112C16D028468178122C07D0132C0AD0E6A1A420FA
:207DA0000BE0E5A1992008E0112908D0E2A19E2003E0112903D0E0A1A12013F0CCF9AC7048
:207DC00070BD10B5DB4894B0007B002819D0172069460870D74900A806220D31023013F0FD
:207DE00030F809A9684603F0A8FE0446112805D0002C03D0D0A1C02013F0ADF9204614B0E7
:207E000010BD3220E4E710B50022022103F08CFF10BDFFB595B01D460E460746FFF7F3FF3E
:207E200004000AD02078222804D3A07F8006C00FA84204D1082019B0F0BDC348FBE7372195
:207E4000684601704780002D05D00121017146711799817102E000206946087109A96846C3
:207E600003F06BFEA07FDF21084069010843A0770020E0E770B50446084620380D46030021
:207E800013F08AFA0A060A11232C334249505761FF20A9A10D3052E02078202851D1FF2022
:207EA000A5A110304BE0A3480178032949D08078132846D02078242843D0252841D023287F
:207EC0003FD0FF209CA1133039E02078222838D0232836D8FF2098A11A3030E02078222804
:207EE0002FD0FF2094A11E3029E02078222828D0242826D0262824D0272822D0292820D0F8
:207F0000FF208DA121301AE02078252819D0FF2089A1283013E02078252812D0FF2086A15A
:207F20002B300CE0207825280BD0FF2082A12E3005E02078282804D0FF207FA1313013F056
:207F40000AF9257070BDFF207BA13430F7E730B57E4C0B887E4A022801D0934204D09D1F75
:207F6000A54225D2022802D04D88954203D04D88AD1FA5421CD24C88A34219D88B88FF2551
:207F8000F435AB4214D8022802D0C888904205D0C8886E4D0A382D1FA84209D2C88890426C
:207FA00008D0944206D05B1C63438000834201DB072030BD002030BDF0B56649884245D3A8
:207FC000654A0125AD041368A84201D398423DD30279002A06D0082A02D8067B082E05D9DC
:207FE0000720F0BD047B002CFAD0F6E7002A06D004688C422AD3AC4201D39C4226D3002E5D
:2080000006D084688C4221D3AC4201D39C421DD300240CE00568A700ED598D4216D3012702
:20802000BF04BD4201D39D4210D3641CE4B2A242F0D800220125AD040CE084689700E45981
:208040008C4203D3AC4203D39C4201D21020F0BD521CD2B29642F0D80020F0BD10B502897B
:208060003E4B111F994213D24189042910D3DB1C99420DD891420BD80178890706D54068B4
:20808000002803D0FFF798FF002800D1002010BD072010BDFFB50022099B002802D099422F
:2080A00005DC6EE0002902D1002004B0F0BD0920FBE7845C002C12D087187D78112D59D020
:2080C00010DC2B0013F068F90A561726262C2C2E2E4C4C56835C002B46D1521CD2B28A42E1
:2080E000F8DBE1E71C2D45DA123D2B0013F054F9044242121A42022CD9D1BB78039C072BE1
:20810000237001D25B0701D40A20CEE7029B01241B782CE0E343DB0708E0012C08D029E084
:208120000620C2E70F2523072D075B19002BF4D03046BAE7640C00207372635C6761705F99
:20814000636F72652E630000023000007B0C0000FFFF000000C0010028000020FD3F0000E9
:20816000029B1B789C0701D50B209EE702242343029C2370835C521C9A18D2B28A4202DDBB
:2081800095E7192676028A4293DB8DE710B504780B46002C08D00121F94A012C07D0022CD1
:2081A0000BD0032C13D10EE00021197011E019708179890903290AD10BE01970817989092C
:2081C000012904D105E019708179890901D0104610BD411C0622581C12F033FE002010BD99
:2081E00008B51346002806D0E6A00068009048796A468009105C18700622581C12F021FE42
:2082000008BD30B50C46097895B0222902D2082015B030BD282369460B704880132A03D056
:208220003B2A01D00720F3E708460A7109A903F084FC050003D121212046FFF71BFE28461B
:20824000E6E700B595B0232369460B704880108888805088C880D08848819088088100207D
:208260008881C88109A9684603F067FC15B000BD70B50C00064610D0FFF7C5FD050003D186
:20828000C149C24812F067FFA6802889E0802889208168896081A889A08170BD70B50E460F
:2082A000050003D00021092004F0A7F90120B84C022E207324D0032E04D0D320B2498000B9
:2082C00012F049FFB24806210D3003F02DFFA07C8006800EA074FFF774FDA08B00280ED0FB
:2082E000002D0CD0830001220021092004F0DEF8092804D0A548A449283012F02CFF70BD2A
:20830000A3480321103003F00FFFA07C40218006800E0843A0749E480C3002F04EFBDAE7FF
:208320007FB501A9022003F06EFD002851D097489549673012F00FFF4BE0029C2078212888
:2083400047D0A07F01072BD520462230009068462346628E80882146343301F084FC050044
:2083600005D011282ED089488749843028E0A07FF7210840A077E17F480889074000C90FA6
:2083800008432021095D4007400FC9000843E0772078282824D129212046FFF76BFD1FE000
:2083A000400716D568462246808821460E32FFF748FF050008D0112804D074487249933065
:2083C00012F0C9FE00250BE0A07FFB210840A07706E001A803F025FD0500AED0052D02D0FF
:2083E000284604B070BD0020FBE7F8B5040004D166486549A13012F0AEFE722020706068E1
:2084000008260178091F0B0012F0C6FF11FD0A4668FC460EFCFC4746464646FD92FD46007C
:208420007B205949C00035E087883846FFF7EBFC050004D11F205449400112F08CFE607865
:20844000042130436070524CA07F0843A07721212846FFF70FFDA87F8007800F012801D1AB
:20846000801EA080384603F0B1F83846FCF7FBFF3846FBF79EFB3946022004F0BEF8A87F3E
:20848000EF210840A877FFF74BFF002804D03F483D49C93012F05FFEF8BD85882846FFF79E
:2084A000B2FC002804D139483749D33012F053FE60688078012804D034483349D53012F0FE
:2084C0004AFE60688179284603F09CF90028E3D06178314361706168C880F8BD8788384650
:2084E000FFF791FC050004D128482749E63012F032FE60783946304360706068C0882881A4
:2085000060680089688160684089A881022004F074F80020A875A87F8007800F0228DCD194
:20852000FFF7FEFE0028D8D0212017494001B1E780783C2803D00025022814D000E0012597
:208540000027002808D03C2806D0022804D00F480D49FF3012F0FFFD002F06D0022630463F
:2085600001F06CF9F8BD0127EBE76078304360700748817F31438177002D0BD00126EEE71C
:20858000023200000302FF01388100002E030000640C002060688788384601F07BF9054623
:2085A00060688079012832D00226A87F0622800880003043A8776068C08A28816068008BB0
:2085C00068816068408BA8816068C079E875616828461830083112F034FC60680622807BC3
:2085E00068706168A81C0F3112F02BFCA87F8107890F384602F0D4FFA87F8007800F0128BD
:20860000ADD101E005E008E0FE488780A7E70126CBE7204601F01EFEF8BD60783043607037
:20862000F8BDF7B505460078002700090C463E4601287DD00022F44902287AD0072804D0C4
:208640000A2877D0F149F24839E1686803780D2B35D006DC042B6ED0072B3AD00A2B69D191
:2086600006E0122B3CD0132B44D0142BF7D1BEE011270726002C7CD08088A0806968FB23E0
:208680008979A171DF4905468A7F1A408A77042103F071FB0521284603F06DFB00212846ED
:2086A00003F069FB0121284603F065FB0321284603F061FB0221284603F05DFB01E10127B9
:2086C0000926002CD7D08088A080686880792072F7E012270E2680882146FFF7C9FDF0E0D6
:2086E0001A270726002CC6D04088A08068680079A071E6E081783C293ED010271E26002C2F
:20870000B9D08088A0806868C08A20836868C08AE0826868008B60836868408BA0836968A2
:20872000607D497F40084000C907C90F084303E06CE097E0BAE029E060756968C007497F9B
:20874000C00F49084900084360756968A21DC8790831FFF745FD69682246887B0D320F3193
:20876000FFF73EFD68688079002803D00120207507E076E00220FAE719270726002C70D035
:20878000A271A048F722817F11407DE01B272E26002C66D0A1806968A21D0879491DFFF791
:2087A0001FFD68682030C07A60736868C0780428A07B19D040084000A073F921084069686A
:2087C0001F22C9788907490F0843A07369684007C97A400FC9000843A073696820460F308A
:2087E0000C3112F02EFB6CE001210843E4E71E270E26002C6DD0A1806868E21D407AA071F0
:2088000069688878C91CFFF7EBFC5AE0287A012805D0022815D07E487C4932384FE01D2774
:208820000E26002C55D06888A080A889E080E8892081288A6081688AA0817248DF22817F9F
:20884000A2E712270E266888FFF712FD002C40D068784007400F032833D16A48FD22817F7B
:2088600092E736E0287A030012F096FD060410102020202619270726002C2AD0A180614822
:20888000A271817F4908490081771AE019270726002C1ED0A180287A012805D00320A071BD
:2088A0005848EF22817F6FE70220F8E721462846029A01F068FEFEBD55485449801F12F052
:2088C0004AFC0298002C068001D0278066800020FEBD02980680FAE710B54A4894B0807839
:2088E000132802D0082014B010BD22206946087009A9684603F021F904460021072003F057
:208900007CFE2046EFE700B53E4895B08078122801D00820AAE41E216846017000218170F8
:20892000C17009A903F009F90028F3D10021072003F063FE1120FFF724FA002096E400B543
:20894000304895B00078022801D0032818D11B2108A801730021817369460BA803F0EDF824
:20896000002804D1684640781B2801D003207DE40021084603F041FE68468078002801D0BC
:20898000082073E40120FFF7E3F900206EE4F8B51C4C030012F000FD0A0679177979797958
:2089A00044356779FFF7CBFF00282AD1F8F7DAFF002826D02221017000210172F8F7B3FFAC
:2089C000A07F01214BE08EB23046FFF71CFA050004D10F480D492E3012F0BDFB28782128E1
:2089E0000FD0F8F7BFFF002814D0122101700227077246800020A875F8F795FFA07F384379
:208A0000A077F8BD640C0020FFFF0000388100005F050000132229463046FFF7F2FBF0E70B
:208A2000A578122D06D0132D07D0F849F84812F092FBE6E7FFF767FF01E0FFF74DFF002869
:208A4000DFD1F8F78FFF0028DBD022210170122D07D002210172F8F766FFA07F10210843C7
:208A6000CEE70121F6E7A07C810901290BD0800904D0E748E549223012F06DFB03210020DD
:208A8000FFF70CFCBDE70221F9E7E148DF492930CDE7F7B514460D0004D1DD48DB49313041
:208AA00012F059FB28780827012807D002281FD0D748D649623012F04EFBFEBD0098FFF714
:208AC000A2F9060004D1D248D049383012F043FB0220B0751030207060783843607007CD37
:208AE000083407C4CB482022817F11438177FEBD0098FFF788F9060004D1C548C34946309A
:208B000012F029FBA988C448814208D1EA88824205D1132231460098FFF773FBFEBD814224
:208B200002D1E888002809D01220207060783843607007CD083407C4002006E0782300226E
:208B40000220009903F0B2FC0120B075FEBDB14840897047FFB591B01498FAF71BF9002871
:208B60005DD10124684603218471C9028180002201A92046FBF7ECFA002850D168461521D8
:208B800084714902818000261C2102A8009612F0B7F9012001466846103101700020014610
:208BA000684641708178F9273940891C21438170017A02252943017212998186C6861F210B
:208BC00001870C9011980F9001A80B9009AA0BA902A8FBF788F8002821D168468D4E808CB3
:208BE000F080684684718D498180807809AA3840801C41084900684681708586058713A849
:208C00000F900BA902A8FBF76EF8002807D16846808C308131460A311498FAF7CEF815B0BA
:208C2000F0BD30B50C467E4995B08C423CD37D49012292040968944201D38C4234D32038A0
:208C400000220125030012F0A7FB06042A44484E575F0021082003F0AAFC002802D0112054
:208C600015B030BD24206946087000A80522A11C023012F0E6F809A9684602F05EFF050085
:208C80002FD1082300221146184603F00FFC082827D05F485D49D63012F05DFA21E0606838
:208CA000002803D0884201D21020D9E73D2168460170218841806188818009A902F03DFF7B
:208CC00005000ED1606800280BD06946098D018007E0206801F0B2FE02E0204600F024FEB5
:208CE00005462846BCE73E2007E0857000E0827009A902F022FFF3E734206946087020785A
:208D0000C0076846F3D0F0E70720A9E730B50C46444995B009688C4201D21020A0E7203863
:208D2000030012F039FB05042121232132002088FFF769F8002804D00078222803D208207F
:208D40008EE739488CE72521684601702188418009A902F0F2FE050015D10AA9052202314F
:208D6000A01C12F06EF80EE006250CE02068002805D0884201D2102505E001F055FE2548DD
:208D80000025808BA08028466AE7072068E721481330704710B520211E4812F0AFF80120B5
:208DA000FEF7D6FF1120FEF7ECFF00211948C943818000218176E1218900818301460C301F
:208DC0000D310446F8F74EFE124807222146133012F037F8FEF7F5FF002803D00B491348DF
:208DE00012F0B9F901F0E5F910BD10B504463C2112F084F8A07F80088000A077202020702B
:208E00000020A0752034607010BD000038810000B5050000640C0020FFFF0000012A000000
:208E200000C0010028000020023000001C0700007047FEB50546FF480C46814207D30120C8
:208E40008004844205D3FC480068844201D21020FEBD002D02D0012D32D126E0F749082220
:208E60000F46684611F0EDFF39462046FFF78EF90028EDD1FEF7A5FF060006D0072269466D
:208E8000384611F0DEFF3046FEBD2078002801D0012805D1E94807223946C01D11F0D1FF2E
:208EA0000021092003F0A9FB0FE00978002907D0012905D0022905D0032903D0E048FEBD80
:208EC0000720FEBD0120FFF7E9F9DC480C3885760020FEBD10B5D8490968884201D2102055
:208EE00092E7D64902460C390B7B0D311846FFF777F9002088E7FFB599B00546002008A91D
:208F000008746946087108A908730875CA4814460121C84A890400681E46002D05D0954232
:208F20000BD38D4201D3854207D3002C08D0944203D38C4204D3844202D210201DB0F0BD76
:208F40002846204318D01F270BAB0CAA009728461A99FFF79FF80028F0D10DAB01AA31469E
:208F600020460097FFF796F80028E7D168460079C00703D00A20E1E70720DFE702AF002D12
:208F80000FD01A20694608721A9888722946F81C1A9A11F056FF0EA902A802F0CEFD002810
:208FA000CCD1002C0ED0202168460172867232462146F81C11F045FF0EA902A802F0BDFD6B
:208FC0000028BBD19D4908A8007B0C3948700020B4E770B506460A200C46087015461146FD
:208FE000204602F0AAFD002807D1392121702046294602F0A2FD002804D0082801D190484B
:20900000401C70BD2A462146304600F0B9FC0446082803D18B498C4812F09DF8204670BDB5
:20902000F0B5044689A003C897B0824D002715911490AC4211D380480121890403688C4244
:2090400001D39C4209D32078012809D16268AA4203D38A4204D39A4202D2102017B0F0BD64
:2090600076490C390A78012A0CD18A88794B9A4203D0002806D0012804D08A7F13079B0F15
:2090800006D101E00820E9E7D30701D1910701D51120E3E7218A704B0A46203A9A4207D345
:2090A000012877D1002975D1628A002A72D111E0022801D0032801D1A0296BD3012809D085
:2090C0005E4A0C3A5278D20704D0628A002A61D0B42A5FD8002806D0012808D0022804D0D2
:2090E000032857D117E0002518E0022516E0002902D1608A00280CD0042560680078002871
:209100000CD0012809D0022807D0032805D04C48A4E70125F1E7032500E00127207A002861
:2091200006D0012806D0022806D0032867D105E0002604E0012602E0022600E00326002DA1
:2091400001D0022D16D1002E14D0E068002803D0FEF732FF002881D138480C384078800730
:2091600002D03748401E79E7022D03D1022E46D0032E44D0182168460170218A4180218AE3
:20918000818085712D480C38007B002803D001286FD104E033E000216846C17102E0012045
:2091A0006946C8716846077221780930012920D0062111F0A3FE69460E74207D8207C107CC
:2091C000D20F4007C90F5200C00F11438000014314A8405C6946C873002810D009A96846AC
:2091E00002F0ABFC002893D1002D0AD0022D08D012E061680622491C11F023FEDBE70720E9
:209200002CE7002E08D0E068002805D009AA6946FFF7DFFE0028A6D11B2069460870012099
:20922000887009A9684602F088FC00289BD108A8407913E000C0010028000020700C0020CB
:209240000232000038810000270800000706050403020100FFFF0000E13F00001B2819D18B
:209260002B0012F099F80504040707040A00032001E00FE00220FEF76BFD012D0CD0608AA1
:20928000002809D0002283001146104603F00EF9002801D00320E1E60020DFE6F3B50326E8
:2092A00087B00D4600290AD0FE4885426FD301208004854203D3FC480068854267D3079844
:2092C000FEF7A1FD040005D02078222804D2082009B0F0BDF548FBE7A07F8707BF0F002D15
:2092E00005D029463846FEF732FE0600F0D139460027EF48012907D0022931D0ED49EE484A
:2093000011F029FF3046E3E7A27D2946012A02D0827F920701D51120DAE700291BD10821B9
:209320006A46049711820592418904AAE348FBF7FFFA0028CCD16846008A082801D0032009
:20934000C6E76846018801814188418181888181C188C18102A9079802F0E7F90646D1E766
:20936000A17D022916D1807F800613D4002D04D0A07F40070CD4002100E00121079802F056
:2093800014FA0600BED1A775002DBBD004E01AE01126B7E7002D16D02A4621460798FEF725
:2093A00050FF06461128ADD1A07F4007AAD42046082229460E3011F044FDA07F0421084369
:2093C000A07700269EE7102082E770B50C460546FEF719FD010004D022462846FEF711FFB5
:2093E00070BDB24870BD00B50146143195B0192901D2810707D001461E3104D00A3102D0A8
:20940000072015B000BD312269460A70887009A9684602F092FBF4E701B582B002206946BC
:209420000880A34802AB00896A460021FBF7EAF869460988022900D003200EBD1CB50021C3
:20944000009102216A461180974901900968884201D210201CBD964801899848FBF768FAF3
:20946000694609880229F5D003201CBDF0B50E468C4985B0174605468E4207D38A48012276
:2094800092040068964204D3864202D2102005B0F0BD1F2F01D90C20F9E7854C8D4226D324
:2094A000954201D3854222D3E08803A9FBF75BF80028ECD1287869464873E08803A9FBF7F7
:2094C00033F80028E3D16946009008780221084369460870497B090703D008210843694667
:2094E0000870E0886946FAF7B8FF0028CFD169468F80E088334601AA0021FBF783F86946E6
:209500008988B942C3D00320C1E71CB50C46002100910191228869460A80634901900968E9
:20952000002801D0884201D38C4201D210201CBD002801D0002A09D05D486A46C1885F48A9
:20954000FBF7F6F96946098821801CBD0C201CBD10B50123FEF75DFC56E4002310B51A46B2
:209560001946FEF756FC4FE470B504464D4894B0844207D301208004844206D34A480068EC
:20958000844202D2102014B070BD2046FEF766FD0028F8D146488178112901D00820F2E7CE
:2095A000817FC90601D51120EDE71D2269460A7021780025CA07D20F69468A7022898A80CB
:2095C0006289CA80217801268907CA0F69464A72007B002803D0012804D00320D3E7084624
:2095E0000D7201E008460E7209A902F0A6FA0028C9D12078800708D56068002805D009AAC3
:209600006946FFF7E6FC0028BDD11E21684601708670C57009A902F090FA0028B3D1A08981
:2096200000F073F90400AED11220FEF7AAFB2046A9E7F0B516461C4A0C4605001948204901
:20964000126899B005D085420FD38D4201D395420BD3844209D38C4201D3944205D38642B7
:2096600003D38E4204D3964202D2102019B0F0BD0F4FB87FC106890F01D1400701D5112007
:20968000F4E72046FEF7EAFC0028EFD120788107C90F294303D0800714D5002D12D00720E9
:2096A000E4E7000000C001002800002002300000640C002038810000F3090000FFFF000061
:2096C0000000040031460220FEF741FC0028CDD1C9488078112803D0122801D00820C5E701
:2096E0000220002714A9189002F08DFB00280DD0C2A1C64811F02FFD08E01598807F810783
:209700001898890F814201D17F1CFFB214A802F088FB0028F1D0032F01D30420A6E7B64851
:209720008078122803D1FFF7EEF800289ED12078800708D56068002805D009AA6946FFF797
:2097400048FC002892D12121684601702189418061898180207800278007C10F68468171CD
:2097600020788007002815DB2878002807D0012808D0022806D0032804D0A54876E768461B
:20978000C77102E001206946C8710622691C02A811F057FB9848007B002803D0012804D0A9
:2097A000032063E76846877302E001206946887331886846018271884182B1888182F1888C
:2097C000C1820783478309A902F0B7F9002886D1A08900F09AF80400A0D11320FEF7D1FA0C
:2097E000204643E730B505468A4895B000680C46814202D2102015B030BD2846FEF703FBFE
:20980000002807D00178222902D3807F800603D40820F0E78048EEE71321684601704580A0
:2098200009A902F08AF90028E5D108AA0A2151567F2901D02170DEE70520DCE710B56E496C
:20984000012807D0022815D0FF206CA14D3011F082FC81E60878032804D0FF2067A1433051
:2098600011F079FC0021084602F0C7FE0120FEF76FFA71E68878132804D0FF205FA14830D0
:2098800011F069FC0021072002F0B7FE1120FEF778FA61E6F8B504460122022102F044FA27
:2098A000074601220321204602F03EFA064601220521204602F038FA05460122042120466C
:2098C00002F032FA0446002F04D1AF204BA1800011F041FC002E04D14C4848A11A3811F0D0
:2098E0003AFC002D04D1494844A1193811F033FC002C04D1454841A1183811F02CFC22210D
:209900003846FEF7B7FA3846F8BD10B5002809D0830000221146072002F0C8FD072801D050
:20992000032019E6002017E610B50446006800280CD03A49884207D301218904884205D3F5
:2099400034490968884201D2102005E601F060F8A088294CA083A07E01280DD100210920E9
:2099600002F025FE002800D00120A17C8909012904D00321FEF792FC0020EDE50221F9E770
:20998000F7B500260C4605460B271AE02968B00009580978002903D0012901D00720FEBD30
:2099A000A170296806220958E01C491C11F049FA27702046029902F0C0F80028EFD1761C1B
:2099C000F6B22879B042E1D800263A270FE0A868B10041581022A01C11F033FA27702046AA
:2099E000029902F0AAF80028D9D1761CF6B2287BB042ECD80020FEBD640C00207372635CC4
:209A00006761705F636F72652E630000D702000002320000280000200230000000C001002D
:209A200030B5FE4B9A4207D301239B049A4205D3FB4B1B689A4201D2102030BD1578EB06B8
:209A40005B0F042B07D85478072C04D39378102B01D8A34201D2072030BDD3785B0702D44A
:209A600013795B0701D5062030BDC37FAC075B085B00E40F2343C3770878EF231840137854
:209A80009B06DB0F1B0118430870F12318401378DB065B0F5B001843087050780873002079
:209AA00030BD30B500240C70C378DB07DB0F0B70C578AD07ED0F6D002B430B70C5786D07BE
:209AC000ED0FAD002B430B7014700179C907C90F117003799B07DB0F5B0019431170007914
:209AE0004007C00F80000143117030BD70B514460D460646F7F736FF002809D0A2210170A8
:209B0000142221460830F7F75FFBF7F70CFF70BD132229463046FEF774FB70BD70B51446D8
:209B20000E460546F7F71EFF002809D02221017045802178017261784172F7F7F4FE70BD5C
:209B4000132231462846FEF75CFB70BD10B5B54C207C00280DD12046B34A21461038FEF703
:209B6000A7F8002803D0B1A1F12011F0F4FA0120207410BDFFB581B00A9D06461C461746E0
:209B80001421284611F0BCF90B9800210160F8070ED0A34920680968884239D312302860E5
:209BA0002068143068602068A8600B9821680160B80726D56068002803D09949096888425A
:209BC00026D3029900290AD0FC3600280ED031461030FEF7DBFA00281BD1606810E0002841
:209BE00016D0E86080366068B0670AE0FFF7CFF801460722304611F024F9FFF7A7FF89488A
:209C0000E860780708D58649A0680968884202D2102005B0F0BD28610020FAE770B505462E
:209C200011200C460870002161702121495D002908D003290ED0042910D0FF207BA152307A
:209C400011F089FA20780009012802D9E87FC008607070BD0007000F203002E00007000F51
:209C600030302070EEE770B594B015460C462C226946189E0A704880002B17D00822194679
:209C800001A811F0DEF868468581102231460E3011F0D7F809A9684601F04FFF002803D13E
:209CA000A17F10221143A17714B070BD002001900290E8E7F0B50646008A97B080B20D469C
:209CC0000190FEF7A0F804465648317848385B4F09900B0011F060FB0EFEFD43084A728318
:209CE000B8D9FCFBFAF9F8FEA07F8007800F012807D000210022019802F016F8050007D105
:209D000001E00121F6E7FF2048A1943011F023FA387CC00904D049484038406DA86112E077
:209D20002B20694608720BA902A801F006FF002804D0FF203DA19F3011F00DFA40490C985E
:209D400011F0E8F8A9617068A862B068E8622078252804D0FF2035A1A53011F0FCF93246E3
:209D600021460198FFF7C2FE17B0F0BDA07F8007800F012807D000210022019801F0D4FFE4
:209D8000060007D101E00121F6E7FF2027A1AF3011F0E1F92078252804D030780121084396
:209DA0003070E1E702202870B068A860B068002802D000202871D7E70120FBE72B206946DB
:209DC0000870184968464C3901F0B7FE002804D0FF2016A1CE3011F0BEF903201BE02A20E1
:209DE0006946087000A810220230716811F029F804A810220230B16811F023F809496846F0
:209E00004C3901F09AFE002804D0FF2007A1DF3011F0A1F904202870099813E000C00100B6
:209E200028000020300D0020FFFF00007372635C6761705F7365632E63000000500E0020FA
:209E400040420F0068608FE7B068002804D1FF20F649EB3011F07FF9E07F400704D5FF208E
:209E6000F249EC3011F077F9B06806220A38009033790421019801F058FA002891D0FF20B3
:209E8000EA49F13011F067F96EE7002C04D1FF20E649F93011F05FF92046223010220546B2
:209EA000716810F0CEFF28212046FDF7E3FFA07F8007800F022814D100231A4621460095B4
:209EC0000198FFF7D0FE06E055E1B6E0ACE089E02CE065E069E111280BD029212046FDF72B
:209EE000C9FFE07F317A4007400FC9000843E0773AE7A07F000703D5CC49CD4811F02BF921
:209F0000A07F08210843A077002060862046343010F0F4FFE07FFD220146C9071040890F57
:209F20000843E077307A203420701DE7A07F8007800F012807D000210022019801F0F4FEF9
:209F4000040007D101E00121F6E7B948B7491D3011F001F92B2069460872B64902A801F0EE
:209F6000ECFD002804D0B248B049223011F0F3F8B0488188204621300176090A41760E21A3
:209F800029702146FC316960017E2974407E6874A8482C30A860103030346C61E860E3E63F
:209FA000002C04D1A248A149363011F0D4F8207821289DD93079012802D0022808D103E0B8
:209FC000E07F04210843E077387C012108433874324621460198FFF789FD23212046FDF7FC
:209FE00049FFC1E601220421019801F07DFC00289BD0A07F8007800F012807D0002100221C
:20A00000019801F091FE040007D101E00121F6E787488649543011F09EF80F2028701720B4
:20A0200028716E34AC609FE60421019801F0ABFC0028B4D11020287096E6A07F8007800FD8
:20A04000012807D000210022019801F06DFE050007D101E00121F6E7754874496D3011F0F3
:20A060007AF82E462036307E41064DD5A17F8F07BF0FC00713D02A468032516F00290ED076
:20A08000087CF37DC007C00F5B0018430874516FE27F40084000D207D20F10430874307E24
:20A0A000000713D528468030026F002A0ED0117CF37DC907C90F5B0019431174E27F490887
:20A0C0004900D207006FD20F11430174307E80070BD5F8204259002A07D0012F05D0294608
:20A0E000307C31311032FEF77BF8307EC0060BD5F8204259002A07D0012F05D12946307C7F
:20A1000031311032FEF76CF8052368460370357E4570484822226038019902704278D20885
:20A12000D200D21C4270418003724572F7F782FD2078252809D021280BD0AD203B498000A0
:20A1400011F009F82078222803D922212046FDF791FEA07F8007800F01280AD00021019821
:20A1600001F009FE002800D1FEE5AF202F49800088E60121F3E774682E4D20786035092825
:20A1800002D00A28F0D10BE0E168002902D02846F8F7D7FE2169002902D02846F8F7D1FEE8
:20A1A00021462846F8F7CDFEDEE521481F49DC3068E6204810B5072228216030F8F7A8FE5E
:20A1C0001D480024017C4906490E017440384465FDF7FBFC17493C3108461038F7F779FC8C
:20A1E00014484C30047410BD70B50D46FDF70BFE040004D103200D49000210F0ACFFFF21AE
:20A200000531284610F07CFEA07F8007800F012816D0022128468830FDF7D8FC002803D0D0
:20A220000249064810F097FF70BD00002C9E000005020000E40C0020500E0020050300005B
:20A240000121E7E70A46014610B510468830FDF7D7FC10BDF0B505464068082601789BB086
:20A2600008290DD00B2903D00C293FD101218171686887883846FDF7C6FD040041D13BE02B
:20A2800047883846FDF7BFFD040003D1FD49FE4810F061FF2078212828D0282828D168680B
:20A2A00002210C3000F0BEFF002821D068680821001D00F0B7FF00281AD02D21684601703E
:20A2C000478021461022223101A810F0BAFD0FA9684601F032FC002804D0CB20E94980004D
:20A2E00010F039FF29212046FDF7C4FD1BB0F0BD687830436870F9E7E348E2492D3010F08B
:20A300002AFFA07F8107890F022902D1EF210840A0772078212810D068688179002902D0E2
:20A320008078002818D0A07F8007800F022864D00720D449C00110F00EFFA07F8007800F3B
:20A340000228D3D1FDF7ECFF0028CFD0CE48CD49733010F000FFC9E7687830436870E07F81
:20A36000C00701D0042100E00321212001552078292818D02428E0D13946062002F03DF9EA
:20A3800022212046FDF776FDA07F8007800F012831D00021384601F0EEFC0028CDD0BA480D
:20A3A000B8495830C7E7A07F8007800F012807D000210022384601F0B7FC050007D101E00E
:20A3C0000121F6E71B20AF49400110F0C4FE25212046FDF74FFD0D2008A90871284609A9E5
:20A3E0008830FDF7FFFB0228A7D00028A5D0A648A4494D309FE70121CCE76878304368709B
:20A400009BE7F7B58AB00A98FDF7FDFC050056D02878222853D3232851D0E87F40074ED4CE
:20A42000A87F8007800F01280ED0002201280DD000210A9801F078FC064694480290F8F7DF
:20A4400077FD040009D103E00122EFE70121F0E775208C49C00010F07EFE002E0FD0883664
:20A4600066610298F8F764FD07460298F8F760FD06462878222807D0242805D008E00020C2
:20A4800007460646606103E025212846FDF7F2FC092020700A9820620C9820710B98E760ED
:20A4A0002661A06004A92046FDF7C0FB022806D0002804D074487349AF3010F04CFE0DB0F9
:20A4C000F0BD30B587B00446FDF79DFC0546807F8007800F01280BD000210022204601F0DE
:20A4E00023FC0446287822281ED9002C07D101E00121F2E764486349BB3010F02CFE0F2195
:20A50000684601701721017120466E30029069461A30FDF767FB022806D0002804D05A48EF
:20A520005849C03010F017FE07B030BD30B587B00446FDF768FC0546807F8007800F01288A
:20A540000BD000210022204601F0EEFB044628782228E9D9002C07D101E00121F2E74A4835
:20A560004849CD3010F0F7FD10206946087020468830FDF737FB0028D6D043484149D030DB
:20A5800010F0E9FDD0E7F7B5054600780027000982B00C463E4602287CD0072802D00A28CE
:20A5A00049D149E068680178082906D00B292FD00C292DD03349364865E114271A26002CBC
:20A5C00069D04088A080FDF71EFC0090002804D12F482C49243810F0BEFD00980099C07D4E
:20A5E000A21D1831FDF7FCFD686808228089E081696820461030091D10F023FC207E012186
:20A600000843F9210840207600984021807F50E018270826002CD3D08088A080FDF7F3FB89
:20A62000050004D11A481749401F10F094FDA11D2846FFF7F3FA28E1002C01D0288BA080A6
:20A64000287A01287ED0022805D0032838D010480C49853017E11C270726002CB0D0A08811
:20A66000FDF7D1FB0090002804D109480549133010F071FD287B8007800F0128A0791CD056
:20A68000400809E02C9E00001A030000440D002027040000E9E0E3E04000A071FD210840C3
:20A6A000297B4907C90F49000843A07100988021807F084300998877E7E001210843ECE707
:20A6C00013270B26002CA6D0A088FDF79CFB0090807F8007800F012807D00021A0880022AA
:20A6E00001F022FB050006D101E00121F6E7FB49FB4810F030FD0098807F8007800F012806
:20A7000050D0E86A81788907890F0129A1794BD049084900A1718278FD255207D20F2940DC
:20A7200052001143A171E322114002785207D20E1143A171DF2211404278D207920E114319
:20A74000A17100E033E00021E171C178217242790179607AD30740084000DB0F1843930765
:20A76000DB0F28405B0018435207FB23D20F1840920010436072A07ACA0740084000D20F16
:20A7800010438A07D20F2840520049071043C90F184089000843A07200980078232874D9D9
:20A7A0002621C4E0A86AADE701221143B2E7297BCC48022911D017270C26002C50D001294E
:20A7C00012D003291FD0042920D005291ED09320C249C00010F0BFFC23E019270726002C6E
:20A7E00053D00121A17105E00121A171E17989088900E171017CCA094906D201890E4900D1
:20A800000A4302740DE00220A07106E0687B0007000F8030A07105291DD0E0798008800039
:20A82000E071A088FDF7EFFA0546007821282CD0232804D0AA48A949573010F08CFCA87F81
:20A840008007800F01280ED00021A08801F093FA222128466CE0E07980088000401CDFE794
:20A860000498068017E00121EFE7002C01D06888A080287A032832D004280FD005285AD089
:20A8800097489649B03010F066FC0498002C068001D027806680002005B0F0BD15270C261C
:20A8A000002CDDD0A088FDF7AEFA807F8007800F012807D00021A088002201F035FA050056
:20A8C00007D101E00121F6E785488449763010F042FC0622A11DA86907F036FAD5E716272B
:20A8E0000726002CBCD0A088FDF78DFA0090807F8007800F012807D00021A088002201F0CF
:20A9000013FA050007D101E00121F6E774487349843010F020FC2878C00601D5022000E0E7
:20A920000120A071009800782328AED927210098FDF7A0FAA9E717270C26002C90D0A088E1
:20A94000FDF761FA00906D7A002804D164486349973010F000FC0621A01D10F0CFFA00204C
:20A96000A071207A032108432072FB2108400099C97FC907490F08432072680685D5E079C0
:20A9800004210843E071A07AE90740084000C90F0843E17A2A0749084900D20F1143FD22C7
:20A9A000AB07DB0F10405B001843A072E806C00F114040000143E17267E710B504468079A8
:20A9C00090B08009012804D045484449C93010F0C2FBFFF7BBF801206946087042480890CE
:20A9E00042480190201D0290601C0B900AA96846FDF71CF9002804D039483849D43010F0EA
:20AA0000AAFB0322601C0B9910F01BFA10B010BD10B5364C002805D001461022204610F087
:20AA200010FA0120207410BD10B50446FFF78EF810222E49204610F004FA10BD70B50025DB
:20AA4000284C00281CD02A49884207D301218904884205D327490968884201D210250DE066
:20AA6000062107F05BF9411C07D01E4940394865207C80210843207400E00725284670BDE0
:20AA8000207C4006400EF6E7F3B5002089B00D46029000290AD0164885421CD30120800407
:20AAA000854203D313480068854214D30998FDF7AAF9060003D03078222826D102E00E4856
:20AAC0000BB0F0BD002D19D1B07FC10903D08007800F022812D01020F2E700002C9E000036
:20AAE0004D040000500E0020FFFF0000300D002000C001002800002002300000B07FC106FB
:20AB000001D4010703D5002D01D00820D8E7FE49097CC90717D1F17F490701D50D20CFE79E
:20AB20008007800F01280CD000210122099801F0FBF8070007D0B07F8007800F022804D010
:20AB40000DE00121F1E71120BAE7002D07D02A4639463046FEF764FF02900028B0D1EB480D
:20AB6000F8F7E6F9040003D1E949EA4810F0F3FA0A2020700998206238468830A060B07F9C
:20AB8000FB218007800F012829D0002D3DD002202071381DE06038780007400F2074387895
:20ABA000C006C00F6074A07C2A788008D2078000D20F1043A0740840F17F01AAC907490FBA
:20ABC0000843A074A878E07469462846FEF769FF68460079207568460078607519E0012057
:20ABE0002071207B2A788008D2078000D20F10432073084029788907C90F89000843207327
:20AC000024213046FDF736F90BE0032020710520207325213046FDF72DF9B07F4006400E66
:20AC2000B07703A92046FDF701F8022806D0002804D0B848B6492B3010F08DFA02983FE751
:20AC4000FFB5B54A0E4607CA97B002AB07C3002701970C971798FDF7D6F8050005D0287811
:20AC6000262804D008201BB0F0BDAC48FBE7A87F8007800F012807D000210022179801F01C
:20AC800053F8040007D101E00121F6E7A148A049623010F060FAA87F8007800F16900128E3
:20ACA00014D0022824D09B4899497B3010F053FA01210022852E31D01EDC002E26D0812E10
:20ACC00026D0822E26D0832E1ED125E0002EEFD121462846199AFEF7A3FE0028C3D11998BA
:20ACE0008078019019980078C007C00F0C90DFE71998002808D1DBE7862E11D0882E11D00A
:20AD0000892E11D08A2E11D00720ACE710460EE008460CE002200AE0032008E0052006E0A8
:20AD2000062004E0082002E0092000E00A200022227101216A461176211D0791002801D0EF
:20AD400020710BE1169801280CD0A66AE06A0222012111900020A0602846173002291AD098
:20AD6000012119E0E66AA06A1190032030702078FB23C006C00F7070B07801221840019B90
:20AD8000F37080080C9B800018430221B070002070713071DEE70021890009190861681CE3
:20ADA000022A01D0012100E00021890009190861B0788007800F01285ED1119880788007A1
:20ADC000800F012858D1119800790190119840790090169801281DD0317908A80174717970
:20ADE000017508A8027C01980099024008A8007D0840149010433FD049491A98884207D3D8
:20AE000001218904884215D346490968884211D2102028E70CAA0DA91998FEF742FE08A8E3
:20AE2000007C01990840307108A8007D009908407071D6E720463C3021460090F0311698CF
:20AE40000191022834D000211A9B20460C33FEF791FE0028DDD12046503021460090F4315B
:20AE600016980191012825D0002120461A9B149AFEF780FE0028CCD111988078400702D494
:20AE8000E87FC0072BD0169902A8012914D0119909784900405A21780907490F4900C840C2
:20AEA0008707BF0F2AD0012F14D0022F0FD113E00121C9E70121D8E721780907490F490027
:20AEC000405A119909784900C8408707BF0F032F04D004E0022711E001270FE0022716980E
:20AEE00001280BD1B078FB210840E97FC907490F0843B07020780007400F30702078400858
:20AF00004000207011990FE0500E0020440D00202C9E0000A90500001CB40100023000005E
:20AF200000C001002800002049781022C907C90ED243114308402070C00622D4022F20D050
:20AF4000012F20D00020A061E0612062606220461830A060E87F40084000E877204606A91A
:20AF60008830FCF73FFE002805D0022803D0B449B44810F0F0F825212846FCF77BFF0020CD
:20AF800071E6032008E020460D211B300FF0B6FF20461830A060042069460875E87F012135
:20AFA0000843E87705AA29461798FEF7B7FDD5E7F0B587B015460F0004460DD0A248854297
:20AFC00007D301208004854206D3A0480068854202D2102007B0F0BD2046FCF714FF060061
:20AFE00004D03078272803D00820F3E79848F1E7B07F8007800F012807D00021002220460B
:20B0000000F092FE040007D101E00121F6E78D488B491F3010F09FF80020002F05D0022F10
:20B0200008D0012F11D00720D4E701216A461171A06018E0234618336946A36008711022E8
:20B04000294618460FF0FDFE0DE021461831A16069460871A061E061206260620621284648
:20B0600006F05CFEA0612078C10714D04008400020700220694608702046183002907030FA
:20B08000FCF7B0FD022806D0002804D06D486C49423010F060F825213046FCF7EBFE002028
:20B0A00098E7F8B515460E460746FCF7ACFE040004D02078222803D00820F8BD6448F8BD00
:20B0C000A07F8007800F022802D06148C01CF8BD5D4886420ED3012189045C4A8E4202D3BD
:20B0E00013689E4206D3854204D38D4204D31068854201D21020F8BD00953288B31C21465C
:20B100003846FEF7B0FD112816D00028F3D1E17F2A7C4908D2074900D20F1143E1772A7C58
:20B1200049079206490FD20ED2001143E177A17F4906490EA177F8BDA17F0907FBD4204679
:20B140000822B11C34300FF07CFE3088608620461022294622300FF074FEE07FFD210840EE
:20B16000297CC907890F0843E077287C410820200155A07F08210843A0770020D7E770B5F0
:20B1800094B00D460646002B02D0072014B070BDFCF739FE040007D02078222802D3A07FDC
:20B1A000400603D40820F1E72948EFE7002D19D02D216846017046801022294601A80FF099
:20B1C00040FEE07F297C4008C9074000C90F0843E077297C40078906400FC90EC9000843A6
:20B1E000E07703E02E2168460170468009A9684600F0A3FCA17FBF221140A177C6E710B516
:20B200000C46FCF700FE002805D0104909688C4203D2102010BD0E4810BD2146FEF7FEFC0B
:20B22000002010BD05E00278401C002A01D0002070470A46491E89B2002AF4D101207047DB
:20B240002C9E0000ED06000000C00100280000200230000030B50346072903D00620DA784D
:20B260001C7916E00320FAE707290BD05500ED186D79072D01D0401EC0B2521CD2B2092AFA
:20B2800007D105E05500ED186D79072DF3D0F4E700222546641EE4B2002DE5D130BDFFB5B6
:20B2A00081B00C461646114620460A9F0B9DFFF7D1FF00280AD02079092803D3FEA1A020DA
:20B2C0000FF049FFA078C00907D019E0072E02D0112005B0F0BDFD48FBE701982880381D1F
:20B2E0006880002068712871EF8004982881284600F04BFC002803D1EFA1AD200FF02BFFF9
:20B30000E07821794018491CC0B22171092801D30938C0B24000001946718179F122490854
:20B320004900114081710020D3E7FFB583B016460F461C46002203210C9D039800F0F4FC43
:20B34000010008D033463A46019500940398FFF7A6FF07B0F0BDDD48801EFAE7F0B50546C3
:20B3600016460F4650888DB00022032100F0DCFC040003D1D0A1DF200FF0EDFE00206946F8
:20B380000871A078400603D1CBA1E3200FF0E3FE042F5ED32A78D007C017401C06D16178F3
:20B3A0006B78994255D12178090752D00121142A46DA012A42D0122A02D0132A40D128E0BD
:20B3C0000C2F3DD1A2785206520E012A38D0207800090001401C20706878607068460171C1
:20B3E00068792A790102114368460181E879AA790102114368464181687A2A7A010211431A
:20B4000068468181E87AAA7A010211436846C1811AE0062F14D12078000900012070718870
:20B42000012001F0EAF8022168460171C91E018168792A790102114368461FE0062F0AD0D5
:20B440006A461279002A1BD07088324601A9FDF720FB0DB0F0BD20780009000120707188DE
:20B46000012001F0CAF802216846017168792A7901021143684601810021C9434181E3E7F1
:20B480000028E6D07488684681766978C176022181830021C18304A80522009006231146A6
:20B4A0002046FFF742FF0028D3D089A1D6200FF052FECEE7F7B58CB015460C990D98FAF782
:20B4C00041F9C0B2082850D100206946888568880022032100F028FC040004D1FF2076A13A
:20B4E00063300FF038FE01230021E07822790BE04600361976799E4201D1491CC9B2401CEF
:20B50000C0B2092800D100201646521ED2B2002EEED1002902D117206946888504AB023387
:20B520000BAA00950C990D98F8F7B6FB0006000E07D002281BD0032817D0FF205EA18930EE
:20B5400011E06846808D00280FD002A9019100906888042301222146FFF7A1FE002804D039
:20B56000FF2055A176300FF0F6FD0FB0F0BD6878102108436870F8E700205A490246430051
:20B58000401CCA520828FAD3704700218170017809090901017000214170C170017170473B
:20B5A00070B50D460022032100F0BEFB040004D1FF2041A1CF300FF0CEFDA0786906C00931
:20B5C000C001490E0843A07070BD704710B50146012001F012F810BD3EB58DB200220321A7
:20B5E000284600F0A1FB040004D1FF2032A1E4300FF0B1FD207869460009000120700220C2
:20B60000087039488880C88000222846FDF741FA3EBDF7B505460078002700090C463E46B2
:20B62000012804D0FF2024A1F3300FF094FD287A03280CD0412020A1C0000FF08CFD0298C9
:20B64000002C068001D0278066800020FEBDEA89702710460A3086B2002C0AD06888A08017
:20B66000A8892081E28020460A3029690FF0E9FBE5E702980680E8E7F8B543680246D979D4
:20B680009C79090221435C7A1E7A25025C88981D3543241FA14238D11B79022B35D1042D59
:20B6A00034D0052D3DD0062D34D0402D2DD3061D0F461446284619E07372635C6C32636164
:20B6C000705F636F72652E6300000000043000007372635C6C326361705F636F72652E631E
:20B6E00000000000680E0020FFFF000000F0E3F908280AD01120207003202072A581E781DC
:20B7000026616078082108436070F8BD001DFFF7D1FEF8BD031D50880A461946FEF771FE2F
:20B72000F8BD001DFFF71AFEF8BD70B50D468CB006460022032100F0F7FA040031D02078B0
:20B740000007000F01282ED012206946887460780523801CC874082088822888C8826888DB
:20B760000883A8884883E888888302A90C20019100901A4621463046FFF791FD00280ED107
:20B78000F02300223146012000F090FE207800090001401C20706078801C607000200CB0B0
:20B7A00070BDCB48FBE71120F9E770B50D468CB006460022032100F0B7FA040006D02078FD
:20B7C0000007000F012803D00820E8E7C048E6E71321684681746178C17402218182C58239
:20B7E00002A906200523019100901A4621463046FFF755FD0028D2D12078000900012070AC
:20B800000020CCE7F3B581B00D4600220321019800F08AFA00260446002803D1AD49AE487E
:20B820000FF099FC2079A8423BD2AB48A949401C0FF091FC35E0E07841000F19401C7979F3
:20B84000C0B20091E070092801D10020E0702079401E2071B879C00708D00098019904286C
:20B8600015D09C49822018310FF075FCB8790007410F08D0400F019904280CD095498F20C5
:20B8800018310FF068FC009807280AD107E00846FEF74CFEEAE70846FEF713FEF3E7761C55
:20B8A000F6B228466D1EEDB20028C4D13046FEBD10B50022032100F037FA040004D1B52080
:20B8C000844980000FF047FCE07821794018C0B2E070092801D30938E07000202071A0786E
:20B8E00080210843A07010BDF8B517460D460022032100F019FA040005D0002D0CD0002FC8
:20B9000007D0062006E0072D01D00620F8BD0320F8BD0820A84204D86F486E4942300FF0BF
:20B920001AFC29462046FFF795FC0646002F28D0002E26D1E07821791CE0420012195379D6
:20B94000072B03D093791B075B0F04D0401CC0B209280CD00CE0400000198079F1231840F1
:20B960006B071B0F1843907100290AD104E00020491EC9B20029E0D1574856495A300FF044
:20B98000EAFB3046F8BDF8B50D460022032100F0CBF9040004D150484E4968300FF0DBFB28
:20B9A000681E052804D34C484A4969300FF0D3FB0921E2782079002310E0560036197779AB
:20B9C000AF4206D1B17949084900B1715B1CDBB21146521CD2B2092A00D100220646401E9C
:20B9E000C0B2002EE9D1092905D24800001981790122114381711846F8BD10B50446402896
:20BA000001D2072010BD00F056F8082802D03120000210BD0021314802E0491C082903D218
:20BA20004A00825A002AF8D1082903D049004452002010BD042010BD10B5402801D2072005
:20BA400010BD00F038F8082805D00021234A40001152084610BD052010BDF0B58BB016467A
:20BA60000C00074607D0002E05D06188402904D207200BB0F0BD1020FBE72088002801D029
:20BA8000172801D90C20F4E7084600F014F808280FD0258803A82A46314602300FF0D1F9F3
:20BAA00001A8009062882B4607213846FFF73DFCDFE70520DDE701460020084A02E0401C77
:20BAC000082803D24300D35A8B42F8D17047000002300000B8B60000AD020000680E0020BF
:20BAE00000B51E2827D00FDC0C2820D008DC03000FF052FC0913211521211B1B17192100F6
:20BB0000122818D1072000BD302814DD3A3803000FF042FC030F11091100002000BD2148A0
:20BB200000BD042000BD0D2000BD0F2000BD082000BD112000BD032000BD10B50C4604F0D3
:20BB4000A0F800281ED0204602F013FE002816D022780E2A0DD00F2A0BD0022A09D0032ACB
:20BB600007D0102A09D010A17E200FF0F4FA002010BDA078FFF7B4FF10BD112010BD0AA17B
:20BB80008420F2E708A18A20EFE710B502F0A2FC10BD10B502F0EDFD10BD10B502F01AFDA1
:20BBA00010BD0000023000007372635C686F73745F6863692E630000F8B5054606ACC1CCC9
:20BBC000E44C21706270A370E070681C420827715200E14B667100218800001984460262C4
:20BBE000605C40008218002D0AD0002005E066464700366A401CF353C0B2665C8642F6D8A4
:20BC0000491CC9B20629E7D30026D21C9708B000BF0000198760304600F02AF9A15D761C20
:20BC20004843C219F6B2062EEFD3501B80B2F8BDF0B504468C46C7490020A500FF230246AE
:20BC40006D18C54E0C5D0BE02F6A5100795AB14204D1401CC0B2FF2B00D11346521CD2B25F
:20BC60009442F1D8002801D061460B70F0BD70B5B84C0023655CA678B54200D10346890098
:20BC800009199D420AD90C6A5E00A45B844202D11370012070BD5B1C9BB2F2E7002070BD99
:20BCA000FFB583B00C9C1F460D46060009D0002D07D0F01C80088000B04204D0102007B099
:20BCC000F0BD0E20FBE70598A04201D8A74201D90720F4E701460094019423463A46002011
:20BCE0000294FFF769FF2988814207D0814201D2042100E0092128800846E0E7009401945A
:20BD000023463A46029430460599FFF755FF28800020D4E710B5044600F0B4F8002801D01F
:20BD2000E0B210BDFF2010BDF8B505468A4816460C46854201D0062C01D30020F8BD0027A6
:20BD400069460F7028466A462146FFF790FF00280DD068460178204600F09CF8002EEDD0AA
:20BD60000028EBD12146284600F0A0F8F8BD3846002EF7D1F8BDF8B505460C460020764E76
:20BD80006946764F0870B5423BD0062C01D30720F8BD0A4621462846FFF769FF002830D028
:20BDA00068460178204600F075F823000FF0F4FA060404090C11161B01462846FEF742FA3E
:20BDC00015E0FDF735F812E001462846FFF7FDFB0DE001462846F7F7E4FE08E001462846A9
:20BDE000F9F73AFB03E05EA17C200FF0B4F9594A6846A10000788918096A40000E520020B6
:20BE0000F8BD3846F8BD5A4A1268914201D210207047062801D3072070470872002048725B
:20BE20007047F8B5044652480068844201D21020F8BD207A474A83009B18617A464D125C97
:20BE400011E01E6A4F00F65BAE420AD04A1C62721A6A4B00D25A228000F01CF86060002044
:20BE6000F8BD491CC9B28A42EBD861720520F8BD0EB5404B40000ECB009102930192694622
:20BE8000085A0EBD33498978814201D9012070470020704770B50C460546FFF7E9FF2D4A95
:20BEA000A900891889686043401870BDF8B504460E4600206946087005462046FFF7E2FF05
:20BEC000002803D126A1F3200FF045F92148214B815D8278B000C718914209D1E0B2694625
:20BEE0000870396A4000085A1B49884206D02EE069463046FFF79CFE002828D06846007878
:20BF0000396A40000C52684601783046FFF7C2FF054633000FF040FA060404090C0F141778
:20BF200029462046FEF760F911E0FCF75EFF0EE0FFF72BFB0BE029462046F7F7F9FD06E009
:20BF4000F9F783FA03E006A162200FF004F92846F8BD0000780E0020FFFF00000230000073
:20BF60007372635C686F73745F636D2E630000002800002028B401008107C90E002808DA11
:20BF80000007000F08388008C24A80008018C06904E08008C04A800080180068C840000672
:20BFA000800F7047BD4948788978884201D3401A02E02122511A0818C0B27047B74923314F
:20BFC00048788978884201D3401A02E02122511A0818C0B27047B1494631487889788842D3
:20BFE00001D3401A02E02122511A0818C0B27047A94910B50C310868FF22120290430122AB
:20C00000D20310430860A5490020233148708870233948708870463148708870A04806F06D
:20C02000BCF89F48401C06F0B8F8F6F7A3FB00F028F910BD20207047B4E770B50C460546A6
:20C040000026FFF7AFFF9549A04214D30A46203A00232046641EE4B200280BD08878105CB5
:20C06000287088786D1C401CC0B288702128F0D18B70EEE7012600F004F9304670BD202008
:20C0800070479BE770B50C4605460026FFF796FF82492331A04214D30A46203A00232046D9
:20C0A000641EE4B200280BD08878105C287088786D1C401CC0B288702128F0D18B70EEE738
:20C0C000012600F0DEF8304670BD202101700020704710B50446FFF77EFF2070002010BD48
:20C0E00070B50C460546FFF776FF6C494631A04215D30A46203A00232046641EE4B20028AA
:20C100000BD08878105C287088786D1C401CC0B288702128F0D18B70EEE7002400E0614C66
:20C1200000F0AFF8204670BD70B50C460546212904D9FF205CA147300FF00DF85548406810
:20C14000103840B2FFF718FFC6B20D20FFF714FFC0B2864207D2FF2053A14D300EF0FBFF4F
:20C1600001E0F6F74AFB21462846FFF766FF0028F7D070BDF8B507464948484C401E474E4E
:20C180000078254646362335002806D1A9786878212200F06BF800280ED0A1786078212218
:20C1A00000F064F8002814D0B1787078212200F05DF8002828D033E038496878C91C0F54B2
:20C1C0006878401CC0B26870212829D10020687026E03249607820390F546078401CC0B2E3
:20C1E0006070212801D1002060702D4F7F1E3878002815D0A1786078212200F037F8002813
:20C200000ED0002038700BE02449707826310F547078401CC0B27070212801D100207070CD
:20C22000A9786878212200F021F800281DD0A1786078212200F01AF8002816D0B178707847
:20C24000212200F013F800280FD0F6F7B8FA144805F0ABFF01214903884203D016A1C1205C
:20C260000EF079FF0E4805F0B8FFF8BD401C884205D0904201D1002901D000207047012000
:20C28000704710B5064805F090FF002801D1F6F785FA10BD00ED00E000E400E0F00E00206E
:20C2A00069000020072000007372635C736F635F72616E642E6300007372635C736F635F08
:20C2C00072616E642E630000FEB5F54C07466068FF213E0181552178FF2913D00901083103
:20C2E00041583246491E083209020192090A805800F0CCF9002802D02478254615E061688F
:20C30000207888552770FEBDE548426801981158280100900830105800F0B8F9002806D184
:20C32000DF482C46416800980D5CFF2DECD1DC482101406885554754FEBD70B5D84A044622
:20C340000020157A53680AE00201561C9E5DA64203D10C329A588A4204D0401CC0B28542F8
:20C36000F2D8FF2070BDF8B5CD4F3E7801F00AFE0146FF2E68D0340125467868083540592D
:20C3800000F084F9022802D9786840595AE0C4494868025D0A70A11C425C002A0CD0521E11
:20C3A000425441590122D20589180902090A41513046FFF789FF30E0631CC25C0092221D90
:20C3C00094468258002A10D001239B029A420FD99205920D43595703DB191B021B0A435124
:20C3E0006346C3589A1A920A09E0FF21C1540AE0435952039A181202120A42510022425403
:20C400003046FFF761FFA6480C344168C268009809598000125800989047A14C2078FF2850
:20C4200012D001F0AFFD01462078626800010830105800F02BF9012896D920786168000125
:20C440000830085801F091FDF8BDF8B51C4615460E460746FF2B03D392A1D3200EF07BFE68
:20C460008F48FF21C760456004720674017000224270104604E00201521C401CA954C0B24E
:20C48000A042F8D3F8BD70B5854C06466578207C854203D383A1E6200EF05DFEE068A9006E
:20C4A00046506078401C6070284670BDFFB581B01D46FF2401F066FD794F064679780198EA
:20C4C000814203D877A1F4200EF045FE74480021037A406810E00A019446521C825CFF2A05
:20C4E00024D0019FBA4205D162460C328758029A97421DD0491CC9B28B42ECD8FF2C17D02C
:20C5000021014B1C019AC2540B33029AC250039B634F0022012B0ED00B1DC25001239B027E
:20C520009D4216D9AA05920D08D008E00C46E1E7FF2005B0F0BD0B1DC550EFE71A465303BB
:20C540009B190E461B0208361B0AAA1A8351920A09E0002D00D101256B039B191D022D0A9A
:20C560000B460833C550891C42543D463E782046FFF7AAFE2878B04217D001F003FD0146F1
:20C5800028786A6800010830105800F07FF8012807D92878696800010830085801F0E5FC3C
:20C5A00003E001F010F9F5F7AFFE0198C1E770B50C46054601F0E6FC064621462846FFF718
:20C5C000BCFEFF2817D0364D04012046696808300858314600F05AF801210903401869682C
:20C5E000A41C095D400B002901D089020818002800D1012070BD002070BDF3B581B00F4663
:20C600000198FFF79AFEFF282AD0254D2E7869683246344604E0844205D026462301CC5CC0
:20C62000FF2CF8D11CE0FF2C1AD0A64221D11001085C2870FF281AD001F0A4FC2A78014683
:20C64000120168680832805800F020F8012809D92878696800010830085801F086FC08E06D
:20C660000020FEBD01F0AFF8F5F74EFE01E001F084FC39460198FFF79AFF22016968FF2300
:20C68000541C0B558A5C3301CA54FEBD401A00020121000AC905884200D900207047000007
:20C6A0003C0F00207372635C736F635F74696D65722E6300F0B500241C4A01211C4B080352
:20C6C000546018601B4B1C601B4C20601B480469E443E406E617046910252C430461184CAD
:20C6E0006160184D2960761C00E020BF1F68002FFBD0002E03D107691026B74307619068B7
:20C700008005906801D5104A10436960A160002119600121084A09031160F0BD10B5044608
:20C72000FFF7C8FF2060002010BD000000C5004080E100E000C1004080E200E000ED00E079
:20C7400000C3004000C0004000FCFFFF70B51F490A68002A17D000231D4601244A68521C01
:20C760004A60092A00D34D600E792246B2400E6816420AD072B60B6893430B6062B649682E
:20C780000160002070BD052070BD5B1C092BE5D30FA136200EF0DFFCF5E70120104980057C
:20C7A00008607047EFF31081CA07D20F72B6012181400648036819430160002A00D162B6A1
:20C7C000EBE702480021016041607047700000207372635C736F635F6576742E63000000AB
:20C7E00000E200E0012081070860704701208107486070471048C068C00700D001207047B8
:20C800000D488068C00700D0012070470A484069C00700D0012070470748C0697047064984
:20C820008A69D20306D589698907890F814201D1012070470020704700040040F8B5F74CC3
:20C84000207EE17D88421CD00126F54D0027E07D215C14200A4642435019037C052B11D0BA
:20C86000037C062B1CD0037C072B28D0437C012B33D0ECA1EE480EF06EFC207EE17D884294
:20C88000E5D1F8BD0674E07D162807D0E07D401CE075491CC8B2AA5802210CE00020F7E745
:20C8A0000674E07D162808D0E07D401CE075491CC8B2AA5803219047DFE70020F6E7067464
:20C8C000E07D162807D0E07D401CE075491CC8B2AA580821EFE70020F7E74774E07D1628A4
:20C8E00007D0E07D401CE075491CC8B2AA580721E1E70020F7E770B50024CE4E0C20707211
:20C90000CD4825464473047328300476C475CB4805F043FCCA480575F572CA49601E8860AB
:20C920007571B570F57035717570C748E839057045701420604340180574641CE4B20B2CAD
:20C94000F7D30120F5F7E0FF0020F5F7DDFF0120B071F5F7A3FCBD48F5F7B2FCBC4C207035
:20C96000BC48F5F7ADFC6070F5F76EFF70BD10B5F5F795FFB64C2078F5F7C0FC6078F5F77D
:20C98000BDFCAC4C207A002803D0F5F746FD0020207210BD70B5A74CA079002804D0A1A134
:20C9A000AD480EF0D8FB70BDE07A002803D19DA1AA480EF0D0FB0126A6710025E572607AA1
:20C9C000042114225043964A801801749D488168491C04D0691E81600120F5F795FF00204C
:20C9E000F5F792FFF5F776FF05F018FDF6F777F89B480560056001209A49C0030860F6F72A
:20CA0000EDF891480078022804D0032804D1E078002801D0A67000E0A570F6F74CF870BD28
:20CA200003467F490B20142242435218203A127F002A04D0401E0006000EF4D17047142288
:20CA4000424351180A46803AD366012220390A777047012805D0032805D1002903D10020D5
:20CA600070470029FBD010B4724C00236370764A002890700CD002280AD007291AD20800A7
:20CA800078440079001887441505070D0F111300D37003E01B2000E03A20D0700120607051
:20CAA00010BC70475820F8E77720F6E79620F4E7B520F2E710BC0020704710B5624840781F
:20CAC000F6F714F880B210BD411E1422504310B5534A8418203C0A2902D8207F002803D134
:20CAE00050A161480EF037FB207F012804D0B3204CA180000EF02FFB0020207710BD70B5BF
:20CB00004D4C607B217B884201D1012500E00025F5F785FFF5F7EAFF617B227B914201D1DB
:20CB2000012100E00021A942EBD170BDF7B50646481E84468EB0C0B2142205905043384A46
:20CB400085180495287C2D1D07282AD1334C0027E07D227E824221D0235C059A934201D16A
:20CB6000012701E0002F04D0162811D0421CA25C225416280ED0401C227EC0B28242EBD1AE
:20CB8000002F0BD0207E002806D0207E401E04E00022ECE70020EFE7162020760498012299
:20CBA00002746046234C0A2813D8142041431C4808182038007F00280BD00498007C012876
:20CBC0000BD00498007C012803D01098807A012807D014A125480EF0BEFA1098807A012821
:20CBE0006DD104980E4B007C022843D00B4C207E162870D0207EE17D401C884203D109A136
:20CC00001B480EF0A8FA049901204874217E05986054207E162862D063E0000038110020ED
:20CC2000541100207372635C72656D2E63000000D40500005C1200201011002068120020B4
:20CC4000201100203C1200207A00002067C30000780000203DC800007D0200005E020000D5
:20CC600000F5004080E200E0CB0200001503000022030000607A059A0146904206D0014684
:20CC800014277843C018807C9042F8D1627A824208D1617A14225143C918897C6172012136
:20CCA000A17207E014224243D21814277943927CC9188A7414220C215043C0188174109886
:20CCC000007A06281DD201007944097949188F440C161412100EE07D002890D093E7002064
:20CCE00001E0207E401C2076B5E000210FE0B4210DE073210BE0322109E00A2107E0062168
:20CD000005E0FF20FDA1E0300EF025FA0021109802910068401A28601099097A002912D067
:20CD20000221401A0102090A296010980268406810180002000A68601098807A02281098AD
:20CD400003D0007B71E00421EBE7007A002812D002220298121810984368104610301818B8
:20CD60000A90E948029B4078984202D9E378002B03D00A9805E00422EBE7029BC31A0A98EA
:20CD80001818637A10300C2B1CD0637A14277B43DE4FDB195B68994214D0DD4F617ABC46A1
:20CDA00014235943D94BC9184B6889689B1B891B1B0209021B0A090A984237D8634535D89F
:20CDC000614533D831180A980123081A0002000A286010998018C9680002000A471ACD4AE7
:20CDE0009B05BC469F4201D2384610E00F1A9F4201D260460BE0944503D9511A0818401C65
:20CE000005E0974206D9101A4018401C404200285FDC03E0B9A1C0480EF09DF929680A98A6
:20CE200008180002000A6860002028726868102710300002000A68601098407AA872109805
:20CE4000007A687203280ED200280CD0FFF7D2FC002803D007E0002011B0F0BD029842213E
:20CE60000F1A32200290A8490878012801D0032809D148780299884205D9E178002902D1DD
:20CE80000299401AC7196B6828689B1B801B9C4601021B029E4A090A1B0A8F4219D81746C8
:20CEA000914216D8BB4214D8617A0C2915D0677A61460C22039200921422944B7A43D2183A
:20CEC00093689B1B834216D80397977C0C2FF3D173E0059801F04CF9BDE70498022205991A
:20CEE0000274627A0C2A00D0627A827461720120A07211B0F0BD0C2F5FD0002238469446B0
:20CF00001422824B4243D21853689B1B8B4225D2907BAB7A98421BD804980521059D017494
:20CF20007E4C207E16280FD0207EE17D401C884203D172A17A480EF00EF9207E2554207EE7
:20CF4000162800D0CDE6CAE6E07D0028F1D0F4E701208446907C0C28D2D102E061460029BF
:20CF60002AD03D46009014202A46424367480621161831741C38007E1628684816D0017EAD
:20CF8000C07D491C814203D15CA166480EF0E3F86248017E4554017E16290BD0017E491C95
:20CFA0000176B57C0098A842DDD106E0C07D0028EAD0EDE70021F3E7009704990220534DCF
:20CFC0000874607AB84207D1049900988874059860720120A07221E003980C2F0FD00C286C
:20CFE00003D146A150480EF0B6F80398142250434019059981740499009888740EE00C288F
:20D0000003D13EA149480EF0A6F803981422504340190599817404990C208874012011B039
:20D02000F0BD70B50D46424A441900210B46101A8B4103D231A13F480EF08DF83E4885427C
:20D0400003DD2EA13D480EF086F83D48854203DA2AA13C480EF07FF83B48844205DA002CDF
:20D0600001DB204670BD384800E03848201870BD401E70B5C0B21421484324494418607BA3
:20D08000062813D201007944097949188F44020C0A080604002067E0B42010E073200EE033
:20D0A00032200CE00A200AE0062008E0FF2013A1E0300EF050F8617B0020002954D002217B
:20D0C0004018616840180002000AF5F70FFD0C256557174A441900210B46101A8B4103D2EB
:20D0E00006A114480EF037F81348854203DD03A112480EF030F81248854229E07372635C0C
:20D1000072656D2E630000007A00002054110020FFFF3F00FFFFFF0013070000381100205E
:20D1200007020000C5030000DD030000E3030000FF7F841EF50300000020A107F60300007F
:20D1400000E05EF8F70300000080841E00807BE103DAF749F7480DF0FEFFF748844207DA65
:20D16000002C03DB204670BD0421A9E7F24800E0F248201870BDF0B5064683B0F0480190B7
:20D18000457A029534687068001B0702ED483F0A001B00900C2D2DD0142029464143EA48E9
:20D1A0000122081884464168E64892058646081B904210D3631A93420DD302467046724569
:20D1C00003D900984018401C05E073450ED9411A0819401C404200280CDA60460295857CFD
:20D1E0000198C0790028D5D003B0F0BDD049D7480DF0B1FF0298854226D014214843D24919
:20D200000123401802908068CE499B058C46011B8646994210D3221A9A420DD363466145A2
:20D2200003D900997144491C06E0194662452DD9091A0819401C4142002905DD0298B17A7A
:20D24000807B814200D374460C2D15D0BE491420454368184268121B1202120ABA420BD242
:20D26000B37A827B934200D38468857C0198C0790028B9D10C2DEAD13068A042B4D0E01980
:20D280000002000A3460706003B0F0BDA849AF480DF061FFD8E7F0B5AD490446486885B0F0
:20D2A000C005C00D1CD0103840B200280CDA0207120F083A920892005118C9698007C00E20
:20D2C000C1400806800F09E08108A24A8900891809688007C00EC1400806800F002808D0C4
:20D2E00000272078002806D0012804D0002005B0F0BD0127F5E72079062813D20100794484
:20D30000097949188F44020C0A080604002018E0B42010E073200EE032200CE00A200AE07E
:20D32000062008E0FF208249E0300DF014FF21790020002905D002214618814D002F02D0CD
:20D3400003E00421F8E70020E871694602AAA068F5F7D6FB694608228A56E06801A980180A
:20D360000122C01C1F2801DA019209E003AAF5F7C7FB6846007B002802D00198401C01900C
:20D3800000990198401810300002000A0190881B0002000A0090607969468872009803903A
:20D3A000F5F73DFB009A019B121A181A6A4912020002120A000A8A4216D8884214D86846A8
:20D3C000FFF7D9FE00990398814205D088190002000AF5F78BFBA0600120E979002986D093
:20D3E000002FB0D005B0F0BD0020F6E7F3B58FB05A480C460B9004F0D8FE594A0F99504FF5
:20D400005618584D203E00280BD05748007D002803D056A158480DF09EFE207801287CD044
:20D420005AE1687B16280CD0687B297B401C884203D14EA151480DF08EFE2078012804D08D
:20D440000CE0287B0028F4D0F7E7F07F002803D046A14B480DF07FFE0120F077697B0F9802
:20D460001422484E5143891908742078022822D0687B142148438619207930726079707242
:20D4800032460C323146A068F5F73AFB0C2030560F2804DD1F3830733068401C30600C21C1
:20D4A0007156301DE26801905018C01C1F283EDA01200199F7E026494868C005C00D21D0A6
:20D4C000103840B200280CDA0207120F083A920892005118C9698007C00EC1400806800FDE
:20D4E00009E081081B4A8900891809688007C00EC1400806800F002804D105201BA10002E7
:20D500000DF029FE687B1421484386190021E0686A460691117006A900E0D3E0F5F7F0FA5C
:20D520006A46002010560F282EDD01202DE0AEE0FCD00000F70300000080841E00807BE1F3
:20D540005C120020FFFFFF00541100201307000000ED00E000E400E0FFFF3F006812002039
:20D560003012002010110020201100207372635C72656D2E6300000011050000EF04000035
:20D58000F4040000500F002000200699401807900220B0722079307260797072A068311DD6
:20D5A000C01C06911F2801DA012009E0F5F7A8FA68460078002804D0069806990068401C1B
:20D5C0000860307A062813D201007944097949188F44020C0A08060400200FE0B4200DE0B8
:20D5E00073200BE0322009E00A2007E0062005E0FF20FE49E0300DF0AEFD00202179002955
:20D6000043D00221401806907168103008180799089009180698081A0C900020F871F5F783
:20D62000FEF904463060079820180002000AF060787A0C2825D0797A14204143EC480818CC
:20D6400040680899029040180002000A0390707A6946887402A8FFF78EFD0299039A091BDC
:20D66000121B09021202E34B090A120A0C98994207D8824205D80299069808180002000A9D
:20D680003060F8790028C8D110E00421BAE704AA0199F5F735FA6846007C002804D00198F0
:20D6A00001990068401C08602078B072687B162806D0687B401C68730B9804F08EFD47E090
:20D6C0000020F8E7F07F002804D0A320CAA1C0000DF041FD0120F077CA490F980874207861
:20D6E000022803D1C4A1C8480DF035FDC54E207930726079707232460C323146A068F5F75E
:20D70000FFF90C2030560F2804DD1F3830733068401C30600C22B256301DE16801908818CC
:20D72000C01C1F2802DA012001990BE003AA0199F5F7E6F96846007B002804D001980199DA
:20D740000068401C08602078B072AE4901200875687B297B884224D07C7A0C2C23D0F5F7FC
:20D760005EF914214C43A24961180A7C042A18D00A7C032A15D04B6889681B1A081A1B02DE
:20D7800000029C4A1B0A000A102B0AD31146934207D8884205D8687B297B884201D0F5F79A
:20D7A0008AF911B0F0BD687B297B8842F7D111B0F0BD10B50020F5F794F810BD10B50120E1
:20D7C000F5F78FF810BD914800787047F1B5009802281ED08E4C607A0C2803D186A18D48F3
:20D7E0000DF0B9FC0026A6710125E572607A032114227F4F5043C0190174F5F761F90098FC
:20D8000000280BD001282AD003287AD07AA1824845E07E480078F4F777FDF8BD7F48007FCB
:20D82000002804D02B2074A140010DF094FC65717A4D00202E60F5F767F8A968481C04D0DF
:20D84000012300221846F5F795F8607A617A401CC0B2142251437A5801219047F8BD0120BD
:20D86000F5F752F8607900280DD06C488068401C09D0607A617A401CC0B2142251437A58A4
:20D8800006219047F8BD6548007F01280AD0022812D0032822D0042834D057A160480DF0B0
:20D8A0005AFCF8BD2079002803D02671F5F70DF9E5705A480677F8BD207A002802D1F4F797
:20D8C00083FD2572607A617A401CC0B2142251437A580021904751480677F8BD4F4F01238D
:20D8E000397B78680022411A1846F5F743F82079002803D02671F5F7E8F8E5700220387775
:20D90000F8BD19E0454E217870680123411A00221846F5F72FF8207A002802D1F4F754FD72
:20D920002572607A617A401CC0B2142251437A58002190473577F8BD607A617A401CC0B255
:20D94000142251437A5805219047F8BD10B5304C607A0C2803D128A132480DF0FCFB607A45
:20D96000617A401CC0B214225143214A52580421904710BDF0B583B00C200290F5F74FF88D
:20D98000234C0090617A284801900C2920D0617A1420414316480918097C042918D0617A00
:20D9A000142251430818007C032879D0019900980B6849681B1A081A1B0200020D4A1B0A45
:20D9C000000A102B6CD31146934269D8884267D812488068401C03D007A114480DF0BBFB25
:20D9E00000206071607A0C282AD121E0FCD0000054110020FFFF3F007372635C72656D2E88
:20DA000063000000201100201E050000780000205C12002054050000A70500003C12002096
:20DA20009B050000AE0500004C120020EA0500006078002804D0FE48C178417081780170B8
:20DA4000607A0C2815D0607A1421FA4A48438018007C04280DD1607A0290607A0121142338
:20DA6000584380180174607A58438018807C6072A172F14D687B297BF04F884233D0F04E01
:20DA8000287B142148438019007CC05D0128287B07D048438019007CC05D02282FD044E044
:20DAA000FCE1142148438019807A01280AD0287B0221142250438019007CC155287B162898
:20DAC00008D009E0287B0021142250438019007CC1552AE0002001E0287B401C2873687B45
:20DAE000297B8842CCD1D74D287D00284DD0287CC15D012928D0C05D022830D03BE0287B24
:20DB0000142148438019807A012803D0CEA1D1480DF021FB297B00201422514389198872EB
:20DB2000297B51438919097CC855287B142148438219287B48438019017C0098FEF7F6FFA5
:20DB4000287B1628C8D1C5E7A97A012904D00221C155002028750EE00021C1550BE0A87A56
:20DB6000012804D0C520B8A1C0000DF0F4FA0020A872297CC855287D002806D0297CB14A80
:20DB80000098FEF7D3FF0020287502980C281ED014214843A7494018017C012917D10721EE
:20DBA0000174AD4D287E16283CD0287EE97D401C884203D1A4A1A9480DF0CDFA297E0298C5
:20DBC0006854287E162831D0287E401C2876607A0C287DD0A07A00287BD00020A072617A0F
:20DBE0001420414393480E189D49B56873680A46F6687C32CB67966055609A4D697E00295E
:20DC000016D00226617A14228A4851430818407B06281BD201007944097949188F440A14F7
:20DC200012100E0CE87D0028C4D0C7E70020CDE70426E7E700210FE0B4210DE073210BE0BC
:20DC4000322109E00A2107E0062105E0FF208649E0300DF080FA00212973687E022801D057
:20DC6000012810D12869009A4018821A1202120A422A08D93238032100026976000A2861FC
:20DC80003220287308E0322906D2207A00280AD1F4F79AFB012005E0207A002803D0F4F7D9
:20DCA000BCFB0020207262491022487820700978012901D0032906D101212171297B88422D
:20DCC00001D9421A1032A378002B00D0921C01E08DE09BE02179002901D1002B5DD0944678
:20DCE000624A00990092019A176852687F1A511A3F0209023F0A090ABC451BD85B4A97425B
:20DD000018D8009A914215D8297B884223D92B69421A9A1A1202120A101880190002000AAE
:20DD20002A616860002914D0032028770006000E3ED14CE000202071A070297B002925D0EF
:20DD40002869401880190002000A6860022028772EE00120E9E781420BD92A695118891968
:20DD60000902090A6960002801D00420DDE70220DBE7002B03D134A13D480DF0ECF928692B
:20DD800080190002000A6860002004E0296989190902090A6960287719E0287B00280FD0B5
:20DDA0002969081880190002000A68600220287728690123811900221846F4F7DBFD09E008
:20DDC000286980190002000A6860002028770120F4F79AFD607A1421484316490C22401864
:20DDE0008256012300206968F4F7C4FD0EE00120F4F78AFD0020F4F787FDF4F76BFD207A8D
:20DE0000002803D0F4F709FB00202072A078002804D0F4F75AFE0020E070A070607800288F
:20DE200004D00348C178417081780170207921E07A00002054110020101100202F12002014
:20DE4000500F0020201100207372635C72656D2E630000000C060000381100203A060000BE
:20DE6000D01100203C120020FCD00000FFFF3F008C060000002806D00020CF49E070097891
:20DE8000002900D12071CD48017EC07D814203D0CB484078F4F738FA0120E07103B0F0BDD6
:20DEA000F0B5C84C0746607A83B00C2803D1C6A1C8480DF050F9607A1421C74E4843801942
:20DEC000007C032804D06F20BFA100010DF043F9C24DA868401C03D0BBA1C1480DF03BF9BA
:20DEE000607A1421484381190C20085600216A4600911171C01901AA6946F4F701FE6A46B3
:20DF0000042010560F2801DD012000E0002000994018696840180102090AA9606079002807
:20DF200004D0012300221846F4F724FD03B0F0BD70B5AD4CAB4A0B1AA34214D3451AA542B3
:20DF400011D3934203D9101A43185B1C0BE0954204D9511A0818401C434204E0A349A44869
:20DF60000DF0F9F80023184670BD10B50146012300220220F4F7FEFC10BD10B50220F4F70D
:20DF8000C3FC10BD10B5F4F74AFD10BDF0B58D4D0446E87A83B0002803D18BA195480DF0D1
:20DFA000DAF8642C4DD3944900200246091B824147D39248417B007B814242D19048007D5D
:20DFC00000283ED1687A1421834F4843834EC519306801AA00196946F4F792FD694604208F
:20DFE0000856002802DD0098401C0090A96800986B680A18D21A1202824B120A9A4220D8DD
:20E00000AA7C0C2A08D014235A43D2195268511A0902090A814214D3B068401C05D00120B6
:20E02000F4F772FC0020C043B060306800193060A868009940180002000A7061012003B061
:20E04000F0BD002003B0F0BDF8B50646401EC5B21420614968434418207C002803D15AA14D
:20E0600069480DF078F86548017B407B81420CD0664A14234B439B181B7CB3420CD0162930
:20E080000CD0491CC9B28142F3D15D48017D002964D0007CB04261D10020F8BD0021F1E74F
:20E0A000217C052905D0217C062902D0217C072928D101212174C17D0023027E8A4221D007
:20E0C0000246565CAE4201D1012301E0002B04D0162911D04E1C965D565416290ED0491CD7
:20E0E000167EC9B28E42ECD1002B0BD0117E002906D0117E491E04E00026ECE70021EFE726
:20E1000016211176617C00292AD06774C17D0023027E8A4224D0425CAA4201D1012301E064
:20E12000002B04D0162912D04A1C825C425416290FD0491C027EC9B28A42ECD1002B0FD0D4
:20E14000027E0146002A06D00A7E521E04E00022EBE70021EEE716220A7601E01748002713
:20E16000217C01299CD1617C002999D10120F8BD70B505461420184A052168438018017441
:20E180000E4C207E162811D0207EE17D401C884203D116491E480CF0DEFF207E2554207E1F
:20E1A000162807D0207E401C207670BDE07D0028EFD0F2E70020F7E77A000020381100206F
:20E1C000780000205C1200207372635C72656D2E63000000EF060000541100203C120020B8
:20E1E000F1060000FF7F841E0020A107FCD000001307000032070000FF1FA107101100201A
:20E2000020110020FFFF3F006F070000500F00200702000010B509F063FC042803D009F05D
:20E220005FFC052803D106F0D1FE00280BD104F007F9032803D004F009F9032805D109F0D7
:20E24000B0FD002801D0012010BD002010BDF0B585B00746002668460D460672694638464A
:20E2600005F05CFA00287DD16846007800280BD009F009FDB84275D00022294638460AF06D
:20E28000CCFE00283ED120E006F077FCB842F2D000222946384608F01DF900287DD1019C28
:20E2A0009020005D2834002804D1607E002801D0012000E0002004902046603003908078EB
:20E2C00006F08AFB002804D008E0019C2834607EF1E7FF20FDA1DA300CF03DFF204620307B
:20E2E000417B00290FD0817B89070CD56E7001212970AE70AF80C17BA971218E2981618E69
:20E300006981467349E0039802A9807806F030FA002804D1FF20EDA1EE300CF01CFF684646
:20E32000007A002809D06E700D202870AF806846007AE8800120A8702FE0049800282FD0F5
:20E3400006F0B5FB00282BD068460078002806D101988030406A4188B94200D10670039836
:20E36000807800E01CE006F0CAF8002803D1D7A1DA480CF0F0FE6E700A202870AE70AF80A4
:20E38000A07EA8716676684605F07EFA002804D0D248CEA10E300CF0DEFE012005B0F0BD31
:20E3A0000020FBE77CB5CEA103C9CF4D002401910090AC7001F067FD2946EC7004204039B4
:20E3C000088710204887C81DC84AF93042800471C280E03844740C7084730475C0300477EF
:20E3E0001D300522694604460CF02BFD28462146BC3008F0F7F97CBDF8B5BD4C0D466060E1
:20E40000217006F057F805F0D1F8FFF7CBFF207809F03AF9B4498431084681380F4606468A
:20E4200006F08CFC606808F0D8F8284604F06EFC3946304609F057FC60680AF08AFE01F086
:20E4400022FDA9480021C170F8BDFEB50E461D46144601A905F062F9002839D1029880306B
:20E46000807A06F079F800280CD0684606F087F8002806D0002C03D006F01DF8A04206D252
:20E480000020FEBD91A19B480CF065FEF8E7009805F0AAFB3146009805F0ABFBE2B229466F
:20E4A000009805F063FD06F08FF8002804D1914886A11E300CF04FFE68460079012807D136
:20E4C00001A801F0E7FC8A4800218068803041820120FEBD30B40179002904D0012907D039
:20E4E00030BC00207047831D42880488022103E042880488831D0121204630BCA5E7FFB5B3
:20E50000794C85B00E460746C034608869460880154602A905F002F9002811D0002168467F
:20E5200005F059F9002823D1684602A9008805F0F5F8002804D06F4864A13C300CF00BFE8C
:20E5400068460088388068460088608066480021C23005F040F9002802D00020C0436080CB
:20E5600003988030807A06F037FA002803D007E0002009B0F0BD5F4854A156300CF0EBFDC1
:20E5800004A806F03CFA0028F3D0049805F068FB3070022807D0012805D056484BA17230F9
:20E5A0000CF0D9FDE4E70899049805F0F6FC2880002804D14F4845A165300CF0CCFD06F028
:20E5C00045FA002804D1E92040A180000CF0C3FD0120CEE73EB50446831D02AA694601A822
:20E5E000FFF78DFF002813D06846808820806846008960800020607168460078012808D009
:20E60000022806D03B4831A192380CF0A4FD01203EBD2071FBE7FEB5040004D135482BA1DA
:20E620007E380CF098FD304D0026203D687C002808D0667010202070A87CA070E87CE07031
:20E640006E7430E0284F403F3878002808D02C22B91C20460CF0F5FB0E2020703E7022E03F
:20E66000A87B002809D00120E070E87BA070287C60700F202070AE7315E01B480221C630CD
:20E68000029005F0A8F8002871D1174FC037F8880190F888042808D0052831D02146FFF76C
:20E6A000D6FD002859D00120FEBD0021204606F019FA0028F7D1287D00284ED066701320E6
:20E6C00020701C21A01C0CF019FC15E07372635C6C6C5F6374726C2E630000000D0200007B
:20E6E000FFFFFFFF1F000000AC120020FFFF000080000020390300000220A0702E75D2E7B9
:20E700000021204609F098FA002826D020781328C9D1A0783C28C6D1A088694604F07CFF03
:20E72000002803D0FD49FE480CF015FD00988030807A05F0E4FE002804D1F948F749001D90
:20E740000CF009FD009804F09FFF0028ABD0F448F24908300CF0FFFCA5E70221029805F006
:20E760003AF8002803D1F9880198814291D10020FEBD50E710B508F011FF002804D0E84821
:20E78000E649BE300CF0E7FC07F01FFF06F09AFA04F07AFA002804D07920E049C0000CF0FC
:20E7A000DAFC0AF0CEFC002804D03D20DB4900010CF0D1FC09F070FA002804D0F520D749E4
:20E7C00080000CF0C8FCFFF7EDFD04F0ABFE002804D0F720D14980000CF0BDFC05F01CFE0B
:20E7E00001F051FBCF480021C17040380171012141710222C270017010BD10B5C94C403CCB
:20E800002078002804D00A210E2001F002FB10BDFFF700FD002801D00C2002E001F033FB37
:20E8200000202071012060710A21E170207010BD70B5BC4C0646403C2078002804D03A2178
:20E840000E2001F0E6FA70BDFFF7E4FC002801D00C2010E0B34DE87808280BD2000100191A
:20E8600010223146443001F0DEFAE878401CE870002000E007202071012060713A21E17048
:20E88000207070BD70B5A74C0646403C2078002804D00B210E2001F0BCFA70BD3078002849
:20E8A00003D0012801D0122015E09E4D80352879082817D2FFF7AEFC002801D00C200AE05B
:20E8C000984833782979721C883001F098FB2879401C287100202071012060710B21E1708B
:20E8E000207070BD0720F6E710B58E4C403C2078002804D039210E2001F08BFA10BDFFF7E7
:20E9000089FC002801D00C2002E086490020C8702071012060713921E170207010BD8148F0
:20E9200010B540380178002904D00F210E2001F070FA10BD002101710E2181700F21C1708A
:20E94000FF2181710021C9430181774949680A7882728A8882814988C181012141710170A2
:20E9600010BD704910B540390A78002A04D03C210E2001F04EFA10BD6A4A0088C0325080C4
:20E980000120107100220A7148713C22CA70087010BD10B5634C403C2078002804D02B21D2
:20E9A0000E2001F036FA10BD0821A01DFDF7BCFB00202071012060712B21E170207010BD0D
:20E9C00010B5584C403C2078002804D005210E2001F01FFA10BD05F06EFDE08005F0C6FE1A
:20E9E000207200202071012060710521E170207010BD10B54B4C403C2178002904D031214E
:20EA00000E2001F006FA10BD00214156042911D000290FD0081D0DD0001D0BD0001D09D04C
:20EA2000001D07D0001D05D00A3003D00A3001D0122003E0084601F033FB00202071312054
:20EA4000E07001206071207010BD30B5354D0446403D28788DB0002805D02A210E2001F0A5
:20EA6000D8F90DB030BD10222146684601F0DBF91022A11804A801F0D6F9684603F00BFC10
:20EA800010222C46A81D08A901F0CDF9002020710E20A0702A20E070012060712070E0E7D3
:20EAA000F0B5204C85B0403C2078002804D03B210E2001F0AEF971E40020A0711948694648
:20EAC000C0304088888002A904F028FE002805D0002101A804F07FFE002865D16846114D0F
:20EAE00081880180283D684602A9008804F016FE002803D009490D480CF02DFB039E04A92A
:20EB000037468837B878283605F04BFE002804D106480249401D0CF01EFB09E0CCE600004A
:20EB2000FF020000AC1200208000002014050000767EB87805F050FF002803D1FB49FC4851
:20EB40000CF009FB05F0B3FF01214840314601431FD06A461188A279FD2352001219118127
:20EB6000A2794000515D4908490031435155A2791940014351556A46107C002802D0042020
:20EB8000014301E0FB200140A0794155A079401CA0710021684604F01EFE002804D1684635
:20EBA0000188808881429ED100202071012060713B21E17020707EE770B5DE4C054620781B
:20EBC000002804D034210E2001F023F970BD08F087FF052804D0284608F03FFD002000E05B
:20EBE0000C202071012060713421E170207070BD10B5D04C2078002804D00E21084601F020
:20EC000008F910BD0622CC49A01D0CF01AF900202071012060710E21E170207010BD70B578
:20EC2000C44C06462078251D002804D032210E2001F0EFF870BD3146002009F032F92870C9
:20EC400000280CD100213246084606F080F92870002804D106223146B7480CF0F2F801201F
:20EC600060713221E170207070BD70B5B14C05462078002804D030210E2001F0CAF870BD02
:20EC800008F073FD002803D104F0DEFA00280DD0287804F08AF8287806F0C0F90020207129
:20ECA000012060713021E170207070BD0C20F6E7F8B5A04C06462078251D002804D0172107
:20ECC0000E2001F0A6F8F8BD3146012009F0E9F80127287000280FD13246012106F037F9C8
:20ECE0002870002808D19348062231463C300CF0A8F890484030877067711720E0702770C4
:20ED0000F8BDFEB58B4C05462034A07B002804D028210F2001F07DF8FEBDA8781A2824D00F
:20ED20000EDC03000CF038FB16333333333321333333333333333333333333332121213354
:20ED40002A2824D00ADC1E3803000CF025FB0C20202020202020202020200E203A38030003
:20ED60000CF01AFB0415031503152888734988420DD81F21E173282121740120A0732888C8
:20ED8000694604F0CBFC002803D0022014E0122012E068460078019F00280FD0C637019E6B
:20EDA00000280DD0C736684601F05CF8002802D03878002806D00C20E073FEBD9C37EEE7D4
:20EDC0009D36F0E701203870A87830700020E073684601F05FF8FEBDF0B5564C07462078B0
:20EDE00085B0002804D025210E2001F012F862E6388802A904F092FC4E4E0021083600281B
:20EE00000CD00220207131603171E1800E20A0702520E0700120607120704CE6039D28463A
:20EE20000A30483501900020A8750522304601990CF007F8A87D0028F5D13888E080E5E71C
:20EE4000FEB53C4C06462034A07B002804D010210F2000F0DEFFFEBD1F20E0731020207482
:20EE60000127A7733088694604F058FC002810D1684600F0F7FF00280BD06846019D00783D
:20EE800028350028019806D0CA300178002909D104E0022007E08030406AF6E72035697BAB
:20EEA000002902D03A20E073FEBDA97B89070DD10621017068460078002804D10198318850
:20EEC0008030406A4180684600F0E4FF0020E0736F73FEBD70B5174D04462878002804D017
:20EEE00038210E2000F095FF70BD1F202871012068713821E97028702078002808D00128FD
:20EF000006D0022804D0032802D01220287170BD002606F051F8207807F061FC207808F047
:20EF2000E6FF20780AF0ABFA2E7170BDCCE600001F0500006C1200208C000020FF0E0000BC
:20EF4000F8B5FE4D06462878002804D01D210E2000F05FFFF8BD1F202871012068711D2152
:20EF6000E970287008F0BCFD0C27042857D0052855D0B0791224012801D000281DD1307800
:20EF8000002801D0012818D1F079002801D0012813D17088EA49021F30248A420DD2B28872
:20EFA000121F8A4209D22887B0886887B0790024012804D000280CD016E02C71F8BDDF48E6
:20EFC0004030807800282AD0DC4A3C320121084602E0DC4A0021012005F0B9FF040003D0D5
:20EFE000D949DA480CF0B7F8F079012801D0002802D105F0C8FF0446002C01D01F2011E091
:20F000003078012802D0002803D00AE00021022001E00021012005F0C6FF002801D02F71AF
:20F02000F8BD00202871F8BD70B5C44C2178002904D01E210E2000F0ECFE76E71F2121716C
:20F04000012161711E22E270217002781221012A01D0002A04D14078002803D0012801D044
:20F06000217162E700260C25012A09D008F038FD052803D008F042FA002806D0257154E72A
:20F08000618F208F08F083FBF6E726714DE7F0B5AD490446143103C987B0A84D05912035A6
:20F0A0000490A87B002805D021210F2000F0B1FE07B0F0BD1F20E873212028740126AE7369
:20F0C00022889F4B111F3020994243D261880F1F9F42FAD291423DD8E2899D4B911F9942A2
:20F0E000F3D2218A8F1F9F42EFD28A42F3D8628AFF23F4339A42EED8A28A954F13460A3B34
:20F100003F1FBB42E1D2C9088A4223D9E18A228B9142E0D821791220002902D0012919D1CA
:20F1200002E061790029F9D1217B002901D00129F5D108F0D5FC05280BD008F0D1FC0428D8
:20F1400007D0287D002804D105F017FD8149884201D00C20BDE0684604F0AEFA002801D0BC
:20F160000920B6E001220321009804F0E6FF009F042178880F3703903846FCF7D5FF3846B8
:20F18000039905F0C2F874A0009F00680690032106A81337FCF751FF002006A90A5C3A5451
:20F1A000401CC0B20328F9D30098218A8180618AC180A18A01810146002720318F73CF736A
:20F1C0006179002902D0012903D101E0C77600E0C6760622A11D1C300BF033FE0098052205
:20F1E00004A90A300BF02DFE0098A030067369460F71012101A8FCF720FF6946087941079D
:20F20000C206490F920F80068918C00F081869460871401D009B0928987601D2083098769F
:20F2200001220021184604F088FF00988A3005F044F9002804D145484349FC300BF08BFF66
:20F24000207B002806D0012808D03F4943480BF082FF40E000213B4A012008E037484030C7
:20F26000807800280FD0354A01213C32084605F06EFE00282FD000988030807A05F03FF93B
:20F28000002816D01AE000988030807A05F037F9002804D131482C490D380BF05CFF0098E1
:20F2A00004F0DAFA002800D153E72C482649093841E02A482449C01D0BF04DFF009804F07F
:20F2C000CBFA002804D025481F490B300BF043FF1F20E873ECE62079012801D0002803D125
:20F2E00005F051FE00280CD10320009905F05BFE002806D162882188009808F0F5F9002883
:20F3000007D000988030807A05F0F9F8002805D009E00098A0300770EF73C9E60F480A496E
:20F3200031300BF018FF009804F096FA0028BBD00A48054935300BF00EFF0AE76C120020EF
:20F34000FD3F00008C000020CCE60000060700007B0C0000FFFF0000112233001C080000F7
:20F3600038B5F94C2078002804D022210E2000F050FD38BD1F202071012565712220E070C6
:20F38000257008F0ADFB052802D00C20207138BD00202071684608F059FA0028F7D1009855
:20F3A0008030807A05F0ABF8002803D1E749E8480BF0D1FE009804F04FFA002804D0E448E8
:20F3C000E249001D0BF0C7FEDF4820300575E1480078F2F799FF38BDF8B5DB4D04462035A9
:20F3E000A87B002804D023210F2000F012FDF8BD1F20E873232028740120A8736288D64B07
:20F40000911F302099424CD2A1888E1F9E4248D28A4246D8E288FF23F4339A4241D82289E6
:20F42000CD4E13460A3B361FB3423AD2C9088A4237D96189A289914233D8002620886946A0
:20F4400004F05EF9022700280BD1009800F0F8FC002806D000988030416A0A78002A06D144
:20F4600001E0EF73F8BD826B1278002A01D03A2017E005228A71416A0E81426AA1885181CE
:20F48000426AE1889181426A2189D181406A01894289914204D88179082901D8914202D343
:20F4A0001220E873F8BD2188418000988030406A0770EE73F8BDFEB5A34C06462078002873
:20F4C00004D024210E2000F0A4FCFEBD012565712420E0702570304604F039FF002801D0DA
:20F4E000002000E0122020710028EED1964F0522E03738463D7731461D300BF0A2FC00268A
:20F500003E77701E69460880684604F031F9002819D168460788684601A9008804F0F0F89A
:20F52000002804D08A4889498F300BF014FE0198A0300573684604F01BF9002803D168461E
:20F5400000888742E7D12671FEBD38B57E4C05462034A07B002804D026210F2000F059FC28
:20F5600038BD1F20E073262020740120A0732888694604F0C5F800280BD1009800F060FCFE
:20F58000002806D000988030416A0A78002A06D101E002200DE0806B0078002801D03A2051
:20F5A00007E007200870009829888030406A41800020E07338BD10B5634C2078002804D0F1
:20F5C00006210E2000F025FC10BD002020710E20A0700620E0700821A01D0BF08FFCA1790D
:20F5E00001200143A1716071207010BD38B5564C05462034A07B002804D02C210F2000F0B5
:20F6000008FC38BD1F20E0732C2020740120A0732888694604F074F800280CD1009800F0FF
:20F620000FFC002807D00098014680314B6A1A78002A06D101E0022025E0896B0978002942
:20F6400001D03A201FE04030007F00281DD00822A91C181D0BF0F5FB00986A898030416A87
:20F660008A81406A294610220C310E300BF0E9FB009803218030406A01700098298880305A
:20F68000406A41800020E07338BD0C20FBE770B52D4E044630780C25002804D018210E2063
:20F6A00000F0B7FB41E402F0CBFE032865D002F0CDFE032861D06079002801D001282DD156
:20F6C000A079002801D0012828D1A07B002805D0012803D0022801D003281FD1607B0028C9
:20F6E0001CD0C0081AD1628801208003824202D82188814203D9207901280FD119E02079C3
:20F70000002806D0012814D0022805D0032805D102E0202A0BD30CE0A0290AD2207904287E
:20F7200005D12088202802D36188884201D9122523E00548217920308175607900280DD05C
:20F7400001280FD019E000006C120020CCE600007F080000800000207B0C0000FA4A002145
:20F76000204607E0F9488078002806D0F74A0121121F204608F01BFB05460120357170710A
:20F780001821F170307058E410B5F04C403C2178002904D01A210E2000F03BFB10BD01780B
:20F7A0001F2902D91220207106E0002121710278411C104608F09EFB012060711A21E1708E
:20F7C000207010BD10B5E14C403C2178002904D020210E2000F01DFB10BD01781F2902D9E8
:20F7E0001220207106E0002121710278411C104608F06FFB012060712021E170207010BD3D
:20F80000F8B5D24C403C2178002904D01B210E2000F0FFFAF8BD012666710C2121710078CE
:20F820000025012804D000285CD01220207188E002F006FE002835D102F008FE002831D1E1
:20F8400008F021FAC24988422CD108F07AFA002877D0684603F0C6FEBB4A00990C3A9160AE
:20F86000002803D0BB49BC480BF075FC01220321009804F008FC009808F0CDFB00988A3098
:20F8800004F01BFE002804D1B348B24908300BF062FC009803F08CFA002851D0AE48AD4991
:20F8A0000C301CE002F0CCFD02284AD102F0CEFD002846D1A5482038807D002841D0012870
:20F8C0003FD004283DD008F03CFA002839D0002003F06EFA002833D09F489E4924300BF0BE
:20F8E0003AFC2DE002F0ACFD032804D002F0AEFD032820D025E002F0A6FD0090002003F036
:20F900004FF900281DD1257100988030807A04F0F6FD002804D190488E493E300BF01BFC9E
:20F92000009803F0B1FE00280BD08B48894942300BF011FC05E0002003F032F9002800D14F
:20F9400025711B20E0702670F8BD38B57F4C0546403C2078002804D02D210E2000F059FA69
:20F9600038BD2888694603F057FE002801D002200FE00098CA21095C002909D13321095C3D
:20F980000F2901D0102903D1FC21095C00290BD00C2020710E20A0702D20E0702888E08023
:20F9A00001206071207038BD1022A91CD8300BF048FA00980421C03081720020E9E738B517
:20F9C000624C0546403C2078002804D02E210E2000F01FFA38BD2888694603F01DFE00280E
:20F9E00001D002200CE000980146C030827A002A05D12031C97C0F290DD010290BD00C2072
:20FA000020710E20A0702E20E0702888E08001206071207038BD052181720020F0E77CB5B1
:20FA20004A4C0546403C2078002804D037210E2000F0EFF97CBD2888694603F06FFE002857
:20FA400007D002202071012060713721E17020707CBD01987F220146283002724272002295
:20FA60008272A87822318870E878C870287908712271E8E71CB5354C403C2178002904D0AF
:20FA800013210E2000F0C5F91CBD0088694603F045FE002801D0022006E001982421095CCC
:20FAA000801C012902D00C20207107E00022019922712831097A21720088E0800120607172
:20FAC0001321E1700E21A17020701CBDF8B51F4C0546403C2078002804D035210E2000F011
:20FAE00098F9F8BDA878002801D0012804D1A888FF21F531884201D912202071288869466D
:20FB000003F08AFD0126002806D00220207166713520E0702670F8BD009800270246C030D5
:20FB20000770AB8801464380104680300677AA78012A00D000220A70407F002801D003F02A
:20FB400027FA2771E3E700008C000020AC120020FFFF0000CCE600002D0A0000F8B5D44EE2
:20FB600004463078002804D03D210E2000F051F9F8BD2088694603F04FFD002801D002206B
:20FB800027E0009F6488FD883A896800B988401C844217D3C7484143800050430BF0BAF982
:20FBA000401EFF2180B2F531884200D90846844200D22046691C401C0BF0ACF96D1C6843CB
:20FBC000401E85B2E820C05D002800D17D84F58000203071012070713D21F1703070F8BD25
:20FBE00070B5B34C05462078002804D033210E2000F00FF956E502F023FC002801D00C2017
:20FC000018E02978002911D00A290FD014290DD01E290BD0282909D0322907D04B2905D04E
:20FC2000642903D0FF2901D0122003E0284603F04BF900202071012060713321E1702070D9
:20FC400030E570B59A4C05462078002804D03E210E2000F0DEF825E502F0F2FB002803D16D
:20FC600002F0F4FB002801D00C2003E0287808F04DF900202071012060713E21E1702070DA
:20FC800010E510B5017801240B000BF085FB3FBFBF21BFBF4C94BFBFBF2427BFBF464F614E
:20FCA000BFBF59BFBFBF2B97BF9B9FBF797DBFA38185888C6590BF5DBF555275A7ABBF3710
:20FCC0002F33BB6DAFBF71423F3B4969B3B7C000FEF750FD9BE0FEF790FD98E0801CFEF7DB
:20FCE000D1FD94E0801CFEF7E3FF90E0801CFEF780FE8CE0801CFEF792FF88E0801CFEF749
:20FD0000B4FF84E0801CFEF793FD80E0FEF7ECFD7DE0801CFFF7DEF879E0FEF769FF76E09C
:20FD2000FEF7BEFE73E0FEF74BFE70E0FEF7F7FD6DE0FEF72EFE6AE0801CFEF786FE66E035
:20FD4000801CFFF797FE62E0801CFEF7DAFF5EE0801CFFF775F85AE0801CFFF73DF856E05C
:20FD6000801CFEF7FEFD52E0801CFEF725FF4EE0801CFFF754FE4AE0801CFFF737FC46E0E9
:20FD8000801CFFF7DDF842E0801CFFF74DF93EE0801CFFF77CF93AE0FFF7E2FA37E0801C3E
:20FDA000FFF71AFB33E0801CFFF785FB2FE0801CFFF7CBFB2BE0FFF7FEFB28E0801CFFF718
:20FDC00066FC24E0801CFFF7DFFC20E0801CFFF717FD1CE0801CFFF7F5FC18E0801CFFF7A1
:20FDE000B4FD14E0801CFFF7EAFD10E0801CFFF76DFE0CE0801CFFF7B1FE08E0801CFFF751
:20FE000020FF04E0801CFFF7EBFE00E00024204610BD274A2032537C002B03D19074D17453
:20FE200001205074704730B5134606E0CC18203CD51AE47F5B1E4455DBB2002BF6D130BDF2
:20FE4000017800290CD14121095C002908D18030017C002904D0007C042801D001207047DF
:20FE60000020704701784068002903D00178002905D100E0E4E740304078002801D000202A
:20FE80007047012070470A4900208031886740310871704710B50178012908D14068803086
:20FEA000417F002903D00021417703F071F810BD6C120020C409000070B5FC4D00246C70AB
:20FEC0002C70AC616C72AC720120E872F8484470C473AC62F7482C6302F05FF9002804D0B5
:20FEE000FF20F5A14F300BF036F92C7770BDF8B5F54902250D60F5490026CE630127CF6366
:20FF0000F349C96A09070DD4F24AD36AF2494B62136B8B62536BCB62936B0B63D26BCB0551
:20FF20001A434A63ED4C002823D0012825D0FF20E1A1A2300BF00FF9E948A063FF20043048
:20FF40006063276303202061E64996204860D7491C2008560B22D243811A904237D011DCC6
:20FF60001C313AD00A2938D0142934D0182911D12FE0DD486061DD4802E0DD486061DD4884
:20FF8000A061D9E708301FD004281BD0082817D00C2812D0FF20D8A176300BF0DCF8DB4904
:20FFA000D9488860DB48DA494160DB490160DB480560DB4910204860F8BD0420E060EEE75A
:20FFC000E660ECE7FC2000E0F820E060E7E7F420FBE7F020F9E7EC20F7E7D820F5E710B57D
:20FFE0000C460146CF480BF0B2F9B048047210BDAF4840787047AD4A517010707047F8B56E
:020000040001F9
:2000000004460D465079117900020843690009190884501C01460E78012730464E783602B7
:2000200030438E78C9783604304309060843117800020843A9006050284608303E468640E0
:20004000002B0CD0012B04D0FF209BA1E9300BF082F8206B3043AF4038432063F8BD206B85
:20006000B043F8E770B50D460446082904D9FF2091A1FA300BF06FF80022002D0CD9AA48DB
:200080009100635809180B6053001B191B8C0B62521CD2B2AA42F3D3206BA449086070BD3C
:2000A00010B504460B22D2430C308C49944223D008DC1C3026D00A2824D0142820D018285D
:2000C00009D11BE02046083014D0042810D008280BD00C2807D0FF2087A176300BF03BF88C
:2000E0007248047710BD042000E00020C860F7E7FC20FBE7F820F9E7F420F7E7F020F5E700
:20010000EC20F3E7D820F1E76948007B70477349C2784A6202461378184653781B02184330
:200120009378D2781B041843120610430002C8617047252808D0262808D0272808D04100F0
:200140000A2807D8091D06E0022105E01A2103E0502101E0891DC9B2604A916061494861FB
:20016000704752498861704770B5002816D002224E4C6F4BA27203201860644D6248686010
:2001800000200126207500290AD001290FD002291DD049A167480AF0DEFF70BD0122E7E7D1
:2001A0006548012A01D0466070BD066070BD3F48012A006B05D00121490508432063696037
:2001C00070BD0121090508432063696070BDA069002804D1492038A1C0000AF0BCFFA16937
:2001E000A06A4018554988604A48554981605549C1600120216BC0030143216368602C48D3
:20020000C67370BDF8B54A4801688F084449BF004A68D206D60F10228A60002404603B4857
:20022000394981600C2069460870474D2C614249012008610BE000BF00BF00BF00BF00BF2C
:2002400000BF00BF00BF69460878401E087068460078002802D028690028ECD068460078A1
:20026000002804D14D2024A1C0000AF074FF2C610E48012144728472C1722D480760002E34
:2002800002D0274910204860F8BD01460A7810464A78120210438A78C9781204104309068C
:2002A000084300020D49000AC86370477413002094130020A81300207372635C68616C5F2E
:2002C0007263732E6300000080E100E0C01F004080000010C00000100017004000150040D9
:2002E0005B060000401500400601020025000302050103001F0003027372635C68616C5F70
:200300007263732E630000000040000400F501404080004080F501401011004080E200E031
:200320000013004076130020001600404016004000120040550200000010004040850040D7
:20034000488100401010004000110040FB4902200860FB4908607047FA490220086070472E
:20036000F9490870704710B5F84801F01EFF002803D0F749F7480AF0EEFE10BD10B5F348CC
:2003800001F02BFF10BDF4494860704770B5F34C0546A06AA84203D3ED49F1480AF0DBFE1E
:2003A00001202073EF49002025614860EE4845600120216B800501432163EC49486070BD24
:2003C000E64802210173C6210161E64A00215160816AE54AC63151600121026B89050A43E1
:2003E0000263E248416070470121E04889058160DA48026B8A430021026301737047DC482C
:2004000001214160C160D74900204860D6494860D24988627047D74940200862D6490A6812
:2004200002430A607047D4480168402291430160D049002008627047CF480168102291435A
:200440000160CE49012088617047CD490020C861C94801681022114301607047C849CA69A8
:20046000012A01D000207047C24A92685206520E524202700020C8610120704770B50C0093
:20048000054604D1D920B24980000AF064FEE00705D0012C03D0AE49BA480AF05CFE002D36
:2004A0000DD00221AD4801294172C472B24808D002290BD0A649B4480AF04DFE70BD0121DD
:2004C000F0E7016804221143016070BD016808221143016070BDF8B5A04C0025E27A9107AD
:2004E00001D5410713D4D306A849002B05DA4B7B002B02D08B7B002B09D0130702D50B78E2
:20050000002B04D1520703D54978002900D10125677A002201239849002F1BD0022630400F
:20052000284348D0084601688E089949B6004D68ED06ED0F10278F60002101608B4A954855
:2005400090600C206A4610708D4F39618B490120086114E0854D8F48A8600868800880005E
:200560000860A272E372F8BD00BF00BF00BF00BF00BF00BF00BF00BF1078401E107010780F
:20058000002802D038690028EED01078002804D14D208149C0000AF0DEFD002038616072FE
:2005A000A0720120E07274480660002DDBD0784810214160F8BD012F06D0022F0CD06449B5
:2005C00076480AF0C8FDF8BD08680425A84308606272E372A372F8BD08680825A84308601A
:2005E0006272E372A672F8BD5C4908757047F8B5664D5A49EC7B086B002C58D001245B4A31
:20060000E4039460A04308635B480768604C1021A16000210160001490600C206A461070DF
:20062000574C21615548012606610AE000BF00BF00BF00BF00BF00BF00BF00BF1078401EA2
:2006400010701078002802D020690028EED01078002804D14D205049C0000AF07CFD00204B
:20066000E060206160606061A061434807603F4900144860464910204860384CA07A0128D3
:200680000FD0022810D0444945480AF064FD0020E873207D022803D1424801688907FCD592
:2006A000F8BD36480660F2E734484660EFE72F4A906000200863087B2A4E002802D070680F
:2006C000012809D000222E4C2069012806D00023887A012804D006E00122F4E74023F7E7AD
:2006E000E768012F04D000271F43012802D004E02027F9E76368012B05D000233B432A4F32
:20070000022802D007E01023F8E73968012902D1E168012904D000211943022802D007E09F
:200720000821F9E73B68002B02D1E368012B3DD000230B4302283BD03EE0000080E100E086
:2007400080E200E000E100E092000020A8130020B8020100A20200000015004074130020AE
:20076000B3020000408100404085004000F501400080004040150040001200400010004091
:2007800000110040690300007E030000941300200013004000400004F8020100CF030000F0
:2007A0005E03000000E200E0001400400423C0E7002A01D0022100E000211943022807D177
:2007C0006068012804D17068012801D0012700E0002790480F4301680906090E02D06169FD
:2007E000012900D00021297300680006000E02D0A069012800D0002068738748006A002896
:2008000003D000F0DCF9012800D00020A8730020E060206160606061A06180494860804E6A
:200820008049307548683C4670620968B1620B46B17A022909D17178002906D07A4A5268DB
:2008400012780A40317891430ED000212970774FE10710D03978032908D0022906D002F079
:20086000D1FC0121B06A20E00121EFE707F022F90121B06A27E0A0060ED53878032806D0E8
:20088000022804D00221184602F0CBFC0FE00221184607F010F90AE0A00708D53878032867
:2008A0000FD002280DD00021184602F0BAFC5E4841680622B01C09310AF096FA002805D027
:2008C0000DE00021184607F0F6F8F0E75648317A40680078C009814201D1012000E0002008
:2008E00068702046FFF7F7FD387800280DD001281ED002282FD003284AD04D494D480AF071
:200900002AFCB07A022856D075E0A00701D507F0C6FC200702D5012007F0FDFC600702D55F
:20092000002007F0F8FCA006EBD507F059FCE8E7A00701D508F0E8FF200702D5012008F0B8
:200940004DFE600702D5002008F048FEA006D8D508F098FDD5E7A007BF25002802DA2C4019
:2009600004F022FF200703D52C40012004F05DFB600703D52C40002004F057FBA00602D5FC
:200980002C4004F061FE6006BBD504F04AFBB8E7A00701D506F0F0F8200702D5012005F05B
:2009A000B1FF600702D5002005F0ACFFA006A8D505F01CFFA5E7307B00281CD01749002289
:2009C0004A60022820D0012803D019491A480AF0C2FBB16A3069884203D8154917480AF0CC
:2009E000BAFB1048316941600120316B80050143316313494860307D012800D050E611485C
:200A000001688907FCD5F8BD3169B06A411805484160E9E740160040401500404081004060
:200A200074130020408500400015004092000020B8020100FD040000120500001305000018
:200A400000F5014000E200E02E48002101704170704770B5064614460D460120F0F7A2FC6A
:200A600028490120284B08709E60DC601D6170BDF8B504460120F0F795FC22490120087080
:200A800021494C60214900264E600321204D0906A960204F002C0AD0012C03D01EA14120C4
:200AA0000AF059FB3E60032000066860F8BD386001200006F9E710B51248017800290ED066
:200AC0000321134A0906916010494A680021002A03D0154A1268427000E0417001700020BF
:200AE000F0F760FC10BD07480178002907D007484068002802D00C480068C0B27047407890
:200B0000704700009300002000F5004000F1004000F5014000F200407372635C68616C5F65
:200B200063636D2E6300000000F400403B4800210170417010218170704770B50646144653
:200B40000D460220F0F72EFC01203449344A0870E41E14619660556070BD10B50220F0F75E
:200B600021FC2E49012008702E48002101604160816001202C49C005486010BD10B52748CA
:200B80000178002917D00121274AC905916025490B680022002B05D04B68002B02D08968D6
:200BA000002902D04270102103E0012141701F490968817002700020F0F7F4FB10BD174843
:200BC0000178002912D01748016800290AD00168002905D04168002902D08068002803D0D8
:200BE000002070470220704701207047407870470A48017800290FD00A480168002905D072
:200C00004168002902D08068002801D01020704706480068C0B27047807870479500002025
:200C200000F5004000F1004000F5014000F40040FFB593B0044600201D9E049015981C9DCE
:200C40001027082806D0E06901F014F8002809D03770CCE028880921384328801F980227E0
:200C6000017016E0E169012088710521E269C9029180E1698872E169F9480881E16900209A
:200C80008873288820210843288011211F98042701701F980225801C0390307810900A2071
:200CA0003070204618301190F5F7A1FC00206FE01598102809D1022D07D06846828A049931
:200CC0000398401A8270110AC1706846C08A1699884203D9E349097A149106E0884204D1BB
:200CE0001099002901D0317021E003990870000A48701E980088401BC01B83B2FF20C01B36
:200D0000984200D203460398149AC0190CA90092019002912020015D6846C08A0022F5F7AD
:200D2000DBFC3070002806D0C0B2832862D06846C08A208345E00F98002805D0C948006812
:200D400000790A2830D33CE06846008EC119C9B20491022D0FD01F99049A4978914203D1D7
:200D60006A46128C824209D0BE48049100680178032909D027E008461F994870B9480068D9
:200D80000178042906D008E000790A281BD201200F9009E06946C98A818003990498081853
:200DA00003900498281885B205AA14991198F5F721FC002805D11E980088401BB84200DB13
:200DC00076E7022D0ED01598102807D1049A03996846808A891A8870000AC8701E980580E2
:200DE000002030709F4800680078032802D0002017B0F0BD0220FBE7F8B50446406B00260F
:200E0000134600282BD0491F8DB2618F2A460832278F8A18BA4221D89A7840185F78110274
:200E200039430170090A41701A79DF78110239438170090AC1700571290A41712A46591D12
:200E4000801D09F0FEFF608FAD1D401980B26087626B002110180170417000E00926304617
:200E6000F8BD30B50B88048F9C4212D9446BE0184478057824022C430BD044790579240238
:200E80002C436404640CA41D1B190B801060002030BD822030BDF7B588B000256846058241
:200EA00005275DE00398417802780E0216434179027908021043000452D40A98012306808A
:200EC00005A802905B0200220097019530460999F5F702FC04004AD16846018A01830398AE
:200EE0004179027909021143437802781C021443B4421ED10A041CD44B0401215B0C89036D
:200F000000950B4301970295C17880780A02024320460999F5F7FCF9040011D10399487911
:200F20000A79000210430122D20310430871000A487103AA06A90898FFF793FF0400CED02C
:200F40000399009501970295487809780002084369468B8A00220999F5F7DAF9822C06D1D7
:200F600003AA04A90898FFF77CFF04009AD06846058209E0039841790279090211434904FE
:200F8000490C0171090A417103AA04A90898FFF768FF0028EED0822C02D020460BB0F0BD3A
:200FA0000020FBE730B50446406B002597B000280DD00B2268460270228F0281606B039104
:200FC000019000216846F2F72AFB6846057065636587258717B030BDF8B50F460546696B4B
:200FE0000020069E144600290FD0012B0DD1324639462846FFF74FFF002806D1002C04D019
:2010000032463946284600F044FEF8BD00220280C262831D0263C36142634287028720304C
:201020000170704710B50022D24302800420FBF7E4FA10BD10B596B00446FFF7B3FF208E9E
:20104000002808D0012069460870E06A019000216846F2F7E4FA0020E062206316B010BD5F
:2010600001280000AC1300200146098800200A0700D501200A06120F01D002221043CA0521
:2010800001D5042210438A0501D510221043490501D5202108437047FFB5A9B00600329DCE
:2010A000359C2B981F46229016D0007841060FD48106890E1E2909D021884A05520E0BD18B
:2010C0003A88172A08D3FE4A914205D0C10906D08006800E122802D003202DB0F0BD20466F
:2010E0002C302690F7492A980872002018AA039010726A46107404AA0A60339A4A6020AADE
:20110000908090812298007801908106681C1C90701F1D902B98890EC21C24922246203250
:201120001B92083A401C02920B000AF035F91FFDFD11FD1FFD8EFDFCFDFBFDFAFDF9FDFCF5
:20114000FDF8FDFDFDF7FDF6FDFDFDFDFDF5FD00032E76D102E018A9087219E3032028708A
:201160001C9917220A7000224A70CFE2052EF0D14178027808021043208320A98880249AC4
:201180005178127809021143618300287ED088427CD800202072E080401E60840298F5F74B
:2011A00026FA05202870A81C0190022000901BAA2A990298F5F71EFA002868D118A8807C08
:2011C000012803D002206870102002E00120687002202490002225A91CA8F1F7AAFD0028CD
:2011E0002BD120A8007D2499814226D13A880099801C511A814220DB10A8C18D0198017007
:20120000090A417001991CA8891C01910099019A891C009125A9F1F78CFD20A8007D0199ED
:201220001BAA091801910099081880B200902A990298F5F7DFF90028CCD00098022826D01E
:2012400064E272E018A9087261E2072E6DD341780346027808021043208320A98880249AF8
:201260005178127809021143618300280ED088420CD8012020725879197900020843E08061
:2012800000202073E06900F0F5FC01E098E0A9E000280ED1E169012088710521E269C902E8
:2012A0009180E1698872E16987480881E16900208873F01F60842298C01D60620298F5F700
:2012C00096F907202870681C009001200190002010A9C8852FE00198012814D0E0698079DD
:2012E000012830D000981E38417F007F0902014300980170090A41700098801C009001981F
:20130000801C80B2019010A8C18D00980170090A41700098801C09E00AE296E13BE1DFE040
:2013200004E29BE077E036E016E2AFE000900198801C80B201901BAA2A990298F5F75AF96F
:20134000002803D007E010A8818DD1E739880198081A0428BFDA0198012843D0E0698079D5
:20136000012804D010A8818D5548814206D110A8818D00980170090A417009E000981E3809
:20138000417F027F0802009910430870000A48700198801CBAE1072E01D0152E76D14178C3
:2013A000027808021043208320A98880249A51781278090211436183002801D0884201D9F1
:2013C00001203FE7012020720020E0802073052E0AD01D982299E269C0B2491DF1F783FCF9
:2013E000002801D00A202DE70020C04360841AA8019023A922980297039500910078002379
:201400008206920E20462A99FFF712FC0390208B20A988807BE1032EC0D1402220A98A8114
:201420004178027808021043208320A988802A991EAB1C9A02930192009139880022491E63
:201440008BB21B990978F5F747F918A90872002833D10B20287010A8008F3FE0052E9DD1BD
:20146000802220A98A8141780278080210432083249984464A78097812020A43628420A9E9
:2014800088801248824202D30720DBE6AFE03F208002024362842A981FAB1C990293019166
:2014A00000903888401E83B21B9801786046F5F713F918A9087200280CD08328AAD107E033
:2014C000FFFF0000AC13002001280000010200000220B8E00D20287010A8808F401C15E16B
:2014E00001990C22C9095143C91CB14204D9019840067CD5002009E142780378100218432D
:2015000020AA9080844622980078400609D505206A46107422980078C00905D00020107404
:201520001DE106206A46107424981F902A9A00900023701A029383B21E9001921B98002207
:2015400001786046F4F7E4FE18A90872002269460A74832801D1022003902298007840066B
:201560000DD52088C00506D520A9208B8988884201D100206062002018A90872C6E0FF211D
:20158000013120A88181808820831E9860841F9860621320B8E0052E29D34178027808025A
:2015A000104320A98880218F002902D0FE4A914206D10A216A4611740121C943218702E052
:2015C00007216A46117422992A9A491D0192009101221D990023D203029311438BB22499F1
:2015E0004A78097812020A431B99097800E0C9E0F4F78EFE18A90872002269460A74012265
:20160000520220A98A81832808D0002809D0218FE54881427ED10020208778E0888820835D
:201620004DE7606B002808D031462046229AFFF7E3FB18A90872002869D12B463A4630463A
:20164000229900F056FB039061E02298022E407801907DD1002801D0012879D108206946F6
:2016600008740198087521A800901B98002201782046019BFFF7B0FC6946002248758A7500
:20168000002802D10198012809D0208F002806D0002008740120800220A988810EE004A85C
:2016A0003399F1F7BCFF03900020694608740120800220A988810398022807D0BB48006861
:2016C0008079002805D018A908722BE0019820831DE00398002803D0812018A9087240E003
:2016E00021A800901B98012201782046019BFFF773FC18A9087220463499FFF753FC18A967
:20170000087A002803D119202870012038806846007C00E03CE0002804D004A83399F1F71F
:201720007EFF0390039800282ED01AE0062012E52078000713D5012E11D1092168460174DC
:20174000A188818204203499FAF757FF082100E005E020A88181CDE60198400612D50320D1
:20176000039020A9208889890843208020A988894005400E04D026992B9808602698868079
:201780000398AAE40420E6E418A8007A00280ED00120287022980078687020A88088A87047
:2017A000000AE87018A8007A28710520388020A92088898988432080E2E7FFB50746A1B00E
:2017C00000201C903A7801209040794A7C68104010AA1087744B22885B1C9A4203D000289B
:2017E00004D0100702D5012025B0F0BD249E0020307023980025028810A8028518A805751F
:201800006A4B68461972057404A8186020462C301B902A985860249E94463878721C052156
:20182000039201282DD0022808D003287DD13078800980011D303070B889A0803878022898
:2018400004D13078800980011B303070F01C1FAA01900292009110A8008D0022C01E83B211
:201860002020015DB889F4F737FF0028DED10398B9890170090A417010A9888FC01C088546
:2018800028E1787B18AA10753A7B012A02D0022ACCD1FCE022887F231B011A4010AB1A8790
:2018A000802A4AD006DC102A10D0202A0ED0402A0AD124E0FF3A013A65D0FF3A013A79D091
:2018C000FF3AFF3A022A76D00525A2E02078C00601D5082000E010201C9004206A46107408
:2018E000002090821AA81DAA1EAB03960192029000933B8A20461C9AFFF79AF984E0228B98
:201900003B8A9646934268D10A221C92002839D1039801906046401E1FAA83B2029220200A
:201920000091015D0022704600E0BAE0F4F7D4FE014618A801750B201AE0228B3B8A9646B9
:2019400093424AD10C221C92002862D10398019060461FAA401E0292009183B22020015D6F
:20196000628C7046F4F7B8FE014618A801750D20307010A8818F491C0185042168460174DD
:20198000218B818245E0238B3A8A9C469A4224D112221C9200283CD1606A002813D0002240
:2019A0006B4607C3638C07E0FEFF0000AC13002009F800000DE04BE02020015D6046F4F7B2
:2019C000A7FC18A9087513203070012010A908851FE0398A228B914201D00425B6E01621E3
:2019E0001C91002815D11B98818802682046FFF703FA18A9087500280BD11B9833460168D6
:201A000080881AAA00F075F9054602281BD0042D19D01B988088002811D06846007C00280C
:201A200004D004A82A99F1F7FAFD05460120694608741B981B990068059000208880002D34
:201A400048D0052D2ED06846007C032878D07DE018211C91002806D0388A20832046B96874
:201A6000FFF7A0FAD5E72046183000902020015D237E01222046FFF7AFFA18A9087500280F
:201A8000ECD119203070012010A90885E6E7208801214902084010A90887FF38FF3802283F
:201AA00006D0052510A92088098F884320804DE0208F9849884290D116201C90386900282F
:201AC00005D06063B88A20870020608702E00020C043208710A8008F7F21090102468A43CC
:201AE0000DD0782300220420B968FAF7DFFC3878A07010A92088098F0843208002E021880C
:201B0000814321806846007C002805D08248416804A8F1F784FD054618A8007D002815D01C
:201B20001C98707001203070208BB070000AF07018A8007D3071052110A8018506E0FFE70D
:201B40007548416804A8F1F76AFD05467248017A20884005400E22D11B98808800281ED0A5
:201B6000239A0026138810AA1385249A2A9B6F464CC71B9A039412681AABFFF78DFA0546F7
:201B800002280CD00120694608741B982A990068059004A8F1F743FD05461B98868010A8F0
:201BA000018D2398018028461EE600B597B0042807D102206A461070019100216846F1F74E
:201BC0002EFD17B000BD10B5534C037800222168012B02D0022B42D126E00B78002B01D009
:201BE000042B03D10A71226803211170216883880A79D200921D8B5221680A79D2000832AB
:201C00008918C2880A80216803890A79D2000A328B52428920680179C9000C3142522168DC
:201C20000879401C08711EE00A7482888A802168C288CA80226801891181226841895181D5
:201C4000C1682068C1606168F1F7E9FC0146022807D02068007C002802D1002903D0812038
:201C600010BD832010BD002010BD406B002800D0012070478178012909D100880521C90249
:201C8000884202D0491C884201D10020704705207047F7B586B00024684615460F4684818B
:201CA00005261AE0049841780278090211432980811D019602940091417902790B02134334
:201CC000C178827809020A4341780078090208433946F4F71DFB002806D104AA03A9069879
:201CE000FFF7BFF80028DDD0822800D1002009B0F0BD10B51488844201D2052010BD17243A
:201D00001C701080421E581C491C09F09AF8002010BD0000FEFF0000AC13002030B50346EC
:201D2000002002460DE09C5C2546303D0A2D02D30020C04330BD0A25684330382018521C7A
:201D4000D2B28A42EFD330BD70B50D46144608E00A2109F0DFF82A193031203A641ED17707
:201D6000E4B2002CF4D170BD10B5002310E0040A00020443A0B2CC5C44402006000F6040AD
:201D80000407240C44402006C00C60405B1C9BB29342ECD310BD000010B572B600F0DCF81C
:201DA00000280BD0EFF77CFAFAF7E1FD08F097FB6E490020C86288626D49086062B600202A
:201DC00010BDF3B5002501200007C06A81B0C0430006000E04D167480068401C00D1012590
:201DE00072B600F0B9F8002802D062B60820FEBDEFF7ACF9EFF758FA5F4B604E00211A6867
:201E0000CA40D2071FD00246CA40D20718D14AB2002A07DA1407240F083CA408A400A41936
:201E2000E46904E09408564FA400E41924689207D20ED4402206920F012A04D0032A02D0AF
:201E400062B65048FEBD491C2029D8D30198030009F0A2FA142123232323232323230B0D28
:201E60000F11131F1517191B1D2E002416E0012414E0022412E0032410E004240EE00824C1
:201E80000CE009240AE00A2408E00B2406E00C2404E0052402E0072400E00624F069012145
:201EA0000002000AC9070843F061002D04D009E062B601200003FEBD2C4D3348E862EFF7A5
:201EC000F3F9A8622A4931480860314902980860EFF7EAF9214608F0E9FAFAF70CFD08F03F
:201EE000EFFC08F065FB0198EFF7A8F9040062B603D0FFF751FF2046FEBD0020FEBD10B589
:201F0000044600F029F8002800D001202070002010BD204908600020704710B50C461028D9
:201F200008D011280BD012280CD013280ED00120086010BD03CC083CFFF743FF0AE0FFF705
:201F40002BFF07E02068FFF7DAFF03E01149206808600020206010BD05480C4900688842AB
:201F600001D10120704700207047000000050040640000200010001000E100E000ED00E069
:201F800000E400E00110000000220000BEBAFECA980000200400002010B520380C460300BC
:201FA00009F0FAF933A6AAAEB2B8BCC0C5E0DBE41B1F23272C31373C41474D5054585C60D9
:201FC0006D71656974787C8084888C9094989C9FA2CACFE9F0F3D3D7F800206800F0DDF8E8
:201FE000D6E0206800F0E1F8D2E0206800F0F5F8CEE0207840B208F0C9F8C9E0207840B29F
:2020000008F0E7F8C4E02078616840B208F0FAF8BEE0207840B208F00AF9B9E0207840B2C2
:2020200008F015F9B4E02078217940B208F020F9AEE02078616840B208F04AF9A8E008F035
:2020400056F9A5E0206808F05AF9A1E0207808F06FF99DE02068FAF738F899E02068FAF748
:2020600038F895E021792068FAF73AF890E0206807F0D8FF8CE0206807F0D9FF88E02078ED
:2020800007F0D9FF84E007F0E3FF81E0207807F0E5FF7DE0207807F0F7FF79E0206808F0A5
:2020A00010F875E0206808F012F871E0206808F014F86DE0206808F015F869E0206808F0B9
:2020C00017F865E0206808F019F861E0206808F01AF85DE00846EFF751F859E0F0F787F9EE
:2020E00056E0F0F7B4F953E02068F0F7BCF94FE0206800F0E1F84BE0206800F0E9F847E094
:20210000206800F0F0F843E02078A268616800F0F5F83DE0207800F006F939E0207800F0AF
:2021200017F935E02078616800F027F930E02078616800F03AF92BE02179207808F008FA3E
:2021400026E0206800F06BF822E02068FAF7FEFA1EE02068FAF7E2FA1AE007CC0C3C08F0CB
:20216000F1FA15E0206808F044FB11E003CC083C08F06FFB0CE0206808F065FD08E009E0BB
:2021800003E0FFE708F077FD02E0206808F0AEFD206010BD0120086010BD0021017008467A
:2021A00070470146002008707047EFF31081C907C90F72B60278012A01D0012200E00022F4
:2021C00001230370002900D162B6002A01D000207047012040037047E7E7EFF31081C90758
:2021E000C90F72B600220270002900D162B600207047F2E710B52848FFF7CFFF002803D095
:2022000026A11D2008F0A7FF2348401CFFF7C5FF002803D021A1212008F09DFF10BDF1B596
:20222000224D6F6801261C48FFF7BFFF1A4C002803D10026601CFFF7D0FF1D4A1D49012062
:20224000506000BF00BF00BF00BF00BF00230B604B60009B6B60106000BF00BF00BF00BF08
:2022600000BF0868002802D148680028F9D048680028E4D1002E04D06F60601CFFF795FF2F
:2022800007E0601CFFF791FF0028D3D10248FFF7A4FF0020F8BDC2E79C0000207372635CC8
:2022A000736F635F6563622E6300000000E5004000E0004000E100405A495B4B0A685B49FA
:2022C0009A42096801D18904890C0160002070475449554B0A6855499A4201D18004800C7A
:2022E0004860002070474F494F4B0A684F499A4201D18004800C88600020704730B5494B2D
:20230000494D1C684A4BAC4202D0102802D203E00E2801D3184630BDC30044481818016129
:202320004261002030BD3F493F4B0A684049491C9A4202D0042802D203E0022801D308469E
:2023400070473C4A0121C00080180160002070473449354B0A683649491C9A4202D0042861
:2023600002D203E0022801D308467047314A0121C000801841600020704770B5294A2C4B27
:2023800014682D4E284D82005B1C9219AC4203D0042803D2116006E0022801D3184670BD8B
:2023A0008804800C1060002070BD70B51D4A204B1468214E1C4D82005B1C9219AC4203D098
:2023C000042803D2106806E0022801D3184670BD10688004800C0860002070BD10B5134AB6
:2023E000164890600E200021C3009B1819615961401C1028F8D300200F4A05E0022803D3D9
:2024000083009B18196005E083009B181C68A404A40C1C60401C0428F0D310BD03490748E7
:202420008860704764000020BEBAFECA00F501400820000000F0014000F8014000C0FFFFB3
:20244000FE48C07E7047FE4840687047FD48C07E7047FFB5F94E85B0706A34680568606887
:202460000190306A0390298D0798401A80B202900898002804D0274638372046483002E0F3
:20248000371D2846A030009003203871059800281FD001287ED0022863D003287BD0EAA1C5
:2024A000ED4808F058FE0898002806D03879032803D0E5A1E94808F04EFEA16A7069FAF77C
:2024C000B0FDB860216A606A814265D90099086034E1306A002803D1DBA1E14808F03BFE5F
:2024E000288BE0494843421806980021002804D05043DD4908F00EFD411CA1610191AA8881
:20250000D848002142430698002804D05043D64908F000FD411CE161306AD24A801CA062C1
:20252000298BD04B5143019A891AD04A89180918A162AA7D01985A4340008018FF3019306E
:2025400020626062306A081AC949FF3815388842A9D2C84988427DD2BBA1C74808F0FBFD1B
:202560008BE0288BBF4AE16850430A1806980021002804D05043BC4908F0CCFC411CA161C4
:20258000AA88B848002142430698002808D05043B54902E03EE073E0CEE008F0BBFC411C27
:2025A000E161306A002803D1A7A1B44808F0D3FDA620405BAB4A0028288BE16821D0504339
:2025C0000818A169401AA0622169A068A54A4843A1694018A97D400051434018FF3017303F
:2025E0002062A888E1695043411AA54808186062A06A316A401A9E49FF38553888423CD39F
:2026000051E750430818A169401A3168D63849684018D8E7284680300190C08C002802D007
:20262000306A002803D188A1964808F094FDA8888C49E3694843C01AA06201999C46CA8CEA
:202640002169A368521A4B43A169591863465343C91800E011E0AA7D824B49005A43891804
:20266000FF3117312162864941186162316A401A7F49FF3855388842C2D20120387112E7D2
:202680000898002803D03420005D00287ED1A88874494843E169401A02994843A0622846C5
:2026A00080300490C08C0028019825D0002803D065A1754808F04FFD04986A4AC18C02989B
:2026C0000818E16948434000FF3017302062A8885043411A6A48081860626C484068002897
:2026E00019D0A26A03990120511A614AFF395539914285D23871D6E6002802D00398002800
:2027000003D151A1624808F026FD0198A16AD6380818A062D0E7FAF7F2F97269014610464F
:20272000FBF706FCA16A081A5149FF3850388842A5D2012009B0F0BD009801600098554928
:2027400000684018F86028468030028A0799511A09B2002904DD0599022901D0032100E049
:20276000002179710E99002915D0028F002A1ED0418F4187A0352B7F491C4B4393420AD235
:202780007979491E002906DD012100E00CE07971418F491C4187089838700898002808D017
:2027A0003420005D002804D0022009B0F0BD0021DFE708980121484020346075307FF27E6B
:2027C0003946B37E9A4202D0FAF710FE04E00020F076B07630607062002009B0F0BDF0B57F
:2027E0002A4F83B038680568416A2E460C682036717D00290AD0698E228D914206D1407A3C
:20280000002803D110A1244808F0A5FCFAF777F91E4F39684A6901461046FBF789FB3F682A
:202820000028796A096807D089880E4A51433A68D269891A08F06EFB698E2FE0B813002076
:20284000B8000020E01300207372635C6C6C5F6C6D2E73302E630000310500003A05000002
:20286000B7040000E204000040420F00330400005C0800001D030000D4040000DC040000B3
:2028800094FBFFFFF50400001B050000A800002014050000FF0B000021060000228D1318A6
:2028A000994202DB491C698602E0401C10186886B07D002806D19421688E095B884201D1E1
:2028C000401C6886388BFB4E401C3883204640300190C1888088081A218D401E401887B214
:2028E000C03418E03068F449406A002300794000085A009323795B00C95A081881B2287D8A
:202900000023FFF7A6FD00280FD001280FD0EB49EB4808F020FC6A8EB81A00B20028E1DA12
:2029200001980821817005F0BDFF03B0F0BD688E401C6886EFE770B5DE4D09292B686A68D6
:202940007BD20C007C4424792419A7440463869683A5A575A20000201062D17E042956D2FC
:202960000B007B441B79DB189F4451510147516A0C68116808701168486010682030407D73
:20298000002808D1FAF7BBF869680968096CFBF7CFFA002817DC6868228D0168498E914273
:2029A00005D123468033998A8A1ADA8204E0891A962211530168498E21850268C168116471
:2029C000C168416111E068680168098E228D8B1A22468032D3820168098E218501680B6C22
:2029E000C3600B6C4361886C1062204606F0C8FB002821D0B3A1B74829E0D068506105F0C1
:202A000088FA002818D0EF20AEA180001FE0ADA1B1481CE0D07E042817D201007944097961
:202A200049188F441212010B06F0E6FC002803D0A4A1AA4808F08FFB70BD2DE005F09FFBDD
:202A40000028F9D09FA1A64801E09EA1A54808F082FB70BDFDF7CBFD70BDD87E022806D069
:202A6000D87E032806D0FF2096A1AB300EE0FFF7B6FE70BD00F013FC70BDD87E0228F6D097
:202A8000D87E0328F6D0FF208EA1B83008F063FBF0E7FAF719F870BDFF208AA1C630D6E760
:202AA000F3B50126834C904D81B00F46092945D208007844007900188744042D38382D409E
:202AC000403838000121884800F0D0FB39460198FFF731FFE87E022826D160680468406AF6
:202AE0000768F9F7EAFFB988804A5143E269891AD639E162B72803D283200001081A02E053
:202B0000081A7B494018E0627A48E16A814200D80846E06205E00198FFF70DFFE87E0228ED
:202B200002D128682030067503B0F0BD25600198FFF701FF0020206003B0F0BDFF2061A1D2
:202B4000623008F008FB03B0F0BD70B506460C4609291FD208007844007900188744040D71
:202B600011110D1A1A1111000121634800F07EFB21463046FFF7DFFE70BD3046FFF7DBFE78
:202B800070BD4C4D5C4828603046FFF7D4FE0020286070BDFF204BA1883008F0DCFA70BD72
:202BA000F0B5514985B0CA7E0026424C032A03D02831CA7E032A64D100252160002824D0E0
:202BC00001280ED03FA14D4808F0C5FA2068002E05604562256054D049484560002005B04C
:202BE000F0BD0320887600E020BF2068C17E002903D0C17E827E9142F6D0C17E002902D073
:202C000000268576E2E70126FBE70026032708468F76C97E032903D0C07E00282DD02DE068
:202C2000007F002803D127A1364808F094FA2068067F684607714771F9F761FF0290FF2061
:202C4000F530039001216846017069463046FAF7CDFB2068007FFBF7F7F900280BD0206829
:202C6000007FF9F731FF20680577C576857605600126456202E020BFEBE70126206885760B
:202C8000A4E70C2005B0F0BD10B5174800F04DFB194800F04AFB1C4900200875184948700E
:202CA00011494861144A50618876907601494860086010BDA800002034B4010048280100B5
:202CC0005B0600007372635C6C6C5F6C6D2E73302E630000B6030000C3030000D603000025
:202CE000DB030000E2030000B8130020E204000087F8FFFFEC060000E01300201E0300009D
:202D0000B80000207E02000008140020F8B5FF4E05463068002401270004810FFC480068B6
:202D2000800F814204D0FF20FA49D03008F013FA3068F94E0004810F30680006800F8142A3
:202D400004D0FF20F349D13008F005FAF348C0693168800F0904890F884204D0FF20ED4928
:202D6000D23008F0F8F9EE480570EE4DEC76AC76ED4EF476B476ED48077104606C6274627A
:202D80002C60EB4F346028467C6000F0CEFA304600F0CBFAE74804757C706C617461AC7654
:202DA000B476E54844600460F8BDE04908717047F8B5DC490546CA7EDB48DF4C002A02D1F6
:202DC000C27E002A03D0C97E022907D009E0DB482160F9F725FE216808770AE0C17E002973
:202DE00001D00C20F8BD2060D548F9F719FE21680877CF48456021680860D2484862284696
:202E00000121BC30F9F790F9A035287F8007800F401C28772068007F002803D1BD49CA4883
:202E200008F099F9F9F749FEC849884200D20846C749401886B221680320C87604F084FFD5
:202E40002168086104F0A8FF01270025002826D004F0A2FF21684A6A10600868012107702F
:202E60006846F9F7EAF868460078BA49000208F051F80F46F9F743FEF119FAF7D2F8216892
:202E8000C86022680320107250721571107FD37E111D967EB3420ED0FAF7A8FA0FE0F9F72C
:202EA0002EFE3146FAF7BDF82168C8600868057008684770E5E7D576957615605562206836
:202EC000058300202560F8BD7047F8B5954EF17E002903D19449C97E002901D00C20F8BD5E
:202EE0000221F176914F934D77623560002438602C7500943979C0304A00974900798A5A00
:202F00004000085A2346101881B222462046FFF7A0FA002803D07F49904808F01CF92C61B8
:202F20000120AC6028756C862C868D4884753968088D401E088534830020F8BD10B57E481D
:202F400001244068817E03290CD001684978002906D0006A8349884202D9002405F03CF94B
:202F6000204610BD0024FBE77348406802681178491C1170016A0068C26A914204D8007DB1
:202F8000012801D0012070470020704700207047F8B5694D63482860416A00270C6800686D
:202FA000342126460F548036B17F002927D1007D032824D1F9F7A3FD29684A6901461046D8
:202FC000FAF7B6FF00281ADD2D68674B6A6A2968126892880091C9695A43511A07F09AFF91
:202FE000218D401C4218009953480A862968B28A0B8ED21A12B2002A03DC0760F8BD2F60DF
:20300000F8BD012220318A7521464031CA888988514F511A228D491E89188EB20546C0340C
:2030200019E0496A09794900795A00220092028E2379007D5B00FB5A591889B20123FFF773
:2030400008FA00280ED001280FD002280AD03149464808F080F829680868028EB21A12B2C3
:20306000002ADEDA00202860F8BD28680068018E491C0186EFE770B52F4900244D68062824
:2030800076D202007A441279921897441820020E240D002000F08FF9EC76AC762C600021D6
:2030A00008466C6200F0E2F870BD1D480D680078EFF72AF9EC76AC762C606C6270BD012076
:2030C00000F079F90021084600F0D0F870BD29680320087570BD686A29680068CA698A60F4
:2030E0008188214A51432A68D1600146C0310A8A02838A7B82754A8A82808A8AC280C98A39
:20310000018129680220087570BD31E000E400E008E400E0C42C010018E400E000ED00E095
:20312000A0000020B8130020E0130020B0000020B800002008140020A8000020A12A010059
:203140004B2B0100A4000020C9020000F6050000BB0200001027000034B40100520300003C
:2031600028140020D9821300E204000007060000DD49DE4807F0EFFF70BD70B500280BD00C
:203180000024DB4D01280ED002282FD0EF20D649C00007F0E0FF70BD00F06BF900210846FF
:2031A00000F064F870BD686801684C70C47684760460D04E446201220021706800F063FFD7
:2031C00071680846C0318C72CC72FFF77EFE002803D0C549C84807F0BEFFF9F7DBFBC74887
:2031E0006C600078EFF790F86C6070BD00F041F96868C4768476046000214462084600F08D
:2032000035F870BDBA494968CA7E022A08D10A681378002B04D150600968CA6A1018C862AF
:20322000704710B5B24A002952680BD0012906D0022906D0AC49B24807F08DFF10BD801E7A
:2032400000E0401F106210BD08B50020C04369460880AC48C07E002801D0002008BD08467B
:2032600000F0F6F90028F9D0012008BD70B5A04C05466268002908D0002A04D0FF209A4971
:203280000D3007F068FF656070BD002A04D1FF209549133007F05FFF0020606070BD38B513
:2032A000934C20680168497801291FD001216846F8F7C3FE684600789349000207F02AFEC1
:2032C0002068426AC06812685118F9F7AAFE2168C8608C4822680321824202D0108B0A2881
:2032E00010D2108B401C108351720DE07D21C068C900F9F796FE2168C86004F025FD21684F
:203300000861E6E702205072117200231371107FD47E111D957EAC4202D0FAF767F838BD42
:20332000D37693761360536238BDF8B5704C05461F27EE7E042E2DD230007844007900180A
:203340008744312801237148854203D06649704807F001FF02202560A87600E020BF216867
:20336000C87E002803D0CA7E887E8242F6D0CA7E002A04D000228A760C27226010E0002205
:203380008A760A604A6222600DE00120FFF708FC074603E054495F4807F0DDFE002F02D046
:2033A000E87EB042C5D1E87E002803D04E495A4807F0D1FEF8BDF8B54D4D01286A68516A0D
:2033C0000C6846D10879554940000B5A1068077D0126032F06D0027D022A13D0007D01283F
:2033E00024D036E0002707611068876094200096025BC420005D4000085AC01881B23B46BF
:2034000003201EE022468032D78C07610096C420005D928A4000085AC01881B200230220C1
:20342000FFF717F8696809680E750CE094200096025BC420005D4000085AC01881B200231E
:203440000120FFF706F8002803D02749344807F082FEF9F79FFA29480078EEF755FF69687D
:20346000002008830B68228D5A86096820318875F8BDF8B51E4D002168680C4600684278AE
:20348000002A01D0447027E00078002809D001216846F8F7F7FD684600781B49000207F0C7
:2034A00039FD6868426AC06812685118F9F7B9FD6A68D060147103205072107FD37E111D2F
:2034C000967EB34202D0F9F791FF03E0D47694761460546268680483F9F75CFA07480078CC
:2034E000EEF712FFF8BD0000C42C010056070000A8000020B800002003070000A000002069
:203500009D070000E013002010270000B813002007020000130200001902000034B40100B0
:20352000BC060000F8B50024E948FEF73EFE002825D1E84FC02026464643F51901462846A9
:2035400007F0DEFC0120B8556C80E34900200870E24A4A8080356962E149641C0870A96219
:20356000E049E4B208704A80A963032CE2D3D848FEF733FED648FEF718FE002801D00C20C6
:20358000F8BDFF211931D84807F0BAFCD648012101704480D5490020087208750877D449F9
:2035A0008872CB48FEF719FE0020F8BD10B5C848FEF7F3FD002803D0CEA1282007F0CBFDF2
:2035C000C348FEF7EAFD002803D0CAA12D2007F0C2FDFFF7A7FF002803D0C6A1332007F053
:2035E000BAFD10BD10B50446B948FEF7DEFD002801D00C2010BDBC490878002807D00020D1
:203600000870B3482160FEF7E8FD002010BDB048FEF7E3FD1F2010BD70B505460C46AC4860
:20362000FEF7C3FD002801D00C2070BDAE4A5088A84202D11078002804D0A548FEF7CDFDC6
:20364000122070BDA2482260FEF7C7FD002070BD10B504469E48FEF7A8FD002801D00C20E5
:2036600010BDA1480178002907D00020C04320809748FEF7B2FD122010BD40882080944892
:20368000FEF7ABFD002010BD10B504469048FEF78CFD002801D00C2010BD2078002804D0B5
:2036A0008B48FEF79AFD0C2010BD012020708848FEF793FD002010BD10B504468448FEF7EF
:2036C00074FD002801D00C2010BD824A0021C0204843105C00280AD0C0230020594350547E
:2036E000881820607A48FEF778FD002010BD491CC9B20329EBD37648FEF76FFD1F2010BD9C
:20370000032805D2C0225043724A135C002B01D012207047801808600020704710B5002264
:203720000C46032809D2C02148436A490B5C002B14D122704018606018E003280ED1644843
:20374000FEF733FD002809D167484188032902D10178002904D05E48FEF73FFD122010BD7F
:2037600060605B48FEF739FD01202070002010BD10B504465648FEF718FD002801D00C2041
:2037800010BD2088534A032804D2C0214843105C002801D00020208000202188491C89B21C
:2037A0002180032900D300212180C0235943515C00290BD0401CC0B20328EED30020C0439A
:2037C00020804348FEF709FD122010BD4048FEF704FD002010BD70B505460E463C48FEF71C
:2037E000E4FC002801D00C2070BD2888341D032804D303D0A04201D3002028800020361DD0
:203800001DD0394B33492A88521C92B22A80A24200D300222A80042A02D3A24217D301E078
:20382000032A05D0C02672438A5C002A0FD002E01A78002A0BD0401CC0B2A042E3D30020FD
:20384000C04328802248FEF7C8FC122070BD2048FEF7C3FC002070BD10B504461C48FEF76A
:20386000A4FC002801D00C2010BD2078002804D01748FEF7B2FC0C2010BD0120207014481A
:20388000FEF7ABFC002010BD10B504461048FEF78CFC002801D00C2010BD217801200029E6
:2038A00002D0012905D008E061680A78002A09D003E061680A78002A04D00548FEF78DFC0A
:2038C0000C2010BD08700248FEF787FC002010BDC00000205814002098160020FFFF000090
:2038E000C1000020C6160020D8160020B8170020D81700207372635C6C6C5F64622E6300AD
:2039000010B5282107F0FAFA10BD70B5054600780A0700090001120F1043287007290ED2C2
:20392000080078440079001887440305030503070300062408E00C2406E0222404E00024D4
:20394000F8A1572007F007FC6878800980012043687070BD00780007000F704710B5C01C25
:2039600007F0F5FC10BD0A4610B5C11C104607F0EEFC10BD10B5093007F0E9FC10BD02787B
:20398000BF23C9071A40490E0A430270704700784006C00F704702785206520EC9010A43C1
:2039A0000270704770B50C460546C11C2046093007F0CDFC20784006400E20702978490634
:2039C000C90FC9010843207070BD70B515460E4604461F2A03D9D3A1A82007F0BCFB2046AA
:2039E0002A463146093007F02CFA6078AD1D80098001A906890E0843607070BD70B50546E0
:203A000040780E468406A40E062C03D2C5A1B82007F0A1FBA41FE4B21F2C00D91F24294657
:203A200022460931304607F00CFA204670BD70B515460E4604461F2A03D9BAA1CC2007F05D
:203A40008AFB20462A463146093007F0FAF96078AD1D80098001A906890E0843607070BD37
:203A600070B5044640780E468506AD0E062D03D2ACA1DD2007F06FFBAD1FEDB21F2D03D93F
:203A8000A8A1E12007F067FB21462A460931304607F0D7F9284670BD0A78C2734A780274AB
:203AA0008A784274C978817470470A78C2744A7802758978417570474176090A817670478A
:203AC000C176090A017770474177090A81777047C175090A01767047817570472030027904
:203AE000C90652095201C90E0A430271704720300279D206D20E49010A430271704710B5F2
:203B00001F3007F019FC10BD417800788906890E0007000F06D0012808D0022809D0062808
:203B200010D10AE0891F1F290AD90BE00C2907D008E0891F1F2903D904E0891F1F2901D88F
:203B400001207047002070474178007889060007890E000F042805D1062903D3252901D81B
:203B6000012070470020704770B401780907090F03292ED0052931D1411C827E0C46437E07
:203B800011021943037FC27D1D02037EC67E1B021343827D407835438006800E22281DD123
:203BA00006291BD31920C001814217D8FF26F436B54213D8002A11D0082A0FD88A420DD23C
:203BC0008B420BD8617F227F09021143814208D904E040788006800E0C2802D070BC0020AF
:203BE000704770BC0120704710B5222107F086F910BD10B502788B07920892009B0F1A43BB
:203C000002704278520952014270012908D0022906D0032905D0FF2042A1E83007F09BFA6E
:203C200010BD01210A43427010BD10B502788B07920892009B0F1A430270427852095201EB
:203C40004270012907D0022905D0032904D035A1384807F080FA10BD01210A43427010BD2F
:203C600000788007800F70470278EF23C9071A40C90E0A43027070474178C078C906C90E65
:203C80000E2835D202007A4412799218974406090C0F1215181B1E2124272A2D0C2929D084
:203CA0002AE0082926D027E0022923D024E0172920D021E00D291DD01EE001291AD01BE049
:203CC000012917D018E0022914D015E0092911D012E009290ED00FE001290BD00CE00129B8
:203CE00008D009E0062905D006E0022902D003E01B2901D8012070470020704770B50546FD
:203D0000C1700E2926D20800784400790018874406131517191B1B151D1D1B1B1F150C24A6
:203D20001DE000007372635C756C5F7064752E630000000001020000082410E002240EE095
:203D400017240CE00D240AE0012408E0092406E0062404E000249A499A4807F0FCF968783E
:203D6000400940012043687070BDC0787047C171090A01727047017AC27908021043704729
:203D80004172090A81727047817A427A080210437047C172090A01737047017BC27A0802B5
:203DA000104370474171090A817170478179427908021043704701717047007970474173B5
:203DC000090A81737047817B427B08021043704770B4017AC37909021943431C857A1C4656
:203DE000467A2B023343657926792C023443C21C754E00798D1FB54215D8FF25F435AB425A
:203E000011D800280FD008280DD888420BD28C4209D8507A117A00020843B11D884202D833
:203E200070BC0120704770BC0020704710B5001D07F082FA10BD0A4610B5011D104607F0D9
:203E40007BFA10BD4172090A81727047817A427A080210437047017170470079704710B5C7
:203E6000001D07F081FA10BD0A4610B5011D104607F07AFA10BD0A78027349784173704702
:203E8000027B0A70407B4870704710B50E3007F06BFA10BD0A46014610B50E31104607F0ED
:203EA00063FA10BD0A7882754A78C2758A780276C97841767047827D0A70C27D4A70027E4B
:203EC0008A70407EC870704710B5001D07F04CFA10BD0A4610B5011D104607F045FA10BDC3
:203EE0000A7802734A7842738A788273C978C1737047027B0A70427B4A70827B8A70C07B91
:203F0000C8707047017170474171090A81717047C171090A017270470079704781794279C7
:203F2000080210437047017AC27908021043704701717047007970470171704710B5001D3F
:203F400007F012FA10BD0A4610B5011D104607F00BFA10BD10B5001D07F006FA10BD0A4649
:203F600010B5011D104607F0FFF910BD70B515460E4604461B2A03D91149144807F0EBF87D
:203F80002A463146E01C06F05CFF6078E90640094001C90E0843607070BD70B50546407855
:203FA0000E46C406E40E1B2C03D90549084807F0D2F82246E91C304606F043FF204670BDC1
:203FC000243D0100A10200007A0C0000F1030000FD03000070B504460020A083208C1E46A0
:203FE00048431546114606F0A3FF2084F000294606F090FF401C80B2014619226943920214
:20400000E083914201DD401EE0837D202946000206F080FF401CA08470BD70B50A7BD20619
:20402000D20E0A73002282758B181B7ADC075B08DD07E40FED0F2C195B08DD07ED0F2C19EC
:204040005B08DD07ED0F2C195B08DD07ED0F2D195C08E307DB0F5B196508EC07E40FE41854
:204060006B081B1984186374847D521CE318D2B28375052AD8D3D8B2252803D9E1A18A2087
:2040800007F069F870BD70B504460B4625462646214600202835C0368031032B0AD0002B46
:2040A0003AD0012B41D0022B03D1A11C2846FFF7B4FF70BD2880A871E871E87228736873CD
:2040C000A873A870E870287168716876A8832B4668842033987128859872E8752876E87314
:2040E0002874D872187398731A752884FF226035AA709875088248828882C882088348832E
:204100004877C884A4221055088748872421085560843070B07170BDC8848877A188238977
:204120000A462846FFF756FFBFE7C884F38A728AA1882846FFF74EFF70BD70B5044603464C
:2041400028348033054603290AD0002933D0012938D0022903D1A91C2046FFF75EFF70BDF7
:2041600000202080A071E071E07220736073A073A070E070207160716076A083214660844C
:204180002031887120858872E0752076E0732074C872087388730A752084FF226034A270CA
:2041A00088751883987618742421586148551877A035287370BDA9882B890A462046FFF775
:2041C00009FFC8E7586AA988C38942892046FFF701FF70BD70B5867D0D460446002E01D0D1
:2041E000252E01D9122070BD002A18D0287EE17D50430818252106F08DFEE1750846CA082D
:204200004907490F834BAA18595C127A914308D0314606F07FFE491CCAB200200AE0002084
:2042200070BD2076002070BD002803D02118097C511ACAB22118497C91423AD32918097A2C
:20424000C943CB07DB17D21A521E1206120E35D08B07DB17D21A521E1206120E32D04B0789
:20426000DB17D21A521E1206120E30D00B07DB17D21A521E1206120E2ED0CB06DB17D21A73
:20428000521E1206120E2CD08B06DB17D21A521E1206120E2AD04B06DB17D21A521E1206B2
:2042A000120E28D00906C917511A491E0A06120E26D0401C0528B7DB1F2070BDC000207622
:2042C000002070BDC000401C2076002070BDC000801C2076002070BDC000C01C2076002001
:2042E00070BDC000001D2076002070BDC000401D2076002070BDC000801D2076002070BD91
:20430000C000C01D2076002070BD70B50D460446072904D9FF203BA15D3006F01CFFE0785D
:20432000502108406907490F88300843E070A078A72108401830A07060785E21084020303A
:2043400060702078BC2108404030207070BD0179490901D000207047002230B41146445C32
:20436000491CE3076408E507DB0FED0FEB186408E507ED0FEB186408E507ED0FEB18640893
:20438000E507ED0FEB186408E507ED0FEB186408E507ED0FA407EB18E40FE318D218D2B27D
:2043A0000529DCDB002A02D030BC0120704730BC0020704738B505460C466846FCF74EF824
:2043C00000281ED06946002008562072092161560022411A00D549422035EB788B420FDCDA
:2043E000FF2B0DD0A17A491CC9B2A1722B79994202D8617A7F2903D160720020A0720122D1
:20440000104638BD7372635C6C6C5F7574696C2E6300000044B40100F8B50024F74EFF20F9
:20442000B470F0702546F64F06E0042D04D3FF20F4A1AB3006F08FFEFF212846A03148435E
:20444000FF213331C0194A1C0C540146FF31145421310C754C75F178A94202D1B470FF215B
:20446000F170FF219D314A1C6D1C0C54EDB21454042DDAD30020FF21A0314143C919FF3112
:2044800081318C77401CC0B20428F4D3E048FFF7ABFB0021DE48FFF7E7FB0121DC48FFF787
:2044A000A8FBDC49FF20087048708870C87008714871F8BDB0E71B20704710B4D04A002146
:2044C000FF23A0334B439B18FF3381339B7F002B04D0491CC9B20429F2D30DE004290BD2DE
:2044E000FF23A0334B439A180124FF32813294770170204610BC704710BC0020704730B492
:204500000025042825D2FF220146A0325143BC4A89180B46FF3381339A7F002A19D0FF2458
:204520003334621C655455541A46603A15755575B24AD478844202D19570FF20D070FF2082
:204540009D304554FF319E310D709D7730BC0120704730BC0020704704280ED2FF2201466A
:20456000A0325143A64A8918FF318131897F002903D0A8494871012070470020704710B441
:20458000A449FF224979A03251439D4A82B089180A46FF322132937C6C462370D27C227122
:2045A000237822795A40802A0AD0227822235206520E5A435118016002B010BC0120704753
:2045C00002B010BC002070479248FF214079A03148438B4981B041180846FF303330FF3109
:2045E0002131CA7C69460A70037809220978594080290ED0037869460B7009784906490EE7
:20460000491C914208D26A461178491CC9B2117009E0002001B0704769460978090601D568
:20462000002100E080210170012001B0704704280ED2FF220146A0325143714A8918FF3178
:204640008131897F002903D072490871012070470020704710B46F49FF220979A03251433C
:20466000674A82B089180A46FF322132947C6B461C71D27C1A701C781A7994420AD01A7853
:2046800022235206520E5A435118016002B010BC0120704702B010BC0020704738B55D4879
:2046A0000179FF20A0304143554808180146FF3121318A7C6C4622700922FF303430037804
:2046C0002478A34223D004786B461C701B785B065B0E5B1C934205D26B461A78521CD2B2F8
:2046E0001A7006E06A461278120601D5002200E080220270087D401C0875087D497D884299
:2047000003D140A1444806F026FD012038BD002038BD4048FF210079A031484338494018BE
:20472000FF302130C17C807C814201D101207047002070473748FF210079A031484330498F
:204740004018FF302130817CC27C092013464B40802B0AD049065206490E520E914201D3AF
:20476000881A01E0511A401AC0B27047092070470022042813D2FF23A0335843204BC018E2
:20478000FF239F331B5C002B09D0FF300A702130027D437DD31A0B7042750120704700205A
:2047A0007047042811D2FF22A0325043144A8018FF229F32125C002A07D0FF302130027D57
:2047C000407D101A0870012070470020704710490160704704280ED2FF220146A032514380
:2047E000074A8918FF318131897F002903D009490870012070470020704700001018002020
:20480000141800207372635C646D5F712E630000901E0020C70000205A020000AC49CA782E
:20482000FF2A03D000210160084670478A78A949012A02D001600120704700207047A64806
:204840000178012907D001210170A4480178A048C170012070470020704704280ED2FF22F1
:204860000146A03251439E4A8918FF318131897F002903D0994948700120704700207047D3
:204880009349964BCA785B789A4206D18A782039002A02D0016001207047002070478C4858
:2048A0008E4AC1785278914209D1FF21C170801C0178002903D00021017001207047002084
:2048C00070478348854AC1785278914204D18078002801D0002070470120704704280ED230
:2048E000FF220146A03251437D4A8918FF318131897F002903D07949C870012070470020AA
:20490000704710B47549FF22C978A0325143744A82B089180A46FF328132147F6B461C7001
:20492000527F1A711C781A79FF3162403731802A0AD01A7822235206520E5A435118016040
:2049400002B010BC0120704702B010BC002070476248FF21C078A0314843614981B041181A
:204960000846FF309D30FF3181314A7F69460A70037803220978594080290ED003786946AE
:204980000B7009784906490E491C914208D26A461178491CC9B2117009E0002001B0704758
:2049A00069460978090601D5002100E080210170012001B070474948FF21C078A031484301
:2049C00047494018FF308130417F007F814201D1012070470020704704280ED2FF22014618
:2049E000A03251433E4A8918FF318131897F002903D03A498870012070470020704710B454
:204A00003649FF228978A0325143354A82B089180A46FF328132147F6B461C71527F1A70DD
:204A20001A781B79FF3137319A420BD06A46127822235206520E5A435118016002B010BCE5
:204A40000120704702B010BC002070472348FF218078A0314843224981B04018FF219D3168
:204A6000095C6B4619700321FF309E3002781B789A4219D003786A46137012785206520EB4
:204A8000521C8A4205D26A461178491CC9B2117006E069460978090601D5002100E08021CE
:204AA0000170012001B07047002001B070470B48FF218078A031484309494018FF30813023
:204AC000417F007F814201D1012070470020704710180020F017002012180020C7000020B3
:204AE00014180020F8B5FD4F0A46044600207978FB4D0646002902D0012909D00FE0F94903
:204B0000497A00290BD0002A08D10120787005E0A97F002903D0002A00D17E7001207978BE
:204B20002B23594349198B7F034311D0002A22D12A22A01C1F3106F084F966700420207086
:204B40000120A07078782B2148434019867712E02878012801D00020F8BD002A0BD16670CA
:204B6000132020701C22A91CA01C06F06AF9A6712E70DD48C6770120F8BDD94801780029AA
:204B800001D080887047D9487047F8B5D44E0746B07F00282DD13846FEF7DCFE00210125A8
:204BA000D34C072824D202007A441279921897440305081F1F1F0A00217006E025702172CB
:204BC00008E0032000E002202070CA493846FEF715FF20723846FEF7DAFE6070C649384664
:204BE000FEF7C1FEBD4CC54F20787F2807D101E02172F8BDFF20C2A1543006F0ACFA20786A
:204C000038707F202070B577032002F0E7FEF8BD10B5002002F072FE002812D0FBF79CFB08
:204C200000210120FBF7A0FABA48FBF7ACFBAE4CA06AFBF7ABFB2079032805D0022803D0D9
:204C400006E000F0F3FD10BD01210020FBF716FCFBF7FBFBB04C6078002803D0FBF77DFF56
:204C6000FBF7D9FB0320E07010BD70B59E490028CA8D08D0FF2A0DD25004000CC885FF28EF
:204C800008D9FF2005E0012A04D95008C88501D10120C88591484268012A01D0002A01D1C7
:204CA0000D224260D24317239B4C5A43637B3B25DB436B43D2184260C98D900C06F02AF9AF
:204CC000617370BDF8B5944CE078022804D0E078012801D00C20F8BD0020814A05462B213B
:204CE000414389188D77401CC0B20228F7D315706078002804D0FBF796FBFBF73FFF6570E8
:204D0000794845778577C5778449257001228A770571A570CA760A774A77714E01463246CD
:204D2000736F7432B46FF66FD7688B60CC600E614F6112698A6105770020F8BD10B5764AB2
:204D40000023D3701371684B596318630120D070FFF7B8FF002803D069A1714806F0FBF9C9
:204D600010BDF1B582B00C2001906B480090C078012806D00098C078022802D00C2003B0AC
:204D8000F0BDFBF7F0FA0020FBF7B1F8564C207F002837D0524920460F4682687437C36849
:204DA000056946694A678B67CD67FE608069386100266677A677594DE87E002805D1287F4E
:204DC000002802D1687F00281AD000980078002816D02079032802D0022805D008E005211E
:204DE000504800F040FD03E003214E4800F03BFDA97E3846FBF7F3F80020019026770CE06D
:204E0000267703E00098C078022804D00098C078022828D00AE0002001900098C0780128BE
:204E200004D10099087300980221C170606B0178002903D00178001DFBF714F9206B0178C4
:204E4000002906D0384A401CFBF777FE0099012048700298A0623548FBF717FAFBF78EFA06
:204E6000019803B0F0BD00990120C8700C2003B0F0BD70B5FBF777FA274CE078022803D06B
:204E8000FBF77CFA0C2070BD012017496073C8850220FBF765FA2648FBF739F9254E002513
:204EA000A0780321401C06F035F8A170885D012844D06D1CEDB2032DF2D3FFF7A9FE2079B1
:204EC000002809D0012807D002283DD003283BD00BA1194806F03FF9002070BDD0000020EC
:204EE000B41E0020F41E0020341F0020FFFF0000D41E0020DD1E0020D61E0020FC1E0020A2
:204F00007372635C6C6C5F64645F7363616E2E63000000006C1F0020541F0020141F0020C8
:204F200051030000941F00206F1F00204CB4010052B401002F1F0020EA030000C8B2FC497A
:204F4000085CFBF7F6F8B8E7EEF762F8C4E770B5F84C0125A577E37F002B01D03A2070BDF4
:204F60000026002802D1A07B884209D1A17366771146F14806F0EBF96577F04805702577D1
:204F8000A677002070BD024600200123E949002A03D0012A03D0122070478B7400E088742A
:204FA0000B774A767047E34A032800D1516110760120107700207047E049012803D00328C8
:204FC00001D0002000E0012008717047D948017F002903D0407E002803D1704740790028C0
:204FE000FBD00120704710B5FBF709FAFBF7FCF9FBF708F9FBF7AAF9D04C6078002805D0F4
:20500000FBF711FAFBF7BAFD00206070012020730220E070FBF7B2F9002010BDC749487181
:20502000704710B500F002FC10BDF0B5C44EC34D83B0002810D0C348FEF766FD002804D1D7
:20504000C048FEF781FD002806D0BA4C207903280DD1A07F00280AD0E87805286BD2010043
:205060007944097949188F44666666F7F600E87805287AD201007944097949188F44757567
:205080007502EE00AF48FEF765FCAD498870AE480190807F002803D1FBF736F8002800D0D6
:2050A000012000906878002813D00526761EF6B2FBF785FD0746022805D1002EF6D1A3494B
:2050C000A34806F048F80098002810D1012F0ED000909B4F9F4EB878072871D20100794439
:2050E000097949188F446DFE056C6C6C28000120EEE76878002803D0FBF795F9FBF73EFDA0
:205100008F48FBF7ABF9002801D17F203870FBF793F9009800280AD02079012801D002280C
